:020000040800F2
:1000000000000220A17A00086179000869790008DF
:1000100071790008797900088179000800000000F2
:10002000000000000000000000000000F16C00086B
:100030008979000800000000416F000897790008E6
:10004000F17A0008F17A0008F17A0008F17A0008E4
:10005000F17A0008F17A0008F17A0008F17A0008D4
:10006000F17A0008F17A0008B1790008F17A000805
:10007000F17A0008F17A0008F17A0008F17A0008B4
:10008000F17A0008F17A0008F17A0008F17A0008A4
:10009000C1790008D5790008F17A0008E9790008EB
:1000A000F17A0008F17A0008F17A0008F17A000884
:1000B000F17A0008F17A0008F17A0008F17A000874
:1000C000F17A0008F17A0008F17A0008F17A000864
:1000D000F17A0008F17A0008F17A0008F17A000854
:1000E000F17A0008F17A0008F17A0008F17A000844
:1000F000F17A0008F17A0008F17A0008F17A000834
:10010000F17A0008F17A0008F17A0008F17A000823
:10011000F17A0008F17A0008F17A0008F17A000813
:1001200021CF0008F9790008F17A00080D7A00085B
:10013000F17A0008F17A0008F17A0008F17A0008F3
:10014000F17A0008F17A0008F17A0008F17A0008E3
:10015000F17A0008217A0008F17A0008357A00085F
:10016000F17A0008F17A0008F17A0008F17A0008C3
:10017000F17A0008F17A0008F17A00080000000026
:08018000F17A0008F17A000891
:1001900053B94AB9002908BF00281CBF4FF0FF31EE
:1001A0004FF0FF3000F00CB8ADF1080C6DE904CE53
:1001B0000DF046FFDDF804E0DDE9022304B07047EE
:1001C000704700BF0348044B834202D0034B03B186
:1001D00018477047AC000020AC0000200000000071
:1001E0000548064B1B1AD90F01EBA301491002D099
:1001F000034B03B118477047AC000020AC0000204F
:100200000000000010B5064C237843B9FFF7DAFF71
:10021000044B13B10448AFF300800123237010BDD9
:10022000AC00002000000000FCE2000808B5054B0F
:100230001BB105490548AFF30080BDE80840FFF752
:10024000CFBF00BF00000000B0000020FCE20008AB
:1002500080B400AF064BD3F88830054A43F47003EE
:10026000C2F8883000BFBD465DF8047B704700BF10
:1002700000ED00E080B584B000AF78607B68002BB3
:1002800001D10123EDE07B6893F82030DBB2002B35
:1002900002D1786807F0F0F87B681B681A687B6801
:1002A0001B6842F001021A6002F036FAF86012E0B0
:1002B00002F032FA0246FB68D31A0A2B0BD97B688C
:1002C0005B6A43F400327B685A627B68052283F8DC
:1002D00020200123C5E07B681B685B6803F00103F5
:1002E000002BE5D07B681B681A687B681B6822F0CE
:1002F00002021A6002F010FAF86012E002F00CFA42
:100300000246FB68D31A0A2B0BD97B685B6A43F45D
:1003100000327B685A627B68052283F82020012323
:100320009FE07B681B685B6803F00203002BE5D14C
:100330007B681B7E012B08D17B681B681A687B6871
:100340001B6842F080021A6007E07B681B681A682D
:100350007B681B6822F080021A607B685B7E012B41
:1003600008D17B681B681A687B681B6842F04002F2
:100370001A6007E07B681B681A687B681B6822F0BC
:1003800040021A607B689B7E012B08D17B681B684A
:100390001A687B681B6842F020021A6007E07B68DD
:1003A0001B681A687B681B6822F020021A607B6851
:1003B000DB7E012B08D17B681B681A687B681B6891
:1003C00022F010021A6007E07B681B681A687B68DD
:1003D0001B6842F010021A607B681B7F012B08D15A
:1003E0007B681B681A687B681B6842F008021A6009
:1003F00007E07B681B681A687B681B6822F00802AC
:100400001A607B685B7F012B08D17B681B681A68C8
:100410007B681B6842F004021A6007E07B681B6877
:100420001A687B681B6822F004021A607B689A686D
:100430007B68DB681A437B681B691A437B685B69CE
:1004400042EA03017B685B685A1E7B681B680A43AB
:10045000DA617B6800225A627B68012283F82020DF
:10046000002318461037BD4680BD000080B487B019
:1004700000AF786039607B6893F82030FB75FB7DB6
:10048000012B03D0FB7D022B40F0BE80654B3B610E
:100490003B69D3F8003243F001023B69C3F8002204
:1004A0003B69D3F8003223F47C523B69C3F8002245
:1004B0003B69D3F800223B685B6A1B021A433B6925
:1004C000C3F800223B685B6903F01F03012202FAB4
:1004D00003F3FB603B69D3F81C22FB68DB431A4043
:1004E0003B69C3F81C223B68DB69002B23D13B69C5
:1004F000D3F80C22FB68DB431A403B69C3F80C229B
:100500003B68DB6819043B685B689BB23A685269D8
:1005100019433B69483243F832103B689B68190421
:100520003B681B689AB23B685B690A433969483388
:10053000DB000B445A603B68DB69012B22D13B692D
:10054000D3F80C22FB681A433B69C3F80C223B68C2
:100550001B6819043B685B689BB23A68526919438F
:100560003B69483243F832103B689B6819043B688A
:10057000DB689AB23B685B690A4339694833DB0040
:100580000B445A603B689B69002B09D13B69D3F847
:100590000422FB68DB431A403B69C3F8042207E0EE
:1005A0003B69D3F80422FB681A433B69C3F8042271
:1005B0003B681B69002B09D13B69D3F81422FB6807
:1005C000DB431A403B69C3F8142207E03B69D3F8C8
:1005D0001422FB681A433B69C3F814223B681B6A68
:1005E000012B07D13B69D3F81C22FB681A433B69F6
:1005F000C3F81C223B69D3F8003223F001023B69A7
:10060000C3F80022002306E07B685B6A43F4802283
:100610007B685A62012318461C37BD465DF8047B8F
:10062000704700BF0064004080B584B000AF7860C0
:100630007B6893F82030DBB2012B2ED17B6802223D
:1006400083F820207B681B681A687B681B6822F08F
:1006500001021A6002F060F8F86012E002F05CF843
:100660000246FB68D31A0A2B0BD97B685B6A43F4FA
:1006700000327B685A627B68052283F820200123C0
:1006800012E07B681B685B6803F00103002BE5D177
:100690007B6800225A62002306E07B685B6A43F4B1
:1006A00000227B685A62012318461037BD4680BD80
:1006B00080B489B000AFF860B9607A603B60FB68D5
:1006C00093F82030FB77FB681B689B68BB61FB7F5E
:1006D000012B03D0FB7F022B40F0AD80BB6903F000
:1006E0008063002B0AD1BB6903F00063002B05D1A6
:1006F000BB6903F08053002B00F09580BB691B0E93
:1007000003F003037B6101227B699A403B681A6016
:10071000BB689B68002B0DD1BB681B685A05BB6882
:10072000DB68F96809681A437B6918331B010B44BD
:100730001A600FE0BB685B68DA00BB689B681A430D
:10074000BB68DB68F96809681A437B6918331B01C9
:100750000B441A60FB681968BB681A697B69183317
:100760001B010B4404331A60BB681B7D012B11D1A4
:10077000FB681A687B6918331B01134404331B6838
:10078000FA68116843F480727B6918331B010B44CB
:1007900004331A607B6807331B781A067B680633BC
:1007A0001B781B041A437B6805331B781B02134319
:1007B0007A68043212781046FA68116843EA000237
:1007C0007B691B010B4403F5C6731A607B68033316
:1007D0001B781A067B6802331B781B041A437B685C
:1007E00001331B781B0213437A6812781046FA68AB
:1007F000116843EA00027B691B010B4403F5C473D3
:100800001A60FB681A687B6918331B0113441B6864
:10081000FA68116843F001027B6918331B010B442D
:100820001A6000230EE0FB685B6A43F40012FB6869
:100830005A62012306E0FB685B6A43F48022FB688E
:100840005A62012318462437BD465DF8047B704781
:1008500080B485B000AF78600023FB607B6893F8BC
:100860002030FB72FB7A012B02D0FB7A022B1DD1C8
:100870007B681B689B6803F08063002B02D0FB68D9
:100880000133FB607B681B689B6803F00063002BEF
:1008900002D0FB680133FB607B681B689B6803F038
:1008A0008053002B02D0FB680133FB60FB681846C5
:1008B0001437BD465DF8047B704780B487B000AF45
:1008C000F860B9607A603B60FB6893F82030FB7594
:1008D000FB7D012B03D0FB7D022B40F00381BB6825
:1008E000002B0ED1FB681B68DB6803F00303002BB1
:1008F00016D1FB685B6A43F40012FB685A6201235D
:10090000F7E0FB681B681B6903F00303002B07D1AA
:10091000FB685B6A43F40012FB685A620123E8E05B
:10092000FB681A68BB681B331B0113441B6803F088
:1009300004027B689A607B689B68002B0CD1FB6883
:100940001A68BB681B331B0113441B685B0DC3F3A0
:100950000A027B681A600BE0FB681A68BB681B33ED
:100960001B0113441B68DB0823F060427B685A605C
:10097000FB681A68BB681B331B0113441B6803F038
:1009800002027B68DA60FB681A68BB681B331B01D4
:10099000134404331B6803F00803002B03D07B6867
:1009A00008221A610BE0FB681A68BB681B331B0145
:1009B000134404331B6803F00F027B681A61FB6861
:1009C0001A68BB681B331B01134404331B681B0AE2
:1009D000DAB27B689A61FB681A68BB681B331B013B
:1009E000134404331B681B0C9AB27B685A61FB6882
:1009F0001A68BB681B01134403F5DC731B68DAB289
:100A00003B681A70FB681A68BB681B01134403F546
:100A1000DC731B681A0A3B680133D2B21A70FB6898
:100A20001A68BB681B01134403F5DC731B681A0CBE
:100A30003B680233D2B21A70FB681A68BB681B01AC
:100A4000134403F5DC731B681A0E3B680333D2B200
:100A50001A70FB681A68BB681B01134403F5DE7348
:100A60001A683B680433D2B21A70FB681A68BB6814
:100A70001B01134403F5DE731B681A0A3B68053338
:100A8000D2B21A70FB681A68BB681B01134403F5E5
:100A9000DE731B681A0C3B680633D2B21A70FB680F
:100AA0001A68BB681B01134403F5DE731B681A0E3A
:100AB0003B680733D2B21A70BB68002B08D1FB68C1
:100AC0001B68DA68FB681B6842F02002DA6007E006
:100AD000FB681B681A69FB681B6842F020021A61F8
:100AE000002306E0FB685B6A43F48022FB685A62DD
:100AF000012318461C37BD465DF8047B704780B45F
:100B000085B000AF786039607B6893F82030FB7364
:100B1000FB7B012B02D0FB7B022B09D17B681B687E
:100B200059697B681B683A680A435A61002306E0EA
:100B30007B685B6A43F480227B685A620123184613
:100B40001437BD465DF8047B704780B58AB000AFAE
:100B5000786000237B627B681B685B693B627B6813
:100B60001B685B68FB617B681B689B68BB617B687B
:100B70001B68DB687B617B681B681B693B617B686A
:100B80001B689B69FB603B6A03F00103002B7CD070
:100B9000BB6903F00103002B23D07B681B68012293
:100BA0009A60BB6903F00203002B03D0786800F061
:100BB00083F916E0BB6903F00403002B04D07B6AC1
:100BC00043F400637B620CE0BB6903F00803002B75
:100BD00004D07B6A43F480537B6202E0786800F0C3
:100BE00089F9BB6903F48073002B24D07B681B68F0
:100BF0004FF480729A60BB6903F40073002B03D03A
:100C0000786800F063F916E0BB6903F48063002B99
:100C100004D07B6A43F400537B620CE0BB6903F4AD
:100C20000063002B04D07B6A43F480437B6202E0C4
:100C3000786800F069F9BB6903F48033002B24D095
:100C40007B681B684FF480329A60BB6903F4003301
:100C5000002B03D0786800F043F916E0BB6903F479
:100C60008023002B04D07B6A43F400437B620CE0BA
:100C7000BB6903F40023002B04D07B6A43F4803368
:100C80007B6202E0786800F049F93B6A03F00803F0
:100C9000002B0CD07B6903F01003002B07D07B6A7C
:100CA00043F400737B627B681B681022DA603B6A46
:100CB00003F00403002B0BD07B6903F00803002B27
:100CC00006D07B681B680822DA60786800F030F98B
:100CD0003B6A03F00203002B09D07B681B68DB68CA
:100CE00003F00303002B02D0786807F019FC3B6A7D
:100CF00003F04003002B0CD03B6903F01003002BE2
:100D000007D07B6A43F480637B627B681B68102298
:100D10001A613B6A03F02003002B0BD03B6903F000
:100D20000803002B06D07B681B6808221A617868CC
:100D300000F012F93B6A03F01003002B09D07B6826
:100D40001B681B6903F00303002B02D0786800F0D6
:100D5000F9F83B6A03F40033002B0BD0FB6903F076
:100D60001003002B06D07B681B6810225A6078683D
:100D700000F0FCF83B6A03F48033002B0BD0FB69D6
:100D800003F00803002B06D07B681B6808225A601A
:100D9000786800F0F5F83B6A03F40043002B7BD041
:100DA000FB6903F00403002B72D03B6A03F48073E9
:100DB000002B08D0FB6803F00103002B03D07B6AF3
:100DC00043F001037B623B6A03F40073002B08D0FD
:100DD000FB6803F00203002B03D07B6A43F002039D
:100DE0007B623B6A03F48063002B08D0FB6803F04E
:100DF0000403002B03D07B6A43F004037B623B6A4D
:100E000003F40063002B43D0FB6803F07003002B56
:100E10003ED0FB6803F07003602B2BD0602B2ED8E4
:100E2000502B22D0502B2AD8402B19D0402B26D81B
:100E3000302B10D0302B22D8102B02D0202B05D0F5
:100E40001DE07B6A43F008037B6219E07B6A43F094
:100E500010037B6214E07B6A43F020037B620FE0A7
:100E60007B6A43F040037B620AE07B6A43F08003C5
:100E70007B6205E07B6A43F480737B6200E000BF25
:100E80007B681B689A697B681B6822F070029A6114
:100E90007B681B6804225A607B6A002B08D07B6841
:100EA0005A6A7B6A1A437B685A62786800F072F863
:100EB00000BF2837BD4680BD80B483B000AF7860E6
:100EC00000BF0C37BD465DF8047B704780B483B02B
:100ED00000AF786000BF0C37BD465DF8047B7047FB
:100EE00080B483B000AF786000BF0C37BD465DF8BA
:100EF000047B704780B483B000AF786000BF0C37CC
:100F0000BD465DF8047B704780B483B000AF786065
:100F100000BF0C37BD465DF8047B704780B483B0DA
:100F200000AF786000BF0C37BD465DF8047B7047AA
:100F300080B483B000AF786000BF0C37BD465DF869
:100F4000047B704780B483B000AF786000BF0C377B
:100F5000BD465DF8047B704780B483B000AF786015
:100F600000BF0C37BD465DF8047B704780B483B08A
:100F700000AF786000BF0C37BD465DF8047B70475A
:100F800080B483B000AF786000BF0C37BD465DF819
:100F9000047B704780B483B000AF786000BF0C372B
:100FA000BD465DF8047B704780B586B000AF7860C1
:100FB0007B68002B01D1012367E27B681B6803F08B
:100FC0000103002B75D0884B9B6803F00C03042BA6
:100FD0000CD0854B9B6803F00C03082B12D1824B7D
:100FE0005B6803F48003B3F5800F0BD17E4B1B6865
:100FF00003F40033002B5BD07B685B68002B57D178
:10100000012342E27B685B68B3F5803F06D1764BF3
:101010001B68754A43F4803313601DE07B685B688E
:10102000B3F5A02F0CD1704B1B686F4A43F480239B
:1010300013606D4B1B686C4A43F4803313600BE004
:10104000694B1B68684A23F480331360664B1B6846
:10105000654A23F4802313607B685B68002B13D000
:1010600001F05AFB386108E001F056FB02463B698B
:10107000D31A642B01D9032307E25B4B1B6803F4EB
:101080000033002BF0D014E001F046FB386108E09B
:1010900001F042FB02463B69D31A642B01D90323BA
:1010A000F3E1514B1B6803F40033002BF0D100E057
:1010B00000BF7B681B6803F00203002B63D04A4B20
:1010C0009B6803F00C03002B0BD0474B9B6803F08D
:1010D0000C03082B1CD1444B5B6803F48003002BEA
:1010E00016D1414B1B6803F00203002B05D07B682F
:1010F000DB68012B01D00123C7E13B4B1B6823F0C8
:10110000F8027B681B69DB00374913430B603AE048
:101110007B68DB68002B20D0344B01221A6001F081
:10112000FBFA386108E001F0F7FA02463B69D31A8E
:10113000022B01D90323A8E12B4B1B6803F0020308
:10114000002BF0D0284B1B6823F0F8027B681B694A
:10115000DB00254913430B6015E0244B00221A6085
:1011600001F0DAFA386108E001F0D6FA02463B698C
:10117000D31A022B01D9032387E11B4B1B6803F011
:101180000203002BF0D17B681B6803F00803002BDF
:1011900036D07B685B69002B16D0154B01221A6094
:1011A00001F0BAFA386108E001F0B6FA02463B698C
:1011B000D31A022B01D9032367E10B4B5B6F03F0BA
:1011C0000203002BF0D01BE0094B00221A6001F053
:1011D000A3FA38610EE001F09FFA02463B69D31A88
:1011E000022B07D9032350E1003802400000474298
:1011F000800E4742884B5B6F03F00203002BEAD15D
:101200007B681B6803F00403002B00F09780002329
:10121000FB75814B1B6C03F08053002B0FD1002317
:10122000BB607D4B1B6C7C4A43F0805313647A4B4C
:101230001B6C03F08053BB60BB680123FB75774BCD
:101240001B6803F48073002B18D1744B1B68734A1E
:1012500043F48073136001F05FFA386108E001F035
:101260005BFA02463B69D31A022B01D903230CE136
:101270006A4B1B6803F48073002BF0D07B689B687B
:10128000012B06D1644B1B6F634A43F001031367C4
:101290001CE07B689B68052B0CD15F4B1B6F5E4A83
:1012A00043F0040313675C4B1B6F5B4A43F001037D
:1012B00013670BE0584B1B6F574A23F0010313676A
:1012C000554B1B6F544A23F0040313677B689B68DC
:1012D000002B15D001F020FA38610AE001F01CFA69
:1012E00002463B69D31A41F28832934201D9032363
:1012F000CBE0494B1B6F03F00203002BEED014E050
:1013000001F00AFA38610AE001F006FA02463B6988
:10131000D31A41F28832934201D90323B5E03E4B00
:101320001B6F03F00203002BEED1FB7D012B05D1D7
:10133000394B1B6C384A23F0805313647B689B69DC
:10134000002B00F0A180344B9B6803F00C03082BAA
:101350005CD07B689B69022B41D1314B00221A6023
:1013600001F0DAF9386108E001F0D6F902463B698C
:10137000D31A022B01D9032387E0274B1B6803F004
:101380000073002BF0D17B68DA697B681B6A1A4313
:101390007B685B6A9B011A437B689B6A5B08013B25
:1013A0001B041A437B68DB6A1B061B4913434B6013
:1013B0001B4B01221A6001F0AFF9386108E001F01F
:1013C000ABF902463B69D31A022B01D903235CE037
:1013D000114B1B6803F00073002BF0D054E0104B4E
:1013E00000221A6001F098F9386108E001F094F9E0
:1013F00002463B69D31A022B01D9032345E0064B71
:101400001B6803F00073002BF0D13DE07B689B6903
:10141000012B07D1012338E0003802400070004062
:10142000600047421B4B5B68FB607B689B69012B3C
:1014300028D0FB6803F480027B68DB699A4221D1E3
:10144000FB6803F03F027B681B6A9A421AD1FA6874
:1014500047F6C07313407A68526A9201934211D1E1
:10146000FB6803F440327B689B6A5B08013B1B040A
:101470009A4207D1FB6803F070627B68DB6A1B0647
:101480009A4201D0012300E0002318461837BD46D8
:1014900080BD00BF0038024080B584B000AF7860E6
:1014A00039607B68002B01D10123CCE0684B1B68BD
:1014B00003F007033A689A420CD9654B3A68D2B2F6
:1014C0001A70634B1B6803F007033A689A4201D015
:1014D0000123B8E07B681B6803F00203002B20D0D7
:1014E0007B681B6803F00403002B05D0594B9B68F5
:1014F000584A43F4E05393607B681B6803F0080389
:10150000002B05D0534B9B68524A43F460439360D1
:10151000504B9B6823F0F0027B689B684D49134356
:101520008B607B681B6803F00103002B44D07B6851
:101530005B68012B07D1474B1B6803F40033002B7A
:1015400019D101237FE07B685B68022B03D07B68A5
:101550005B68032B07D13F4B1B6803F00073002B24
:1015600009D101236FE03B4B1B6803F00203002B02
:1015700001D1012367E0374B9B6823F003027B68AE
:101580005B68344913438B6001F0C6F8F8600AE0E9
:1015900001F0C2F80246FB68D31A41F28832934246
:1015A00001D903234FE02B4B9B6803F00C027B68AF
:1015B0005B689B009A42EBD1254B1B6803F0070345
:1015C0003A689A420CD2224B3A68D2B21A70204B37
:1015D0001B6803F007033A689A4201D0012332E006
:1015E0007B681B6803F00403002B08D0194B9B6831
:1015F00023F4E0527B68DB68164913438B607B68F9
:101600001B6803F00803002B09D0124B9B6823F4DE
:1016100060427B681B69DB000E4913438B6000F05E
:1016200021F802460B4B9B681B0903F00F030A4984
:10163000CB5C22FA03F3094A1360094B1B68184676
:1016400001F026F8002318461037BD4680BD00BFC4
:10165000003C02400038024064E300080000002023
:10166000040000202DE9B04F90B000AF00237B6351
:101670000023FB6300233B630023BB63594B9B6840
:1016800003F00C03082B0DD0082B00F2A180002BD7
:1016900002D0042B03D09BE0534BBB639BE0534B26
:1016A000BB6398E04F4B5B6803F03F037B634D4B9C
:1016B0005B6803F48003002B28D04A4B5B689B09CE
:1016C00000223B627A623B6AC3F308000021474B69
:1016D00003FB01F2002300FB03F31344434AA0FB86
:1016E0000212FA620A46BA62FA6A1344FB627B6B20
:1016F0000022BB61FA61D7E90623D7E90A01FEF7A8
:1017000047FD02460B461346FB6353E0354B5B68CF
:101710009B0900223B617A613B69C3F3080A4FF0E1
:10172000000B52465B464FF000004FF0000159019C
:1017300041EAD261500102460B46B2EB0A0863EB64
:101740000B094FF000024FF000034FEA891343EA00
:1017500098634FEA8812B2EB080463EB09054FF077
:1017600000024FF00003EB0043EA5473E20014461A
:101770001D4614EB0A033B6045EB0B037B604FF007
:1017800000024FF00003D7E9004529468B022146AD
:1017900043EA915321468A02104619467B6B002288
:1017A000BB60FA60D7E90223FEF7F2FC02460B4663
:1017B0001346FB630B4B5B681B0C03F00303013305
:1017C0005B003B63FA6B3B6BB2FBF3F3BB6302E082
:1017D000054BBB6300BFBB6B18464037BD46BDE839
:1017E000B08F00BF003802400024F400001BB70097
:1017F00080B400AF034B1B681846BD465DF8047B00
:10180000704700BF0000002080B500AFFFF7F0FF79
:101810000246054B9B689B0A03F007030349CB5C18
:1018200022FA03F3184680BD0038024074E3000832
:1018300080B500AFFFF7DCFF0246054B9B685B0BF2
:1018400003F007030349CB5C22FA03F3184680BD7B
:101850000038024074E3000880B489B000AF7860BB
:10186000396000237B6100233B610023BB610023BF
:10187000FB616BE10122FB6902FA03F37B613B68C8
:101880001B687A6913403B613A697B699A4240F070
:101890005A813B685B6803F00303012B05D03B686A
:1018A0005B6803F00303022B30D17B689B68BB614C
:1018B000FB695B00032202FA03F3DB43BA691340BE
:1018C000BB613B68DA68FB695B0002FA03F3BA6943
:1018D0001343BB617B68BA699A607B685B68BB61D4
:1018E0000122FB6902FA03F3DB43BA691340BB61CF
:1018F0003B685B681B0903F00102FB6902FA03F312
:10190000BA691343BB617B68BA695A603B685B681C
:1019100003F00303032B17D07B68DB68BB61FB6913
:101920005B00032202FA03F3DB43BA691340BB6195
:101930003B689A68FB695B0002FA03F3BA691343D8
:10194000BB617B68BA69DA603B685B6803F00303DC
:10195000022B23D1FB69DA087B68083253F8223066
:10196000BB61FB6903F007039B000F2202FA03F33C
:10197000DB43BA691340BB613B681A69FB6903F03A
:1019800007039B0002FA03F3BA691343BB61FB69C7
:10199000DA087B680832B96943F822107B681B6853
:1019A000BB61FB695B00032202FA03F3DB43BA6904
:1019B0001340BB613B685B6803F00302FB695B009B
:1019C00002FA03F3BA691343BB617B68BA691A6010
:1019D0003B685B6803F44033002B00F0B4800023C5
:1019E000FB60604B5B6C5F4A43F4804353645D4B28
:1019F0005B6C03F48043FB60FB685B4AFB699B08FC
:101A0000023352F82330BB61FB6903F003039B00F0
:101A10000F2202FA03F3DB43BA691340BB617B6810
:101A2000524A93422BD07B68514A934225D07B681F
:101A3000504A93421FD07B684F4A934219D07B682B
:101A40004E4A934213D07B684D4A93420DD07B6837
:101A50004C4A934207D07B684B4A934201D10723FB
:101A60000EE008230CE006230AE0052308E0042327
:101A700006E0032304E0022302E0012300E0002348
:101A8000FA6902F0030292009340BA691343BB6102
:101A90003549FB699B080233BA6941F823203B4B67
:101AA0009B68BB613B69DB43BA691340BB613B6820
:101AB0005B6803F48013002B03D0BA693B691343BE
:101AC000BB61324ABB699360304BDB68BB613B69E9
:101AD000DB43BA691340BB613B685B6803F40013E6
:101AE000002B03D0BA693B691343BB61274ABB692A
:101AF000D360264B5B68BB613B69DB43BA6913402B
:101B0000BB613B685B6803F40033002B03D0BA6908
:101B10003B691343BB611D4ABB6953601B4B1B6888
:101B2000BB613B69DB43BA691340BB613B685B68DF
:101B300003F48033002B03D0BA693B691343BB61C4
:101B4000124ABB691360FB690133FB61FB690F2B10
:101B50007FF690AE00BF00BF2437BD465DF8047B22
:101B6000704700BF003802400038014000000240CA
:101B70000004024000080240000C02400010024035
:101B80000014024000180240001C0240003C0140CA
:101B900080B485B000AF78600B467B807B681A69A3
:101BA0007B881340002B02D00123FB7301E000234C
:101BB000FB73FB7B18461437BD465DF8047B70470A
:101BC00080B483B000AF78600B467B8013467B7097
:101BD0007B78002B03D07A887B689A6103E07B884E
:101BE0001A047B689A6100BF0C37BD465DF8047B20
:101BF0007047000080B582B000AF0346FB80084B01
:101C00005A69FB881340002B06D0054AFB885361B4
:101C1000FB8818460BF04EF800BF0837BD4680BD64
:101C2000003C014080B586B000AF786000237B6146
:101C300000F072FD38617B68002B01D1012399E02F
:101C40007B68022283F835207B68002283F83420E9
:101C50007B681B681A687B681B6822F001021A60A7
:101C60000FE000F059FD02463B69D31A052B08D955
:101C70007B6820225A657B68032283F83520032382
:101C800078E07B681B681B6803F00103002BE8D138
:101C90007B681B681B687B617A69384B13407B61EA
:101CA0007B685A687B689B681A437B68DB681A43C9
:101CB0007B681B691A437B685B691A437B689B6975
:101CC0001A437B68DB691A437B681B6A13437A6992
:101CD00013437B617B685B6A042B07D17B68DA6AFC
:101CE0007B681B6B13437A6913437B617B681B68BA
:101CF0007A691A607B681B685B697B617B6923F08A
:101D000007037B617B685B6A7A6913437B617B684D
:101D10005B6A042B17D17B689B6A7A6913437B61EA
:101D20007B68DB6A002B0ED0786800F001FB03466D
:101D3000002B08D07B6840225A657B68012283F81B
:101D40003520012316E07B681B687A695A61786840
:101D500000F0B8FA0346FB607B68DB6D3F229A40D7
:101D6000FB689A607B6800225A657B68012283F8D1
:101D70003520002318461837BD4680BD3F8010F03F
:101D800080B586B000AFF860B9607A603B60002330
:101D9000FB75FB689B6D3B61FB6893F83430012B4E
:101DA00001D1022340E0FB68012283F83420FB6864
:101DB00093F83530DBB2012B2FD1FB68022283F878
:101DC0003520FB6800225A653B687A68B968F86874
:101DD00000F04AFAFB68DB6D3F229A403B699A604B
:101DE000FB681B681A68FB681B6842F016021A60E1
:101DF000FB681B6C002B07D0FB681B681A68FB682C
:101E00001B6842F008021A60FB681B681A68FB68CE
:101E10001B6842F001021A6005E0FB68002283F8AB
:101E200034200223FB75FB7D18461837BD4680BD64
:101E300080B584B000AF78607B689B6DFB6000F07C
:101E40006BFCB8607B6893F83530DBB2022B08D0AE
:101E50007B6880225A657B68002283F83420012346
:101E600052E07B681B681A687B681B6822F01602C8
:101E70001A607B681B685A697B681B6822F08002C5
:101E80005A617B681B6C002B03D17B689B6C002B19
:101E900007D07B681B681A687B681B6822F0080201
:101EA0001A607B681B681A687B681B6822F0010255
:101EB0001A6013E000F030FC0246BB68D31A052B11
:101EC0000CD97B6820225A657B68032283F8352071
:101ED0007B68002283F83420032315E07B681B68AD
:101EE0001B6803F00103002BE4D17B68DB6D3F220C
:101EF0009A40FB689A607B68012283F835207B68F2
:101F0000002283F83420002318461037BD4680BDD8
:101F100080B483B000AF78607B6893F83530DBB273
:101F2000022B04D07B6880225A6501230CE07B6879
:101F3000052283F835207B681B681A687B681B685C
:101F400022F001021A60002318460C37BD465DF8E6
:101F5000047B704780B586B000AF78600023BB601B
:101F60008E4B1B688E4AA2FB03239B0A7B617B6816
:101F70009B6D3B613B691B68FB607B68DB6D0822E6
:101F80009A40FB681340002B1AD07B681B681B68C3
:101F900003F00403002B13D07B681B681A687B686E
:101FA0001B6822F004021A607B68DB6D08229A40ED
:101FB0003B699A607B685B6D43F001027B685A6500
:101FC0007B68DB6D01229A40FB681340002B12D026
:101FD0007B681B685B6903F08003002B0BD07B6878
:101FE000DB6D01229A403B699A607B685B6D43F030
:101FF00002027B685A657B68DB6D04229A40FB68AD
:102000001340002B12D07B681B681B6803F002038F
:10201000002B0BD07B68DB6D04229A403B699A60F1
:102020007B685B6D43F004027B685A657B68DB6DFF
:1020300010229A40FB681340002B43D07B681B683A
:102040001B6803F00803002B3CD07B68DB6D10227B
:102050009A403B699A607B681B681B6803F4802385
:10206000002B18D07B681B681B6803F40023002B2F
:1020700008D17B681B6C002B24D07B681B6C7868B4
:1020800098471FE07B689B6C002B1BD07B689B6C88
:102090007868984716E07B681B681B6803F48073B8
:1020A000002B07D17B681B681A687B681B6822F0CD
:1020B00008021A607B681B6C002B03D07B681B6CCA
:1020C000786898477B68DB6D20229A40FB68134054
:1020D000002B00F08F807B681B681B6803F01003E7
:1020E000002B00F087807B68DB6D20229A403B69E3
:1020F0009A607B6893F83530DBB2052B36D17B686C
:102100001B681A687B681B6822F016021A607B68DD
:102110001B685A697B681B6822F080025A617B68E1
:102120001B6C002B03D17B689B6C002B07D07B685A
:102130001B681A687B681B6822F008021A607B68BB
:10214000DB6D3F229A403B699A607B68012283F8ED
:1021500035207B68002283F834207B681B6D002BC0
:102160007ED07B681B6D7868984779E07B681B6838
:102170001B6803F48023002B1DD07B681B681B6841
:1021800003F40023002B0DD17B685B6C002B31D056
:102190007B685B6C786898472CE000BF00000020EB
:1021A000B5814E1B7B68DB6B002B23D07B68DB6B20
:1021B000786898471EE07B681B681B6803F480738F
:1021C000002B0FD17B681B681A687B681B6822F0A4
:1021D00010021A607B68012283F835207B68002298
:1021E00083F834207B68DB6B002B03D07B68DB6BD0
:1021F000786898477B685B6D002B32D07B685B6D9D
:1022000003F00103002B22D07B68052283F83520E0
:102210007B681B681A687B681B6822F001021A60E1
:10222000BB680133BB607A699A4207D37B681B683D
:102230001B6803F00103002BF2D100E000BF7B68B4
:10224000012283F835207B68002283F834207B68E4
:10225000DB6C002B05D07B68DB6C7868984700E06E
:1022600000BF1837BD4680BD80B485B000AFF860B0
:10227000B9607A603B60FB681B681A68FB681B6882
:1022800022F480221A60FB681B683A685A60FB6877
:102290009B68402B08D1FB681B687A689A60FB68D2
:1022A0001B68BA68DA6007E0FB681B68BA689A6066
:1022B000FB681B687A68DA6000BF1437BD465DF8BA
:1022C000047B704780B485B000AF78607B681B6882
:1022D000DBB2103B144AA2FB03231B09FB60134A29
:1022E000FB6813441B781A467B68DA65FB68032B8E
:1022F00009D97B681B6823F47F7323F003031A1D3D
:102300007B689A6507E07B681B6823F47F7323F082
:1023100003037A6893657B689B6D18461437BD4646
:102320005DF8047B704700BFABAAAAAA7CE3000853
:1023300080B485B000AF78600023FB737B689B6A34
:10234000BB607B689B69002B1FD1BB68032B56D8F1
:1023500001A252F823F000BF692300087B23000884
:1023600069230008FF2300087B68DB6A03F08073A1
:10237000002B46D00123FB7343E07B68DB6AB3F19B
:10238000C07F40D10123FB733DE07B689B69B3F5BF
:10239000005F21D1BB68032B37D801A252F823F08C
:1023A000B1230008B7230008B1230008C92300089F
:1023B0000123FB7330E07B68DB6A03F08073002B42
:1023C00025D00123FB7322E07B68DB6AB3F1C07F79
:1023D0001FD10123FB731CE0BB68022B03D9BB6830
:1023E000032B03D018E00123FB7315E07B68DB6A45
:1023F00003F08073002B0ED00123FB730BE000BFB2
:102400000AE000BF08E000BF06E000BF04E000BF34
:1024100002E000BF00E000BFFB7B18461437BD465A
:102420005DF8047B704700BF80B485B000AF786072
:102430007B6803F00703FB600C4BDB68BB60BA688A
:102440004FF6FF031340BB60FB681A02BB681343DF
:1024500043F0BF6343F40033BB60044ABB68D360FE
:1024600000BF1437BD465DF8047B704700ED00E007
:1024700080B400AF044BDB681B0A03F00703184667
:10248000BD465DF8047B704700ED00E080B483B08A
:1024900000AF0346FB7197F90730002B0BDBFB798C
:1024A00003F01F02074997F907305B09012000FA82
:1024B00002F241F8232000BF0C37BD465DF8047BD3
:1024C000704700BF00E100E080B483B000AF034676
:1024D0003960FB7197F90730002B0ADB3B68DAB2F1
:1024E0000C4997F907301201D2B20B4483F800234C
:1024F0000AE03B68DAB20849FB7903F00F03043BBA
:102500001201D2B20B441A7600BF0C37BD465DF8FB
:10251000047B704700E100E000ED00E080B489B08A
:1025200000AFF860B9607A60FB6803F00703FB61F5
:10253000FB69C3F10703042B28BF0423BB61FB69BC
:102540000433062B02D9FB69033B00E000237B61C7
:102550004FF0FF32BB6902FA03F3DA43BB681A405B
:102560007B699A404FF0FF317B6901FA03F3D9434D
:102570007B680B40134318462437BD465DF8047B47
:102580007047000080B582B000AF78607B68013B87
:10259000B3F1807F01D301230FE00A4A7B68013B3E
:1025A00053600F214FF0FF30FFF78EFF054B0022E5
:1025B0009A60044B07221A60002318460837BD466C
:1025C00080BD00BF10E000E080B582B000AF786051
:1025D0007868FFF729FF00BF0837BD4680BD80B58A
:1025E00086B000AF0346B9607A60FB7300237B615D
:1025F000FFF73EFF78617A68B9687869FFF78EFF68
:10260000024697F90F3011461846FFF75DFF00BFED
:102610001837BD4680BD80B582B000AF0346FB7160
:1026200097F907301846FFF731FF00BF0837BD465E
:1026300080BD80B582B000AF78607868FFF7A2FFF8
:10264000034618460837BD4680BD000080B500AF80
:102650000E4B1B680D4A43F4007313600B4B1B6851
:102660000A4A43F480631360084B1B68074A43F42B
:10267000807313600320FFF7A7FF0F2000F008F816
:1026800005F0E2F90023184680BD00BF003C02407F
:1026900080B582B000AF7860124B1A68124B1B787D
:1026A00019464FF47A73B3FBF1F3B2FBF3F3184618
:1026B000FFF7BFFF0346002B01D001230EE07B682C
:1026C0000F2B0AD8002279684FF0FF30FFF787FF01
:1026D000064A7B681360002300E001231846083790
:1026E000BD4680BD0000002008000020040000203E
:1026F00080B400AF064B1B781A46064B1B68134488
:10270000044A136000BFBD465DF8047B704700BFFC
:1027100008000020C800002080B400AF034B1B68F5
:102720001846BD465DF8047B704700BFC800002016
:1027300080B582B000AF78607B68002B01D10123A7
:102740007BE07B685B6A002B08D17B685B68B3F534
:10275000827F09D07B680022DA6105E07B68002275
:102760001A617B6800225A617B6800229A627B684A
:1027700093F85130DBB2002B06D17B68002283F83E
:102780005020786804F03EFF7B68022283F85120D5
:102790007B681B681A687B681B6822F040021A601D
:1027A0007B685B6803F482727B689B6803F4044374
:1027B0001A437B68DB6803F400631A437B681B6978
:1027C00003F002031A437B685B6903F001031A43B9
:1027D0007B689B6903F400731A437B68DB6903F031
:1027E00038031A437B681B6A03F0800342EA030143
:1027F0007B689B6A03F400527B681B680A431A607B
:102800007B689B691B0C03F004017B685B6A03F027
:1028100010027B681B680A435A607B681B68DA6990
:102820007B681B6822F40062DA617B6800225A65CB
:102830007B68012283F85120002318460837BD46E3
:1028400080BD80B58AB000AFF860B9607A607B80E7
:1028500001237B62FFF760FF3862FB6893F8513019
:10286000FB77FB685B68BB617B88FB82FB7F012B8E
:102870000CD0BB69B3F5827F06D1FB689B68002B47
:1028800002D1FB7F042B01D002237FE1BB68002B28
:1028900005D07B68002B02D07B88002B01D101235F
:1028A00074E1FB6893F85030012B01D102236DE1F4
:1028B000FB68012283F85020FB6893F85130DBB2AB
:1028C000042B03D0FB68052283F85120FB6800220B
:1028D0005A65FB687A689A63FB687A88DA87FB68CE
:1028E0007A889A87FB68BA681A63FB687A88DA86FE
:1028F000FB687A889A86FB6800221A64FB680022CB
:102900005A64FB681B681B6803F04003402B07D028
:10291000FB681B681A68FB681B6842F040021A607B
:10292000FB68DB68B3F5006F7ED1FB685B68002B4A
:1029300002D0FB8A012B6CD1FB681B6B1A88FB68E9
:102940001B68DA60FB681B6B9A1CFB681A63FB68E8
:10295000DB8E9BB2013B9AB2FB68DA8659E0FB68DA
:102960001B689B6803F00203022B1BD1FB68DB8E04
:102970009BB2002B16D07B6A012B13D1FB681B6B1B
:102980001A88FB681B68DA60FB681B6B9A1CFB6883
:102990001A63FB68DB8E9BB2013B9AB2FB68DA8656
:1029A00000237B62FB681B689B6803F00103012B1B
:1029B00019D1FB68DB8F9BB2002B14D0FB681B681E
:1029C000DA68FB689B6B92B21A80FB689B6B9A1C5F
:1029D000FB689A63FB68DB8F9BB2013B9AB2FB6892
:1029E000DA8701237B62FFF797FE02463B6AD31A20
:1029F0003A6B9A420DD83B6BB3F1FF3F09D0FB68AD
:102A0000012283F85120FB68002283F85020032321
:102A1000BCE0FB68DB8E9BB2002BA0D1FB68DB8F98
:102A20009BB2002B9BD182E0FB685B68002B02D03D
:102A3000FB8A012B71D1FB681A6BFB681B680C3396
:102A400012781A70FB681B6B5A1CFB681A63FB68D0
:102A5000DB8E9BB2013B9AB2FB68DA865DE0FB68D5
:102A60001B689B6803F00203022B1CD1FB68DB8E02
:102A70009BB2002B17D07B6A012B14D1FB681A6B19
:102A8000FB681B680C3312781A70FB681B6B5A1CAE
:102A9000FB681A63FB68DB8E9BB2013B9AB2FB6852
:102AA000DA8600237B62FB681B689B6803F00103E6
:102AB000012B19D1FB68DB8F9BB2002B14D0FB6874
:102AC0001B68DA68FB689B6BD2B21A70FB689B6B61
:102AD0005A1CFB689A63FB68DB8F9BB2013B9AB27E
:102AE000FB68DA8701237B62FFF716FE02463B6A2A
:102AF000D31A3A6B9A4203D83B6BB3F1FF3F02D132
:102B00003B6B002B09D1FB68012283F85120FB6845
:102B1000002283F85020032338E0FB68DB8E9BB251
:102B2000002B9CD1FB68DB8F9BB2002B97D13A6ABC
:102B3000396BF86800F0B6F80346002B08D0FB6844
:102B400020225A65FB68002283F8502001231DE0F3
:102B5000FB689B68002B0AD100233B61FB681B6864
:102B6000DB683B61FB681B689B683B613B69FB68FA
:102B7000012283F85120FB68002283F85020FB6873
:102B80005B6D002B01D0012300E00023184628379D
:102B9000BD4680BD80B588B000AFF860B9603B60CD
:102BA0001346FB71FFF7B8FD0246BB6A9B1A3A68F1
:102BB0001344FB61FFF7B0FDB861394B1B685B0143
:102BC0001B0DFA6902FB03F37B6155E03B68B3F12F
:102BD000FF3F51D0FFF7A0FD0246BB69D31AFA6947
:102BE0009A4202D9FB69002B3DD1FB681B685A68E9
:102BF000FB681B6822F0E0025A60FB685B68B3F573
:102C0000827F11D1FB689B68B3F5004F04D0FB684D
:102C10009B68B3F5806F07D1FB681B681A68FB6877
:102C20001B6822F040021A60FB689B6AB3F5005FE4
:102C30000FD1FB681B681A68FB681B6822F40052FE
:102C40001A60FB681B681A68FB681B6842F4005234
:102C50001A60FB68012283F85120FB68002283F888
:102C60005020032318E07B69002B02D10023FB6175
:102C700002E07B69013B7B61FB681B689A68BB686B
:102C80001340BA689A420CBF01230023DBB21A46F4
:102C9000FB799A429AD1002318462037BD4680BD61
:102CA0000000002080B588B002AFF860B9607A609B
:102CB0007B680093BB6801220221F868FFF76AFF76
:102CC0000346002B07D0FB685B6D43F02002FB68D6
:102CD0005A65032332E01B4B1B681B4AA2FB0323EC
:102CE0005B0D4FF47A7202FB03F37B61FB685B6858
:102CF000B3F5827F12D17B680093BB6800228021EC
:102D0000F868FFF747FF0346002B16D0FB685B6DA2
:102D100043F02002FB685A6503230FE07B69002B18
:102D20000AD07B69013B7B61FB681B689B6803F0F1
:102D30008003802BF2D000E000BF00231846183734
:102D4000BD4680BD00000020819F5E1680B582B028
:102D500000AF78607B68002B01D1012342E07B68E3
:102D600093F84130DBB2002B06D17B68002283F858
:102D70004020786804F03EFD7B68242283F84120DF
:102D80007B681B68DA687B681B6822F40052DA6093
:102D9000786800F09FFF7B681B681A697B681B6876
:102DA00022F490421A617B681B685A697B681B6831
:102DB00022F02A025A617B681B68DA687B681B680C
:102DC00042F40052DA607B6800225A647B68202259
:102DD00083F841207B68202283F842207B68002210
:102DE0005A63002318460837BD4680BD80B58CB0B5
:102DF00000AFF860B9601346FB80FB6893F8413080
:102E0000DBB2202B62D1BB68002B02D0FB88002BE9
:102E100001D101235BE0BA68FB681A62FB68FA889B
:102E20009A84FB68FA88DA84FB6800225A64FB689B
:102E3000212283F84120FB689B6B274ADA63FB68F9
:102E40009B6B264A1A64FB689B6B254ADA64FB6815
:102E50009B6B00221A6507F10803FB62FB68986B05
:102E6000FB6A1968FB681B6804331A46FB88FEF787
:102E700087FF0346002B08D0FB6810225A64FB68CA
:102E8000202283F84120012321E0FB681B686FF0BA
:102E900040021A60FB681B681433BB61BB6953E8CE
:102EA000003F7B617B6943F08003BB62FB681B686A
:102EB0001433BA6A7A623B62396A7A6A41E800235B
:102EC000FB61FB69002BE5D1002300E002231846DB
:102ED0003037BD4680BD00BF51350008EB350008D6
:102EE0006F37000880B58CB000AFF860B96013464A
:102EF000FB80FB6893F84230DBB2202B46D1BB68E5
:102F0000002B02D0FB88002B01D101233FE0FB689E
:102F100001221A63FB6800225A63FB881A46B968CB
:102F2000F86800F06FFC034687F82F30FB681B6BD6
:102F3000012B25D100233B61FB681B681B683B61AB
:102F4000FB681B685B683B613B69FB681B680C3373
:102F5000BB61BB6953E8003F7B617B6943F01003B1
:102F6000BB62FB681B680C33BA6A7A623B62396ADF
:102F70007A6A41E80023FB61FB69002BE5D102E09E
:102F8000012387F82F3097F82F3000E002231846EE
:102F90003037BD4680BD000080B5BAB000AF786064
:102FA0007B681B681B68C7F8E4307B681B68DB68BC
:102FB000C7F8E0307B681B685B69C7F8DC3000232A
:102FC000C7F8D8300023C7F8D430D7F8E43003F07E
:102FD0000F03C7F8D830D7F8D830002B0FD1D7F867
:102FE000E43003F02003002B09D0D7F8E03003F0E1
:102FF0002003002B03D0786800F0AEFD73E2D7F811
:10300000D830002B00F0DE80D7F8DC3003F001036D
:10301000002B06D1D7F8E03003F49073002B00F0BA
:10302000D180D7F8E43003F00103002B0BD0D7F8A0
:10303000E03003F48073002B05D07B685B6C43F0B9
:1030400001027B685A64D7F8E43003F00403002BD4
:103050000BD0D7F8DC3003F00103002B05D07B68E0
:103060005B6C43F002027B685A64D7F8E43003F0EB
:103070000203002B0BD0D7F8DC3003F00103002B48
:1030800005D07B685B6C43F004027B685A64D7F818
:10309000E43003F00803002B11D0D7F8E03003F040
:1030A0002003002B05D1D7F8DC3003F00103002BFF
:1030B00005D07B685B6C43F008027B685A647B68D0
:1030C0005B6C002B00F00A82D7F8E43003F0200399
:1030D000002B08D0D7F8E03003F02003002B02D0FB
:1030E000786800F039FD7B681B685B6903F040037A
:1030F000402B0CBF01230023DBB2C7F8D4307B6820
:103100005B6C03F00803002B03D1D7F8D430002BFD
:103110004FD0786800F044FC7B681B685B6903F063
:103120004003402B41D17B681B681433C7F89C30A7
:10313000D7F89C3053E8003FC7F89830D7F898305C
:1031400023F04003C7F8D0307B681B681433D7F8EE
:10315000D020C7F8A820C7F8A430D7F8A410D7F813
:10316000A82041E80023C7F8A030D7F8A030002BF2
:10317000D9D17B68DB6B002B13D07B68DB6B8A4A71
:103180001A657B68DB6B1846FEF7C2FE0346002B10
:1031900016D07B68DB6B1B6D7A68D26B1046984744
:1031A0000EE0786800F0CAF90AE0786800F0C6F925
:1031B00006E0786800F0C2F97B6800225A648DE16D
:1031C00000BF8BE17B681B6B012B40F06781D7F858
:1031D000E43003F01003002B00F06081D7F8E030FA
:1031E00003F01003002B00F059810023BB607B68C3
:1031F0001B681B68BB607B681B685B68BB60BB6847
:103200007B681B685B6903F04003402B40F0CE8075
:103210007B68DB6B1B685B68A7F8BE30B7F8BE3015
:10322000002B00F0A9807B689B8DB7F8BE209A42E6
:1032300080F0A2807B68B7F8BE20DA857B68DB6B04
:10324000DB69B3F5807F00F088807B681B680C33F6
:10325000C7F88830D7F8883053E8003FC7F8843083
:10326000D7F8843023F48073C7F8B8307B681B68C4
:103270000C33D7F8B820C7F89420C7F89030D7F8A7
:103280009010D7F8942041E80023C7F88C30D7F885
:103290008C30002BD9D17B681B6814337B677B6F24
:1032A00053E8003F3B673B6F23F00103C7F8B4309E
:1032B0007B681B681433D7F8B420C7F88020FB67FD
:1032C000F96FD7F8802041E80023BB67BB6F002B64
:1032D000E1D17B681B6814333B663B6E53E8003FCB
:1032E000FB65FB6D23F04003C7F8B0307B681B68BB
:1032F0001433D7F8B020FA66BB66B96EFA6E41E8AF
:1033000000237B667B6E002BE3D17B68202283F851
:1033100042207B6800221A637B681B680C33FB64C5
:10332000FB6C53E8003FBB64BB6C23F01003C7F891
:10333000AC307B681B680C33D7F8AC20BA657B6572
:10334000796DBA6D41E800233B653B6D002BE3D1FD
:103350007B68DB6B1846FEF76BFD7B6802225A63C5
:103360007B689A8D7B68DB8D9BB2D31A9BB2194622
:10337000786805F01BFBB3E07B689B8DB7F8BE2037
:103380009A4240F0AD807B68DB6BDB69B3F5807FF0
:1033900040F0A6807B6802225A637B689B8D1946A9
:1033A000786805F003FB9BE0673A00087B689A8D1C
:1033B0007B68DB8D9BB2D31AA7F8CE307B68DB8DA0
:1033C0009BB2002B00F08E80B7F8CE30002B00F0BF
:1033D00089807B681B680C33BB63BB6B53E8003F81
:1033E0007B637B6B23F49073C7F8C8307B681B68E2
:1033F0000C33D7F8C8207A643B64396C7A6C41E8A6
:103400000023FB63FB6B002BE3D17B681B68143349
:103410007B627B6A53E8003F3B623B6A23F0010317
:10342000C7F8C4307B681B681433D7F8C4203A63EC
:10343000FB62F96A3A6B41E80023BB62BB6A002B6E
:10344000E3D17B68202283F842207B6800221A6344
:103450007B681B680C333B613B6953E8003FFB60B2
:10346000FB6823F01003C7F8C0307B681B680C337F
:10347000D7F8C020FA61BB61B969FA6941E8002355
:103480007B617B69002BE3D17B6802225A63B7F82A
:10349000CE301946786805F089FA23E0D7F8E43091
:1034A00003F08003002B09D0D7F8E03003F080034D
:1034B000002B03D0786800F0E7FA14E0D7F8E43086
:1034C00003F04003002B0ED0D7F8E03003F04003A8
:1034D000002B08D0786800F027FB04E000BF02E072
:1034E00000BF00E000BFE837BD4680BD80B483B0B8
:1034F00000AF786000BF0C37BD465DF8047B7047B5
:1035000080B483B000AF786000BF0C37BD465DF873
:10351000047B704780B483B000AF786000BF0C3785
:10352000BD465DF8047B704780B483B000AF78601F
:1035300000BF0C37BD465DF8047B704780B483B094
:1035400000AF786000BF0C37BD465DF8047B704764
:1035500080B590B000AF78607B689B6BFB637B6845
:103560001B681B6803F48073002B37D1FB6B0022B0
:10357000DA84FB6B1B6814337B627B6A53E8003F81
:103580003B623B6A23F08003BB63FB6B1B68143315
:10359000BA6B3A63FB62F96A3A6B41E80023BB629B
:1035A000BB6A002BE5D1FB6B1B680C333B613B69AD
:1035B00053E8003FFB60FB6843F040037B63FB6B19
:1035C0001B680C337A6BFA61BB61B969FA6941E82F
:1035D00000237B617B69002BE5D102E0F86BFFF7EC
:1035E00085FF00BF4037BD4680BD80B584B000AFC9
:1035F00078607B689B6BFB60F868FFF781FF00BF1A
:103600001037BD4680BD80B59CB000AF78607B6848
:103610009B6BFB667B681B681B6803F48073002B45
:1036200072D1FB6E0022DA85FB6E1B680C33FB64E3
:10363000FB6C53E8003FBB64BB6C23F48073BB6638
:10364000FB6E1B680C33BA6EBA657B65796DBA6D1B
:1036500041E800233B653B6D002BE5D1FB6E1B6809
:103660001433BB63BB6B53E8003F7B637B6B23F07E
:1036700001037B66FB6E1B6814337A6E7A643B64CD
:10368000396C7A6C41E80023FB63FB6B002BE5D1BE
:10369000FB6E1B6814337B627B6A53E8003F3B621E
:1036A0003B6A23F040033B66FB6E1B6814333A6EA3
:1036B0003A63FB62F96A3A6B41E80023BB62BB6A7A
:1036C000002BE5D1FB6E202283F84220FB6E1B6BA2
:1036D000012B19D1FB6E1B680C333B613B6953E82E
:1036E000003FFB60FB6823F01003FB65FB6E1B686B
:1036F0000C33FA6DFA61BB61B969FA6941E80023DC
:103700007B617B69002BE5D1FB6E00225A63FB6E67
:103710001B6B012B06D1FB6E9B8D1946F86E05F0D5
:1037200045F902E0F86EFFF7F5FE00BF7037BD46C1
:1037300080BD80B584B000AF78607B689B6BFB6018
:10374000FB6801225A63FB681B6B012B08D1FB68E5
:103750009B8D5B089BB21946F86805F027F902E0DB
:10376000F868FFF7E1FE00BF1037BD4680BD80B5A9
:1037700084B000AF78600023FB607B689B6BBB600C
:10378000BB681B685B6903F08003802B0CBF0123BF
:103790000023DBB2FB60BB6893F84130DBB2212B26
:1037A00008D1FB68002B05D0BB680022DA84B8681A
:1037B00000F0CEF8BB681B685B6903F04003402B48
:1037C0000CBF01230023DBB2FB60BB6893F84230DF
:1037D000DBB2222B08D1FB68002B05D0BB6800228E
:1037E000DA85B86800F0DCF8BB685B6C43F0100267
:1037F000BB685A64B868FFF7A1FE00BF1037BD462A
:1038000080BD000080B598B000AFF860B960134685
:10381000FB80BA68FB689A62FB68FA889A85FB6845
:1038200000225A64FB68222283F84220FB68DB6B8B
:10383000444ADA63FB68DB6B434A1A64FB68DB6B60
:10384000424ADA64FB68DB6B00221A6507F1080361
:10385000FB65FB68D86BFB681B6804331946FB6D7E
:103860001A68FB88FEF78CFA0346002B08D0FB6829
:1038700010225A64FB68202283F8422001235DE075
:1038800000233B61FB681B681B683B61FB681B688E
:103890005B683B613B69FB681B69002B19D0FB68C7
:1038A0001B680C333B643B6C53E8003FFB63FB6BD2
:1038B00043F48073BB65FB681B680C33BA6DFA6414
:1038C000BB64B96CFA6C41E800237B647B6C002B11
:1038D000E5D1FB681B681433FB62FB6A53E8003FC9
:1038E000BB62BB6A43F001037B65FB681B68143352
:1038F0007A6DBA637B63796BBA6B41E800233B63F3
:103900003B6B002BE5D1FB681B681433BB61BB69C3
:1039100053E8003F7B617B6943F040033B65FB68F4
:103920001B6814333A6D7A623B62396A7A6A41E8FD
:103930000023FB61FB69002BE5D1002318466037AB
:10394000BD4680BD07360008333700086F370008D2
:1039500080B489B000AF78607B681B680C33FB6073
:10396000FB6853E8003FBB60BB6823F0C003FB610A
:103970007B681B680C33FA69BA617B617969BA6943
:1039800041E800233B613B69002BE5D17B682022A5
:1039900083F8412000BF2437BD465DF8047B7047A3
:1039A00080B495B000AF78607B681B680C337B6394
:1039B0007B6B53E8003F3B633B6B23F49073FB64EA
:1039C0007B681B680C33FA6C3A64FB63F96B3A6CE6
:1039D00041E80023BB63BB6B002BE5D17B681B6810
:1039E00014333B623B6A53E8003FFB61FB6923F001
:1039F0000103BB647B681B681433BA6CFA62BB6258
:103A0000B96AFA6A41E800237B627B6A002BE5D140
:103A10007B681B6B012B19D17B681B680C33FB6027
:103A2000FB6853E8003FBB60BB6823F010037B6476
:103A30007B681B680C337A6CBA617B617969BA69FF
:103A400041E800233B613B69002BE5D17B682022E4
:103A500083F842207B6800221A6300BF5437BD46BA
:103A60005DF8047B704780B584B000AF78607B68F8
:103A70009B6BFB60FB680022DA85F868FFF75EFD50
:103A800000BF1037BD4680BD80B485B000AF786000
:103A90007B6893F84130DBB2212B3ED17B689B6879
:103AA000B3F5805F14D17B681B69002B10D17B6854
:103AB0001B6AFB60FB681B881A467B681B68C2F3A5
:103AC00008025A607B681B6A9A1C7B681A6208E0CD
:103AD0007B681B6A591C7A6811621A787B681B68BC
:103AE0005A607B68DB8C9BB2013B9BB27A681946BB
:103AF000D184002B0FD17B681B68DA687B681B6858
:103B000022F08002DA607B681B68DA687B681B68D9
:103B100042F04002DA60002300E002231846143726
:103B2000BD465DF8047B704780B582B000AF786019
:103B30007B681B68DA687B681B6822F04002DA60E9
:103B40007B68202283F841207868FFF7CFFC0023B0
:103B500018460837BD4680BD80B58CB000AF786090
:103B60000023FB620023BB627B6893F84230DBB228
:103B7000222B40F0AA807B689B68B3F5805F15D14B
:103B80007B681B69002B11D17B689B6ABB627B68D9
:103B90001B685B689BB2C3F308039AB2BB6A1A80C6
:103BA0007B689B6A9A1C7B689A6224E07B689B6AAC
:103BB000FB627B689B68B3F5805F07D07B689B687E
:103BC000002B0AD17B681B69002B06D17B681B6820
:103BD0005B68DAB2FB6A1A7008E07B681B685B6896
:103BE000DBB203F07F03DAB2FB6A1A707B689B6A70
:103BF0005A1C7B689A627B68DB8D9BB2013B9BB24F
:103C00007A681946D185002B5DD17B681B68DA681C
:103C10007B681B6822F02002DA607B681B68DA6828
:103C20007B681B6822F48072DA607B681B685A69C3
:103C30007B681B6822F001025A617B68202283F8AE
:103C400042207B6800225A637B681B6B012B35D1B5
:103C50007B6800221A637B681B680C337B617B697D
:103C600053E8003F3B613B6923F010037B627B68B4
:103C70001B680C337A6A3A62FB61F9693A6A41E877
:103C80000023BB61BB69002BE5D17B681B681B6807
:103C900003F01003102B0AD10023FB607B681B6824
:103CA0001B68FB607B681B685B68FB60FB687B686C
:103CB0009B8D1946786804F079FE02E07868FFF77A
:103CC00029FC002302E0002300E0022318463037DD
:103CD000BD4680BD2DE9B04FC0B000AFC7F8F400BD
:103CE000D7F8F4301B681B6923F44050D7F8F43040
:103CF000D968D7F8F4301A6840EA01031361D7F89D
:103D0000F4309A68D7F8F4301B691A43D7F8F430C6
:103D10005B691A43D7F8F430DB691343C7F8F8300E
:103D2000D7F8F4301B68DB6823F4164121F00C014E
:103D3000D7F8F4301A68D7F8F8300B43D360D7F8C7
:103D4000F4301B685B6923F44070D7F8F43099694C
:103D5000D7F8F4301A6840EA01035361D7F8F43019
:103D60001A688F4B9A4205D0D7F8F4301A688D4BF9
:103D70009A4204D1FDF75CFDC7F8FC0003E0FDF7B3
:103D800043FDC7F8FC00D7F8F430DB69B3F5004F0A
:103D900040F00C81D7F8FC300022C7F8E830C7F8B3
:103DA000EC20D7E93A4522462B469118B9655B418C
:103DB000FB65D7E91623214612EB0108294643EBA0
:103DC00001094FF000024FF000034FEAC90343EA34
:103DD00058734FEAC80290469946234618EB0303EE
:103DE000C7F8E0302B4649EB0303C7F8E430D7F8B7
:103DF000F4305B680022C7F8D830C7F8DC20D7E978
:103E000036120B46DB183B65134642EB03037B651A
:103E1000D7E91423D7E93801FCF7BAF902460B4673
:103E2000614BA3FB02235B091C01D7F8FC30002285
:103E3000C7F8D030C7F8D420D7E9348942464B467A
:103E40009118B9645B41FB64D7E91223414612EB38
:103E5000010A494643EB010B4FF000024FF000030B
:103E60004FEACB0343EA5A734FEACA0292469B4693
:103E700043461AEB0303C7F8C8304B464BEB03032A
:103E8000C7F8CC30D7F8F4305B680022C7F8C030F0
:103E9000C7F8C420D7E930120B46DB183B64134641
:103EA00042EB03037B64D7E91023D7E93201FCF727
:103EB0006FF902460B4611463B4BA3FB01235B09FE
:103EC000642202FB03F3CB1ADB0003F13202364B10
:103ED000A3FB02235B095B0003F4F8731C44D7F8CF
:103EE000FC300022C7F8B830C7F8BC20D7E92E89CB
:103EF00042464B469118B9635B41FB63D7E90E23F9
:103F000041465118396349464B417B634FF00002EB
:103F10004FF00003D7E90CAB5946CB00514643EABA
:103F200051735146CA0010461946034642469B1833
:103F3000C7F8B0304B460A4642EB0303C7F8B4302B
:103F4000D7F8F4305B680022C7F8A830C7F8AC2077
:103F5000D7E92A120B46DB18BB62134642EB030378
:103F6000FB62D7E90A23D7E92C01FCF711F90246D5
:103F70000B460D4BA3FB02135B09642101FB03F30A
:103F8000D31ADB003233084AA2FB03235B0903F098
:103F90000702D7F8F4301B6822449A6006E100BF9C
:103FA00000100140001401401F85EB51D7F8FC3090
:103FB0000022C7F8A030C7F8A420D7E928894246D4
:103FC0004B46911839625B417B62D7E90823414631
:103FD0005418494643EB01054FF000024FF000032F
:103FE000EB0043EA5473E20014461D464346E318CF
:103FF000C7F898304B4645EB0303C7F89C30D7F819
:10400000F4305B680022C7F89030C7F894204FF076
:1040100000024FF00003D7E9244529468B002146D2
:1040200043EA917321468A00D7E92601FCF7B0F8EC
:1040300002460B46604BA3FB02235B091C01D7F829
:10404000FC300022C7F88830C7F88C20D7E92289D5
:1040500042464B469118B9615B41FB61D7E90623A3
:1040600041465118396149464B417B614FF000028E
:104070004FF00003D7E904AB5946CB00514643EA61
:1040800051735146CA0010461946034642469B18D2
:10409000C7F880304B460A4642EB0303C7F884302A
:1040A000D7F8F4305B680022BB67FA674FF0000274
:1040B0004FF00003D7E91E8949468B00414643EA89
:1040C000917341468A00D7E92001FCF761F8024666
:1040D0000B461146384BA3FB01235B09642202FB0C
:1040E00003F3CB1A1B013233334AA2FB03235B09D0
:1040F00003F0F0031C44D7F8FC3000223B677A67DA
:10410000D7E91C8942464B469118B9605B41FB6078
:10411000D7E9022341465118396049464B417B603B
:104120004FF000024FF00003D7E900AB5946CB0037
:10413000514643EA51735146CA0010461946034698
:1041400042469B18BB664B460A4642EB0303FB669E
:10415000D7F8F4305B6800223B667A664FF00002C5
:104160004FF00003D7E9188949468B00414643EADE
:10417000917341468A00D7E91A01FCF709F8024613
:104180000B460D4BA3FB02135B09642101FB03F3F8
:10419000D31A1B013233084AA2FB03235B0903F045
:1041A0000F02D7F8F4301B6822449A6000BF07F56D
:1041B0008077BD46BDE8B08F1F85EB5180B483B0DA
:1041C00000AF78607B6803F108027B685A607B6807
:1041D0004FF0FF329A607B6803F108027B68DA6077
:1041E0007B6803F108027B681A617B6800221A6011
:1041F00000BF0C37BD465DF8047B704780B483B0C8
:1042000000AF78607B6800221A6100BF0C37BD46A2
:104210005DF8047B704780B485B000AF786039608A
:104220007B685B68FB603B68FA685A60FB689A6869
:104230003B689A60FB689B683A685A60FB683A681A
:104240009A603B687A681A617B681B685A1C7B68B5
:104250001A6000BF1437BD465DF8047B704780B418
:1042600085B000AF786039603B681B68BB60BB6895
:10427000B3F1FF3F03D17B681B69FB600CE07B68F7
:104280000833FB6002E0FB685B68FB60FB685B680F
:104290001B68BA689A42F6D2FB685A683B685A6053
:1042A0003B685B683A689A603B68FA689A60FB68AA
:1042B0003A685A603B687A681A617B681B685A1CC6
:1042C0007B681A6000BF1437BD465DF8047B7047F9
:1042D00080B485B000AF78607B681B69FB607B6849
:1042E0005B687A6892689A607B689B687A685268B3
:1042F0005A60FB685B687A689A4203D17B689A6867
:10430000FB685A607B6800221A61FB681B685A1EB2
:10431000FB681A60FB681B6818461437BD465DF8D9
:10432000047B704780B584B000AF786039607B68EB
:10433000FB60FB68002B0BD14FF0500383F3118817
:10434000BFF36F8FBFF34F8FBB6000BF00BFFDE7B0
:1043500002F09AFDFB681A68FB68DB6BF968096C70
:1043600001FB03F31A44FB689A60FB6800229A631E
:10437000FB681A68FB685A60FB681A68FB68DB6BAD
:10438000013BF968096C01FB03F31A44FB68DA602E
:10439000FB68FF2283F84420FB68FF2283F8452056
:1043A0003B68002B14D1FB681B69002B1AD0FB68FB
:1043B0001033184601F056F90346002B12D00D4B6E
:1043C0004FF080521A60BFF34F8FBFF36F8F09E039
:1043D000FB6810331846FFF7F1FEFB6824331846DC
:1043E000FFF7ECFE02F082FD012318461037BD46B0
:1043F00080BD00BF04ED00E080B58EB002AFF86074
:10440000B9607A603B60FB68002B0BD14FF0500322
:1044100083F31188BFF36F8FBFF34F8FBB6200BF71
:1044200000BFFDE73B68002B0BD14FF0500383F337
:104430001188BFF36F8FBFF34F8F7B6200BF00BF48
:10444000FDE77B68002B02D0BB68002B01D0012365
:1044500000E00023002B0BD14FF0500383F31188B1
:10446000BFF36F8FBFF34F8F3B6200BF00BFFDE70D
:104470007B68002B02D1BB68002B01D1012300E037
:104480000023002B0BD14FF0500383F31188BFF3AF
:104490006F8FBFF34F8FFB6100BF00BFFDE750235D
:1044A0007B617B69502B0BD04FF0500383F3118855
:1044B000BFF36F8FBFF34F8FBB6100BF00BFFDE73E
:1044C0007B693B68FB62FB6A002B0DD0FB6A012213
:1044D00083F8462097F83820FB6A009313467A68E1
:1044E000B968F86800F040F8FB6A18463037BD46F6
:1044F00080BD80B58AB002AFF860B9601346FB7129
:10450000FB68002B0BD14FF0500383F31188BFF3EE
:104510006F8FBFF34F8F3B6100BF00BFFDE7FB68AC
:10452000BA6802FB03F3FB61FB695033184602F0E3
:104530008BF9B861BB69002B11D0BB697B617B69CA
:1045400050337B61BB69002283F84620FA79BB694E
:10455000009313467A69B968F86800F005F8BB69FA
:1045600018462037BD4680BD80B584B000AFF860E6
:10457000B9607A60FB70BB68002B03D1BB69BA6974
:104580001A6002E0BB697A681A60BB69FA68DA638C
:10459000BB69BA681A640121B869FFF7C3FEBB6939
:1045A000FA7883F84C2000BF1037BD4680BD00006C
:1045B00080B58EB000AFF860B9607A603B600023D0
:1045C0007B63FB683B633B6B002B0BD14FF05003CD
:1045D00083F31188BFF36F8FBFF34F8FBB6200BFB0
:1045E00000BFFDE7BB68002B03D13B6B1B6C002BAE
:1045F00001D1012300E00023002B0BD14FF0500329
:1046000083F31188BFF36F8FBFF34F8F7B6200BFBF
:1046100000BFFDE73B68022B03D13B6BDB6B012B3B
:1046200001D1012300E00023002B0BD14FF05003F8
:1046300083F31188BFF36F8FBFF34F8F3B6200BFCF
:1046400000BFFDE701F0CEF90346002B02D17B68E5
:10465000002B01D1012300E00023002B0BD14FF0F0
:10466000500383F31188BFF36F8FBFF34F8FFB614C
:1046700000BF00BFFDE702F007FC3B6B9A6B3B6B92
:10468000DB6B9A4202D33B68022B29D13A68B968A6
:10469000386B00F00FFAF8623B6B5B6A002B10D0AE
:1046A0003B6B2433184600F0DDFF0346002B13D08C
:1046B0003F4B4FF080521A60BFF34F8FBFF36F8FA5
:1046C0000AE0FB6A002B07D0394B4FF080521A608A
:1046D000BFF34F8FBFF36F8F02F008FC012363E03D
:1046E0007B68002B03D102F001FC00235CE07B6BB4
:1046F000002B06D107F11403184601F017F8012327
:104700007B6302F0F3FB00F087FD02F0BDFB3B6B27
:1047100093F844305BB2B3F1FF3F03D13B6B00220F
:1047200083F844203B6B93F845305BB2B3F1FF3F15
:1047300003D13B6B002283F8452002F0D7FB3A1DE2
:1047400007F114031146184601F006F80346002B42
:1047500024D1386B00F0A6FA0346002B18D03B6B2F
:1047600010337A681146184600F02AFF386B00F0C3
:1047700031FA00F05FFD0346002B7FF47CAF0C4B59
:104780004FF080521A60BFF34F8FBFF36F8F72E705
:10479000386B00F01FFA00F04DFD6CE7386B00F04D
:1047A00019FA00F047FD002318463837BD4680BD92
:1047B00004ED00E080B590B000AFF860B9607A60B9
:1047C0003B60FB68BB63BB6B002B0BD14FF050030E
:1047D00083F31188BFF36F8FBFF34F8FBB6200BFAE
:1047E00000BFFDE7BB68002B03D1BB6B1B6C002B2C
:1047F00001D1012300E00023002B0BD14FF0500327
:1048000083F31188BFF36F8FBFF34F8F7B6200BFBD
:1048100000BFFDE73B68022B03D1BB6BDB6B012BB9
:1048200001D1012300E00023002B0BD14FF05003F6
:1048300083F31188BFF36F8FBFF34F8F3B6200BFCD
:1048400000BFFDE702F000FCEFF311824FF05003D0
:1048500083F31188BFF36F8FBFF34F8FFA61BB6192
:10486000FB697B63BB6B9A6BBB6BDB6B9A4202D3BE
:104870003B68022B2FD1BB6B93F8453087F8333060
:10488000BB6B9B6BFB623A68B968B86B00F012F9BE
:1048900097F93330B3F1FF3F12D1BB6B5B6A002B4A
:1048A00016D0BB6B2433184600F0DCFE0346002B09
:1048B0000ED07B68002B0BD07B6801221A6007E0CA
:1048C00097F833300133DBB25AB2BB6B83F8452023
:1048D0000123FB6301E00023FB637B6B7B617B694E
:1048E00083F3118800BFFB6B18464037BD4680BD7F
:1048F00080B58CB000AFF860B9607A600023FB62CD
:10490000FB68BB62BB6A002B0BD14FF0500383F3F3
:104910001188BFF36F8FBFF34F8F3B6200BF00BFA3
:10492000FDE7BB68002B03D1BB6A1B6C002B01D1D8
:10493000012300E00023002B0BD14FF0500383F341
:104940001188BFF36F8FBFF34F8FFB6100BF00BFB4
:10495000FDE701F047F80346002B02D17B68002BEE
:1049600001D1012300E00023002B0BD14FF05003B5
:1049700083F31188BFF36F8FBFF34F8FBB6100BF0D
:1049800000BFFDE702F080FABB6A9B6B7B627B6A2B
:10499000002B1FD0B968B86A00F0F6F87B6A5A1E7F
:1049A000BB6A9A63BB6A1B69002B0FD0BB6A1033CA
:1049B000184600F057FE0346002B07D03C4B4FF043
:1049C00080521A60BFF34F8FBFF36F8F02F08EFAE1
:1049D000012369E07B68002B03D102F087FA0023F2
:1049E00062E0FB6A002B06D107F11003184600F0C5
:1049F0009DFE0123FB6202F079FA00F00DFC02F04B
:104A000043FABB6A93F844305BB2B3F1FF3F03D182
:104A1000BB6A002283F84420BB6A93F845305BB23E
:104A2000B3F1FF3F03D1BB6A002283F8452002F0B7
:104A30005DFA3A1D07F110031146184600F08CFE8E
:104A40000346002B23D1B86A00F016F90346002B69
:104A500017D0BB6A24337A681146184600F0B0FDBF
:104A6000B86A00F0B7F800F0E5FB0346002B89D1E7
:104A70000F4B4FF080521A60BFF34F8FBFF36F8F11
:104A800080E7B86A00F0A6F800F0D4FB7AE7B86ACD
:104A900000F0A0F800F0CEFBB86A00F0EDF8034695
:104AA000002B3FF46FAF002318463037BD4680BD62
:104AB00004ED00E080B586B000AFF860B9607A60C0
:104AC00000237B61FB689B6B3B61FB681B6C002BCD
:104AD0000DD1FB681B68002B4DD1FB689B68184605
:104AE00000F09EFF7861FB6800229A6043E07B68DB
:104AF000002B19D1FB685868FB681B6C1A46B96813
:104B000009F090FAFB685A68FB681B6C1A44FB6852
:104B10005A60FB685A68FB689B689A422BD3FB6813
:104B20001A68FB685A6026E0FB68D868FB681B6C53
:104B30001A46B96809F076FAFB68DA68FB681B6CFC
:104B40005B421A44FB68DA60FB68DA68FB681B6842
:104B50009A4207D2FB689A68FB681B6C5B421A4456
:104B6000FB68DA607B68022B05D13B69002B02D021
:104B70003B69013B3B613B695A1CFB689A637B695B
:104B800018461837BD4680BD80B582B000AF78604A
:104B900039607B681B6C002B18D07B68DA687B68F7
:104BA0001B6C1A447B68DA607B68DA687B689B68F8
:104BB0009A4203D37B681A687B68DA607B68D9689D
:104BC0007B681B6C1A46386809F02CFA00BF08375E
:104BD000BD4680BD80B584B000AF786002F054F966
:104BE0007B6893F84530FB7311E07B685B6A002BB0
:104BF00012D07B682433184600F034FD0346002BA6
:104C000001D000F00DFEFB7B013BDBB2FB7397F99B
:104C10000F30002BE9DC00E000BF7B68FF2283F847
:104C2000452002F063F902F02FF97B6893F84430D5
:104C3000BB7311E07B681B69002B12D07B681033BB
:104C4000184600F00FFD0346002B01D000F0E8FDF0
:104C5000BB7B013BDBB2BB7397F90E30002BE9DC69
:104C600000E000BF7B68FF2283F8442002F03EF999
:104C700000BF1037BD4680BD80B584B000AF7860FE
:104C800002F002F97B689B6B002B02D10123FB60D1
:104C900001E00023FB6002F029F9FB681846103799
:104CA000BD4680BD80B584B000AF786002F0ECF8FE
:104CB0007B689A6B7B68DB6B9A4202D10123FB60B5
:104CC00001E00023FB6002F011F9FB681846103781
:104CD000BD4680BD80B485B000AF786039600023E8
:104CE000FB6014E00F4AFB6852F83330002B0BD105
:104CF0000C49FB683A6841F833200A4AFB68DB003C
:104D000013447A685A6006E0FB680133FB60FB6875
:104D1000072BE7D900BF00BF1437BD465DF8047B01
:104D2000704700BFCC00002080B586B000AFF860AF
:104D3000B9607A60FB687B6102F0A6F87B6993F842
:104D400044305BB2B3F1FF3F03D17B69002283F8AB
:104D500044207B6993F845305BB2B3F1FF3F03D148
:104D60007B69002283F8452002F0C0F87B699B6BC9
:104D7000002B06D17B6924337A68B968184600F0A5
:104D800045FC7869FFF726FF00BF1837BD4680BD98
:104D900080B58EB004AFF860B9607A603B607B6B21
:104DA000002B0BD14FF0500383F31188BFF36F8FAB
:104DB000BFF34F8F3B6200BF00BFFDE7BB6B002B13
:104DC0000BD14FF0500383F31188BFF36F8FBFF304
:104DD0004F8FFB6100BF00BFFDE75C233B613B6978
:104DE0005C2B0BD04FF0500383F31188BFF36F8F10
:104DF000BFF34F8FBB6100BF00BFFDE73B69BB6BDB
:104E0000002B1ED07B6B002B1BD0BB6B7B627B6AA5
:104E10007A6B1A637B6A022283F85920002303937A
:104E20007B6A029307F1140301933B6B00933B6889
:104E30007A68B968F86800F050F8786A00F0DEF82F
:104E400001E000237B617B6918462837BD4680BDA1
:104E500080B58CB004AFF860B9603B601346FB804E
:104E6000FB889B00184601F0EFFC78617B69002B02
:104E70000ED05C2001F0E8FCF861FB69002B03D048
:104E8000FB697A691A6305E0786901F0ABFD01E01E
:104E90000023FB61FB69002B17D0FB69002283F81C
:104EA0005920FA8800230393FB690293FB6A01935C
:104EB000BB6A00933B68B968F86800F00EF8F869BF
:104EC00000F09CF80123BB6102E04FF0FF33BB61AF
:104ED000BB6918462037BD4680BD80B588B000AF9D
:104EE000F860B9607A603B603B6B186B7B689B0035
:104EF0001A46A52109F064F83B6B1A6B7B6803F135
:104F00008043013B9B001344BB61BB6923F0070353
:104F1000BB61BB6903F00703002B0BD04FF05003BC
:104F200083F31188BFF36F8FBFF34F8F7B6100BF97
:104F300000BFFDE7BB68002B1FD00023FB6112E020
:104F4000BA68FB69134419783A6BFB69134434332C
:104F50000A461A70BA68FB6913441B78002B06D006
:104F6000FB690133FB61FB690F2BE9D900E000BF4E
:104F70003B6B002283F8432003E03B6B002283F865
:104F80003420BB6A372B01D93723BB623B6BBA6A2B
:104F9000DA623B6BBA6ADA643B6B00221A653B6BE0
:104FA00004331846FFF72AF93B6B18331846FFF70E
:104FB00025F93B6B3A6B1A61BB6AC3F138023B6B54
:104FC0009A613B6B3A6B5A623B6B00225A653B6BB2
:104FD000002283F858203A68F968B86901F022FE87
:104FE00002463B6B1A60FB6A002B02D0FB6A3A6BED
:104FF0001A6000BF2037BD4680BD000080B582B07A
:1050000000AF786001F040FF2D4B1B6801332C4A44
:1050100013602C4B1B68002B09D12A4A7B68136054
:10502000274B1B68012B10D100F01EFC0DE0264B16
:105030001B68002B09D1234B1B68DA6A7B68DB6A8B
:105040009A4202D81F4A7B681360204B1B680133C9
:105050001E4A13601D4B1A687B685A647B68DA6AC3
:105060001B4B1B689A4203D97B68DB6A184A1360A2
:105070007B68DA6A13469B0013449B00154A1A4466
:105080007B68043319461046FFF7C5F801F02EFF80
:105090000D4B1B68002B0ED00A4B1B68DA6A7B682D
:1050A000DB6A9A4207D20C4B4FF080521A60BFF372
:1050B0004F8FBFF36F8F00BF0837BD4680BD00BF65
:1050C000E00500200C010020EC050020FC0500207C
:1050D000E80500201001002004ED00E080B584B058
:1050E00000AF78600023FB607B68002B18D0144B66
:1050F0001B68002B0BD04FF0500383F31188BFF3D4
:105100006F8FBFF34F8FBB6000BF00BFFDE700F0A4
:1051100083F80021786800F089FE00F08BF8F860D1
:10512000FB68002B07D1074B4FF080521A60BFF38A
:105130004F8FBFF36F8F00BF1037BD4680BD00BFDC
:105140000806002004ED00E080B58AB004AF00231B
:10515000BB6000237B603A46391D07F108031846FF
:1051600001F03EFB39687B68BA6802920193002324
:10517000009300230A4622492248FFF709FE03460E
:10518000214A1360204B1B68002B02D001237B6156
:1051900001E000237B617B69012B02D100F09AFEC4
:1051A00078617B69012B16D14FF0500383F311888E
:1051B000BFF36F8FBFF34F8F3B6100BF134B4FF0B7
:1051C000FF321A60124B01221A60124B00221A6041
:1051D00001F0B6FD0FE07B69B3F1FF3F0BD14FF05B
:1051E000500383F31188BFF36F8FBFF34F8FFB60C2
:1051F00000BF00BFFDE700BF1837BD4680BD00BF40
:1052000014E30008395800080406002000060020B6
:10521000EC050020E405002080B400AF044B1B68BF
:105220000133034A136000BFBD465DF8047B70473D
:105230000806002080B584B000AF0023FB60002387
:10524000BB60424B1B68002B0BD14FF0500383F324
:105250001188BFF36F8FBFF34F8F3B6000BF00BF5C
:10526000FDE701F011FE394B1B68013B374A136023
:10527000364B1B68002B62D1354B1B68002B5ED070
:105280002FE0344BDB68DB68FB60FB6818331846A3
:10529000FFF71EF8FB6804331846FFF719F8FB68A0
:1052A000DA6A2D4B1B689A4203D9FB68DB6A2A4AEB
:1052B0001360FB68DA6A13469B0013449B00274A7D
:1052C0001A44FB68043319461046FEF7A4FFFB6836
:1052D000DA6A234B1B68DB6A9A4202D3214B012214
:1052E0001A601C4B1B68002BCBD1FB68002B01D034
:1052F00000F058FB1C4B1B687B607B68002B10D0B8
:1053000000F046F80346002B02D0164B01221A602B
:105310007B68013B7B607B68002BF1D1124B002244
:105320001A60104B1B68002B09D00123BB600F4B88
:105330004FF080521A60BFF34F8FBFF36F8F01F0B1
:10534000D5FDBB6818461037BD4680BD0806002055
:10535000E0050020A0050020E80500201001002045
:105360000C010020F4050020F005002004ED00E011
:1053700080B483B000AF054B1B687B607B68184628
:105380000C37BD465DF8047B704700BFE405002084
:1053900080B586B000AF00237B614F4B1B68002BAC
:1053A00040F090804D4B1B6801333B614B4A3B6999
:1053B00013603B69002B21D1494B1B681B68002BF4
:1053C0000BD04FF0500383F31188BFF36F8FBFF3FF
:1053D0004F8F3B6000BF00BFFDE7414B1B68FB6088
:1053E000404B1B683E4A13603E4AFB6813603E4BCD
:1053F0001B6801333C4A136000F0D4FA3B4B1B6836
:105400003A699A4249D3364B1B681B68002B04D17A
:10541000364B4FF0FF321A603FE0314B1B68DB68C0
:10542000DB68BB60BB685B687B603A697B689A42FB
:1054300003D22E4A7B6813602FE0BB680433184602
:10544000FEF746FFBB689B6A002B04D0BB6818338D
:105450001846FEF73DFFBB68DA6A254B1B689A4287
:1054600003D9BB68DB6A224A1360BB68DA6A134659
:105470009B0013449B001F4A1A44BB68043319461F
:105480001046FEF7C8FEBB68DA6A1B4B1B68DB6A76
:105490009A42B8D301237B61B5E7174B1B68DA6AE0
:1054A000144913469B0013449B000B441B68012BBB
:1054B00001D901237B61114B1B68002B07D001230D
:1054C0007B6104E00E4B1B6801330D4A13607B695E
:1054D00018461837BD4680BD08060020E4050020A8
:1054E000980500209C050020F805002000060020FB
:1054F000E8050020100100200C010020F405002028
:10550000F005002080B485B000AF284B1B68002B4D
:1055100003D0274B01221A6042E0254B00221A607B
:10552000244B1B68FB6011E0FB68002B0BD14FF094
:10553000500383F31188BFF36F8FBFF34F8F7B60EE
:1055400000BF00BFFDE7FB68013BFB601A49FA683A
:1055500013469B0013449B000B441B68002BE3D0B5
:10556000FA6813469B0013449B00134A1344BB6024
:10557000BB685B685A68BB685A60BB685A68BB689E
:1055800008339A4204D1BB685B685A68BB685A60AA
:10559000BB685B68DB68094A1360064AFB681360F6
:1055A00000BF1437BD465DF8047B70470806002035
:1055B000F4050020E8050020100100200C01002067
:1055C00080B584B000AF786039607B68002B0BD168
:1055D0004FF0500383F31188BFF36F8FBFF34F8FEA
:1055E000FB6000BF00BFFDE7074B1B68183319467F
:1055F0007868FEF734FE0121386800F017FC00BF20
:105600001037BD4680BD00BF0C01002080B586B0BC
:1056100000AFF860B9607A60FB68002B0BD14FF0E7
:10562000500383F31188BFF36F8FBFF34F8F7B61FC
:1056300000BF00BFFDE70A4B1B6818331946F86826
:10564000FEF7E9FD7B68002B02D04FF0FF33BB6013
:105650007968B86800F0EAFB00BF1837BD4680BD26
:105660000C01002080B586B000AF78607B68DB68F5
:10567000DB683B613B69002B0BD14FF0500383F398
:105680001188BFF36F8FBFF34F8FFB6000BF00BF68
:10569000FDE73B6918331846FEF71AFE1D4B1B68E1
:1056A000002B1DD13B6904331846FEF711FE3B6900
:1056B000DA6A194B1B689A4203D93B69DB6A164ABE
:1056C00013603B69DA6A13469B0013449B00134A3C
:1056D0001A443B69043319461046FEF79CFD05E069
:1056E0003B69183319460E48FEF795FD3B69DA6AA7
:1056F0000C4B1B68DB6A9A4205D901237B610A4B7C
:1057000001221A6001E000237B617B69184618378B
:10571000BD4680BD08060020E805002010010020DD
:10572000A00500200C010020F405002080B483B007
:1057300000AF7860064B1A687B681A60054B1A68E0
:105740007B685A6000BF0C37BD465DF8047B70472C
:10575000F8050020E405002080B588B000AF78602F
:1057600039607B68002B0BD14FF0500383F3118815
:10577000BFF36F8FBFF34F8F3B6100BF00BFFDE7EB
:105780003B68002B0BD14FF0500383F31188BFF31C
:105790006F8FBFF34F8FFB6000BF00BFFDE701F0CD
:1057A00073FB1D4B1B68BB617B685B68BA69D31ACE
:1057B0007B613B681B68B3F1FF3F02D10023FB61B3
:1057C00023E07B681A68154B1B689A4207D07B68F8
:1057D0005B68BA699A4202D30123FB6115E03B681A
:1057E0001B687A699A420BD23B681A687B69D21AA5
:1057F0003B681A607868FFF799FF0023FB6104E0BB
:105800003B6800221A600123FB6101F06FFBFB691A
:1058100018462037BD4680BDE4050020F80500206D
:1058200080B400AF034B01221A6000BFBD465DF893
:10583000047B7047F405002080B582B000AF78602B
:1058400000F052F8064B1B68012BF9D9054B4FF0BD
:1058500080521A60BFF34F8FBFF36F8FF0E700BF26
:105860001001002004ED00E080B582B000AF0023FD
:105870007B600CE07A6813469B0013449B00124A3D
:1058800013441846FEF79AFC7B6801337B607B6803
:10589000372BEFD90D48FEF791FC0D48FEF78EFC33
:1058A0000C48FEF78BFC0C48FEF788FC0B48FEF713
:1058B00085FC0B4B054A1A600A4B054A1A6000BF6B
:1058C0000837BD4680BD00BF1001002070050020D4
:1058D00084050020A0050020B4050020CC05002090
:1058E000980500209C05002080B582B000AF19E02B
:1058F00001F0CAFA104BDB68DB687B607B6804331D
:105900001846FEF7E5FC0D4B1B68013B0B4A136084
:105910000B4B1B68013B0A4A136001F0E7FA7868F9
:1059200000F010F8064B1B68002BE1D100BF00BF50
:105930000837BD4680BD00BFB4050020E00500204B
:10594000C805002080B584B000AF78607B6893F80C
:105950005930002B08D17B681B6B184601F042F8C8
:10596000786801F03FF819E07B6893F85930012B13
:1059700003D1786801F036F810E07B6893F859306D
:10598000022B0BD04FF0500383F31188BFF36F8FBE
:10599000BFF34F8FFB6000BF00BFFDE700BF1037B4
:1059A000BD4680BD80B483B000AF0C4B1B681B6844
:1059B000002B04D10A4B4FF0FF321A6008E0074B6E
:1059C0001B68DB68DB687B607B685B68044A13608C
:1059D00000BF0C37BD465DF8047B7047980500207A
:1059E0000006002080B483B000AF0B4B1B68002B77
:1059F00002D101237B6008E0084B1B68002B02D119
:105A000002237B6001E000237B607B6818460C3733
:105A1000BD465DF8047B7047EC05002008060020B9
:105A200080B586B000AF78607B683B6100237B6106
:105A30007B68002B58D02F4B1B683A699A420BD0D9
:105A40004FF0500383F31188BFF36F8FBFF34F8F75
:105A5000FB6000BF00BFFDE73B691B6D002B0BD156
:105A60004FF0500383F31188BFF36F8FBFF34F8F55
:105A7000BB6000BF00BFFDE73B691B6D5A1E3B6961
:105A80001A653B69DA6A3B69DB6C9A422CD03B6948
:105A90001B6D002B28D13B6904331846FEF718FC18
:105AA0003B69DA6C3B69DA623B69DB6AC3F1380255
:105AB0003B699A613B69DA6A0F4B1B689A4203D9CA
:105AC0003B69DB6A0C4A13603B69DA6A13469B0048
:105AD00013449B00094A1A443B6904331946104693
:105AE000FEF799FB01237B617B6918461837BD4699
:105AF00080BD00BF0C010020E8050020100100203F
:105B000080B584B000AF7860396001F0BDF91E4BFC
:105B10001B685B6D002B13D11B4B1B68012283F8A4
:105B200058203B68002B0BD00121386800F07EF92B
:105B3000164B4FF080521A60BFF34F8FBFF36F8F39
:105B400001F0D4F901F0A0F90F4B1B685B6DFB600D
:105B5000FB68002B0CD07B68002B04D00A4B1B6821
:105B600000225A6504E0084B1B68FA68013A5A653E
:105B7000054B1B68002283F8582001F0B7F9FB6839
:105B800018461037BD4680BD0C01002004ED00E032
:105B900080B58AB000AFF860B9603B601346FB7116
:105BA00001237B62FB68002B0BD14FF0500383F382
:105BB0001188BFF36F8FBFF34F8FBB6100BF00BF72
:105BC000FDE7FB683B6201F05FF93B68002B03D007
:105BD0003B6A5A6D3B681A603B6A93F85830FB7712
:105BE0003B6A022283F85820FB79042B27D801A2B4
:105BF00052F823F0615C0008095C0008175C00089B
:105C0000235C00082B5C00083B6A5A6DBB681A4392
:105C10003B6A5A6527E03B6A5B6D5A1C3B6A5A65D2
:105C200021E03B6ABA685A651DE0FB7F022B03D076
:105C30003B6ABA685A6516E000237B6213E03B6A50
:105C40005B6DB3F1FF3F0DD04FF0500383F311882C
:105C5000BFF36F8FBFF34F8F7B6100BF00BFFDE7C6
:105C600000BF00E000BFFB7F012B3BD13B6A043348
:105C70001846FEF72DFB3B6ADA6A1E4B1B689A42F8
:105C800003D93B6ADB6A1B4A13603B6ADA6A134634
:105C90009B0013449B00184A1A443B6A043319467C
:105CA0001046FEF7B8FA3B6A9B6A002B0BD04FF008
:105CB000500383F31188BFF36F8FBFF34F8F3B61A6
:105CC00000BF00BFFDE73B6ADA6A0C4B1B68DB6A6A
:105CD0009A4207D90A4B4FF080521A60BFF34F8F98
:105CE000BFF36F8F01F002F97B6A18462837BD4673
:105CF00080BD00BFE8050020100100200C0100203D
:105D000004ED00E080B58AB000AF786039607B6850
:105D1000002B0BD14FF0500383F31188BFF36F8F2B
:105D2000BFF34F8FBB6100BF00BFFDE701F08CF9EF
:105D30007B687B62EFF311824FF0500383F311888D
:105D4000BFF36F8FBFF34F8F7A613B617B693B621B
:105D50007B6A93F85830FB777B6A022283F85820DD
:105D60007B6A5B6D5A1C7B6A5A65FB7F012B47D1AE
:105D70007B6A9B6A002B0BD04FF0500383F3118892
:105D8000BFF36F8FBFF34F8FFB6000BF00BFFDE716
:105D9000204B1B68002B1DD17B6A04331846FEF78D
:105DA00097FA7B6ADA6A1C4B1B689A4203D97B6AB2
:105DB000DB6A194A13607B6ADA6A13469B00134454
:105DC0009B00164A1A447B6A043319461046FEF7B4
:105DD00022FA05E07B6A183319461148FEF71BFAD0
:105DE0007B6ADA6A0F4B1B68DB6A9A4208D93B6808
:105DF000002B02D03B6801221A600B4B01221A6073
:105E00003B6ABB60BB6883F3118800BF00BF2837C3
:105E1000BD4680BD08060020E805002010010020D6
:105E2000A00500200C010020F405002080B584B0FE
:105E300000AF78603960214B1B68FB60204B1B680A
:105E400004331846FEF744FA7B68B3F1FF3F0AD1EA
:105E50003B68002B07D01A4B1B68043319461948BE
:105E6000FEF7D9F926E0FA687B681344BB60144B4F
:105E70001B68BA685A60BA68FB689A4209D2124B2A
:105E80001A680F4B1B68043319461046FEF7E7F9F2
:105E900010E00E4B1A680A4B1B6804331946104673
:105EA000FEF7DDF90A4B1B68BA689A4202D2084A2B
:105EB000BB68136000BF1037BD4680BDE4050020FD
:105EC0000C010020CC0500209C0500209805002036
:105ED0000006002080B58AB004AF00237B6100F08B
:105EE00013FB1D4B1B68002B21D00023FB600023FC
:105EF000BB603A1D07F1080107F10C03184600F0DA
:105F000089FC7968BB68FA680292019302230093C6
:105F100000230A4611491248FEF73AFF0346114A88
:105F20001360104B1B68002B01D001237B617B6940
:105F3000002B0BD14FF0500383F31188BFF36F8F09
:105F4000BFF34F8F3B6100BF00BFFDE77B69184681
:105F50001837BD4680BD00BF3C0600201CE300088A
:105F6000A16000084006002080B58AB000AFF8604C
:105F7000B9607A603B6000237B62FB68002B0BD129
:105F80004FF0500383F31188BFF36F8FBFF34F8F30
:105F90003B6200BF00BFFDE7194B1B68002B2AD0F6
:105FA000BB683B617B687B61FB68BB61BB68052BA1
:105FB00018DCFFF717FD0346022B09D1104B1868B8
:105FC00007F1100100233A6BFEF7F2FA786212E053
:105FD0000B4B186807F1100100230022FEF7E8FAC6
:105FE000786208E0064B186807F1100100233A6850
:105FF000FEF7E0FB78627B6A18462837BD4680BD15
:106000003C06002080B588B002AF78603960234B31
:106010001B68DB68DB687B617B6904331846FEF72D
:1060200057F97B6993F8283003F00403002B23D041
:106030007B699A697B68D1187B683A68786900F057
:10604000D5F80346002B20D00023009300237A6864
:1060500000217869FFF788FF38613B69002B14D174
:106060004FF0500383F31188BFF36F8FBFF34F8F4F
:10607000FB6000BF00BFFDE77B6993F8283023F089
:106080000103DAB27B6983F828207B691B6A78698F
:10609000984700BF1837BD4680BD00BF34060020BA
:1060A00080B584B000AF786007F10803184600F0AF
:1060B00059F8F860BB681946F86800F005F800F078
:1060C000D7F800BFF0E7000080B584B000AF78607B
:1060D0003960FFF7A1F807F10803184600F066F8E9
:1060E000F860BB68002B30D13B68002B0AD17A687E
:1060F000FB689A4206D8FFF79DF8F9687868FFF7C1
:1061000081FF24E03B68002B08D0134B1B681B6801
:10611000002B01D1012300E000233B600F4B1868E6
:106120007A68FB68D31A3A681946FEF7FDFDFFF757
:1061300081F80346002B0AD1094B4FF080521A60B8
:10614000BFF34F8FBFF36F8F01E0FFF773F800BF0E
:106150001037BD4680BD00BF380600203C06002039
:1061600004ED00E080B485B000AF78600E4B1B6892
:106170001B68002B01D1012200E000227B681A601D
:106180007B681B68002B05D1074B1B68DB681B680D
:10619000FB6001E00023FB60FB6818461437BD4636
:1061A0005DF8047B704700BF3406002080B584B0E2
:1061B00000AF7860FFF7DCF8F8600B4B1B68FA68FB
:1061C0009A4205D200F03AF97B6801221A6002E097
:1061D0007B6800221A60044AFB681360FB6818465B
:1061E0001037BD4680BD00BF4406002080B586B094
:1061F00000AFF860B9607A603B6000237B61FB68A8
:10620000BA685A60FB68FA681A61BA687B689A4291
:1062100012D87A683B68D21AFB689B699A4202D30B
:1062200001237B611BE0104B1A68FB68043319469D
:106230001046FEF714F812E07A683B689A4206D2DC
:10624000BA683B689A4202D301237B6107E0074B9F
:106250001A68FB68043319461046FEF700F87B699C
:1062600018461837BD4680BD380600203406002089
:1062700080B58EB002AFCEE07B68002B19DA3B1DF3
:106280000433FB62FB6A002B0BD14FF0500383F306
:106290001188BFF36F8FBFF34F8FFB6100BF00BF4B
:1062A000FDE7FB6A1B68FA6A5068FA6A9268114651
:1062B00098477B68002BC0F2AE80FB68BB62BB6A6C
:1062C0005B69002B04D0BB6A04331846FEF700F864
:1062D0003B461846FFF76AFF78627B68092B00F29D
:1062E000978001A252F823F011630008116300089F
:1062F00011630008876300089B630008E7630008D8
:106300001163000811630008876300089B6300089D
:10631000BB6A93F8283043F00103DAB2BB6A83F812
:106320002820BA68BB6A9B69D118BB687A6AB86AC8
:10633000FFF75CFF0346002B6CD0BB6A1B6AB86A90
:106340009847BB6A93F8283003F00403002B61D010
:10635000BA68BB6A9B691A4400230093002300219A
:10636000B86AFFF701FE38623B6A002B52D14FF04A
:10637000500383F31188BFF36F8FBFF34F8FBB615F
:1063800000BF00BFFDE7BB6A93F8283023F001038C
:10639000DAB2BB6A83F828203DE0BB6A93F8283064
:1063A00043F00103DAB2BB6A83F82820BA68BB6AFB
:1063B0009A61BB6A9B69002B0BD14FF0500383F3AA
:1063C0001188BFF36F8FBFF34F8F7B6100BF00BF9A
:1063D000FDE7BB6A9A697B6AD1187B6A7A6AB86AF8
:1063E000FFF704FF17E0BB6A93F8283003F00203BD
:1063F000002B03D1B86A00F0F5FA0CE0BB6A93F801
:10640000283023F00103DAB2BB6A83F8282002E0C7
:1064100000BF00E000BF084B1B68391D0022184672
:10642000FEF766FA0346002B7FF426AF00BF00BFDD
:106430003037BD4680BD00BF3C06002080B588B027
:1064400002AF49E02E4B1B68DB681B683B612C4B9D
:106450001B68DB68DB68FB60FB6804331846FDF7EC
:1064600037FFFB681B6AF8689847FB6893F8283089
:1064700003F00403002B2FD0FB689B693A69134497
:10648000BB60BA683B699A420ED9FB68BA685A6029
:10649000FB68FA681A611A4B1A68FB6804331946DC
:1064A0001046FDF7DCFE17E00023009300233A6955
:1064B0000021F868FFF758FD78607B68002B0BD14E
:1064C0004FF0500383F31188BFF36F8FBFF34F8FEB
:1064D0003B6000BF00BFFDE7094B1B681B68002B3A
:1064E000B0D1074B1B687B61064B1B68044A1360E5
:1064F000044A7B69136000BF1837BD4680BD00BFEA
:10650000340600203806002080B582B002AF00F0CB
:10651000BBFC154B1B68002B20D11448FDF74EFE29
:106520001348FDF74BFE134B104A1A60124B104AEA
:106530001A6000230093114B114A10210A20FDF725
:106540005BFF0346084A1360074B1B68002B05D00E
:10655000054B1B680B491846FEF7BCFB00F0C6FC58
:1065600000BFBD4680BD00BF3C0600200C060020D9
:10657000200600203406002038060020E80600200F
:106580004806002024E3000880B483B000AF03462F
:106590003960FB7197F90730002B0ADB3B68DAB2F0
:1065A0000C4997F907301201D2B20B4483F800234B
:1065B0000AE03B68DAB20849FB7903F00F03043BB9
:1065C0001201D2B20B441A7600BF0C37BD465DF8FB
:1065D000047B704700E100E000ED00E080B500AF13
:1065E00000216FF00400FFF7CFFF00BF80BD000067
:1065F00080B483B000AFEFF305833B603B68002BB2
:1066000003D06FF005037B600CE00A4B1B68002B86
:1066100005D1084B01221A6000237B6002E04FF095
:10662000FF337B607B6818460C37BD465DF8047B02
:10663000704700BF3807002080B582B000AFEFF38D
:1066400005833B603B68002B03D06FF005037B6044
:1066500010E00B4B1B68012B09D1FFF7BFFF084B64
:1066600002221A60FEF770FD00237B6002E04FF00B
:10667000FF337B607B6818460837BD4680BD00BF8E
:106680003807002080B58EB004AFF860B9607A603A
:1066900000233B61EFF305837B617B69002B7ED197
:1066A000FB68002B7BD080233B621823FB61002317
:1066B0007B624FF0FF33BB617B68002B45D07B686A
:1066C0001B68002B02D07B681B687B627B689B6920
:1066D000002B02D07B689B69FB61FB69002B08D013
:1066E000FB69382B05D87B685B6803F00103002B3E
:1066F00001D0002354E07B685B69002B03D07B68EA
:106700005B699B083B627B689B68002B0ED07B68B3
:10671000DB685B2B0AD97B681B69002B06D07B6882
:106720005B69002B02D00123BB6110E07B689B6892
:10673000002B0CD17B68DB68002B08D17B681B69C0
:10674000002B04D10023BB6101E00023BB61BB69C6
:10675000012B10D17B681B697A68926802920193C1
:10676000FB690093BB683A6A796AF868FEF710FB28
:1067700003463B6113E0BB69002B10D13B6A9AB220
:1067800007F110030193FB690093BB68796AF8680D
:10679000FEF75EFB0346012B01D000233B613B6902
:1067A00018462837BD4680BD80B584B000AF7860FC
:1067B000EFF30583BB60BB68002B03D06FF00503CC
:1067C000FB6007E00023FB607B68002B02D0786849
:1067D000FEF784FCFB6818461037BD4680BD0000FC
:1067E00080B485B000AFF860B9607A60FB68074A92
:1067F0001A60BB68064A1A607B6880221A6000BF74
:106800001437BD465DF8047B704700BF3C0700208D
:106810009807002080B485B000AFF860B9607A6056
:10682000FB68074A1A60BB68064A1A607B684FF427
:1068300080721A6000BF1437BD465DF8047B704754
:1068400098090020F409002080B58AB000AF786074
:106850000023FB61FEF7E0FC5C4B1B68002B01D1C1
:1068600000F024F95A4B1A687B681340002B40F063
:1068700095807B68002B1ED008227B6813447B60C8
:106880007B6803F00703002B15D07B6823F0070318
:1068900008337B607B6803F00703002B0BD04FF0BD
:1068A000500383F31188BFF36F8FBFF34F8F7B616A
:1068B00000BF00BFFDE77B68002B6FD0454B1B6816
:1068C0007A689A426AD8444B3B62434B1B687B62AE
:1068D00004E07B6A3B627B6A1B687B627B6A5B6865
:1068E0007A689A4203D97B6A1B68002BF1D1374B37
:1068F0001B687A6A9A4251D03B6A1B68082213448B
:10690000FB617B6A1A683B6A1A607B6A5A687B681B
:10691000D21A08235B009A4220D97A6A7B68134412
:10692000BB61BB6903F00703002B0BD04FF0500392
:1069300083F31188BFF36F8FBFF34F8F3B6100BFAD
:1069400000BFFDE77B6A5A687B68D21ABB695A6050
:106950007B6A7A685A60B86900F00AF91D4B1A68B8
:106960007B6A5B68D31A1B4A13601A4B1A681B4B6D
:106970001B689A4203D2174B1B68184A13607B6A44
:106980005A68134B1B681A437B6A5A607B6A002261
:106990001A60134B1B680133114A1360FEF74AFC5F
:1069A000FB6903F00703002B0BD04FF0500383F378
:1069B0001188BFF36F8FBFF34F8FFB6000BF00BF25
:1069C000FDE7FB6918462837BD4680BDFC4900201D
:1069D000104A0020004A0020F4490020044A002008
:1069E000084A002080B586B000AF78607B687B6184
:1069F0007B68002B4FD008235B427A6913447B618C
:106A00007B693B613B695A68254B1B681340002B2F
:106A10000BD14FF0500383F31188BFF36F8FBFF397
:106A20004F8FFB6000BF00BFFDE73B691B68002B79
:106A30000BD04FF0500383F31188BFF36F8FBFF378
:106A40004F8FBB6000BF00BFFDE73B695A68144B26
:106A50001B681340002B1ED03B691B68002B1AD10A
:106A60003B695A680E4B1B68DB431A403B695A600E
:106A7000FEF7D2FB3B695A680A4B1B681344094A6C
:106A80001360386900F074F8074B1B680133064A3D
:106A90001360FEF7CFFB00BF1837BD4680BD00BFB7
:106AA000104A0020004A00200C4A002080B485B023
:106AB00000AF4FF47053BB60274BFB60FB6803F0E3
:106AC0000703002B0CD0FB680733FB60FB6823F047
:106AD0000703FB60BA68FB68D31A1F4A1344BB6004
:106AE000FB687B601D4A7B6813601C4B00225A6068
:106AF0007B68BA681344FB600822FB689B1AFB6042
:106B0000FB6823F00703FB60FB68154A1360144B16
:106B10001B6800225A60124B1B6800221A607B68B7
:106B20003B603B68FA68D21A3B685A600C4B1A68A3
:106B30003B681A603B685B680A4A13603B685B68A5
:106B4000094A1360094B4FF000421A6000BF143726
:106B5000BD465DF8047B7047F40D0020F449002029
:106B6000FC490020044A0020004A0020104A00206E
:106B700080B485B000AF7860284BFB6002E0FB6812
:106B80001B68FB60FB681B687A689A42F7D8FB6851
:106B9000BB60FB685B68BA6813447A689A4208D1A4
:106BA000FB685A687B685B681A44FB685A60FB683C
:106BB0007B607B68BB607B685B68BA681A44FB6873
:106BC0001B689A4218D1FB681A68154B1B689A42D9
:106BD0000DD07B685A68FB681B685B681A447B6849
:106BE0005A60FB681B681A687B681A6008E00C4BE7
:106BF0001A687B681A6003E0FB681A687B681A6091
:106C0000FA687B689A4202D0FB687A681A6000BF13
:106C10001437BD465DF8047B704700BFF44900207F
:106C2000FC49002080B485B000AFF860B9607A609C
:106C3000FB68043BFB60FB684FF080721A60FB68E6
:106C4000043BFB60BB6823F00102FB681A60FB6831
:106C5000043BFB600C4AFB681A60FB68143BFB605A
:106C60007A68FB681A60FB68043BFB60FB686FF0A6
:106C700002021A60FB68203BFB60FB681846143771
:106C8000BD465DF8047B70478D6C000880B485B00C
:106C900000AF00237B60134B1B68B3F1FF3F0BD0A9
:106CA0004FF0500383F31188BFF36F8FBFF34F8F03
:106CB000FB6000BF00BFFDE74FF0500383F3118876
:106CC000BFF36F8FBFF34F8FBB6000BF00BF7B6808
:106CD000002BFCD000BF00BF1437BD465DF8047B1D
:106CE000704700BF0C000020000000000000000002
:106CF000074B19680868B0E8F04F80F30988BFF3C4
:106D00006F8F4FF0000080F311887047AFF3008061
:106D10000C01002000BF00BF08480068006880F335
:106D200008884FF0000080F3148862B661B6BFF3A4
:106D30004F8FBFF36F8F00DF00BF00BF08ED00E093
:106D400080B586B000AF474B1B68474A93420BD1D2
:106D50004FF0500383F31188BFF36F8FBFF34F8F52
:106D6000FB6000BF00BFFDE73E4B1B683F4A9342FC
:106D70000BD14FF0500383F31188BFF36F8FBFF334
:106D80004F8F3B6100BF00BFFDE7394B7B617B69E3
:106D90001B78DBB27B607B69FF221A707B691B78F2
:106DA000DBB2FB70FB78DBB203F05003DAB2314B9D
:106DB0001A70314B07221A6009E02F4B1B68013B08
:106DC0002D4A1360FB78DBB25B00DBB2FB70FB7813
:106DD000DBB203F08003802BEFD0274B1B68C3F19D
:106DE0000703042B0BD04FF0500383F31188BFF33C
:106DF0006F8FBFF34F8FBB6000BF00BFFDE71E4B1F
:106E00001B681B021C4A13601B4B1B6803F4E063E6
:106E1000194A13607B68DAB27B691A70174B1B68DA
:106E2000164A43F470031360144B1B68134A43F073
:106E30007043136000F0DAF8114B00221A6000F082
:106E4000F9F8104B1B680F4A43F040431360FFF7FB
:106E500063FFFEF757FBFFF719FF002318461837AB
:106E6000BD4680BD00ED00E071C20F4170C20F4110
:106E700000E400E0144A0020184A002020ED00E061
:106E80000C00002034EF00E080B483B000AF4FF07E
:106E9000500383F31188BFF36F8FBFF34F8F7B6075
:106EA00000BF104B1B6801330E4A13600D4B1B686B
:106EB000012B10D10C4B1B68DBB2002B0BD04FF019
:106EC000500383F31188BFF36F8FBFF34F8F3B6085
:106ED00000BF00BFFDE700BF0C37BD465DF8047B77
:106EE000704700BF0C00002004ED00E080B483B0C8
:106EF00000AF124B1B68002B0BD14FF0500383F3F4
:106F00001188BFF36F8FBFF34F8F7B6000BF00BF4F
:106F1000FDE70A4B1B68013B084A1360074B1B68DF
:106F2000002B05D100233B603B6883F3118800BF31
:106F300000BF0C37BD465DF8047B70470C00002095
:106F4000EFF30980BFF36F8F154B1A681EF0100F17
:106F500008BF20ED108A20E9F04F10602DE90900EC
:106F60004FF0500080F31188BFF34F8FBFF36F8F46
:106F7000FEF7C8FA4FF0000080F3118809BC1968C9
:106F80000868B0E8F04F1EF0100F08BFB0EC108A90
:106F900080F30988BFF36F8F704700BFAFF30080A5
:106FA0000C01002000BF00BF80B582B000AF4FF0E1
:106FB000500383F31188BFF36F8FBFF34F8F7B6054
:106FC00000BFFEF7E5F90346002B03D0064B4FF058
:106FD00080521A6000233B603B6883F3118800BF36
:106FE00000BF0837BD4680BD04ED00E080B400AFAF
:106FF0000B4B00221A600B4B00221A600A4B1B68D5
:107000000A4AA2FB03239B09094A013B1360044B74
:1070100007221A6000BFBD465DF8047B704700BFC1
:1070200010E000E018E000E000000020D34D621006
:1070300014E000E0DFF80C00016841F47001016029
:10704000704700BF88ED00E080B485B000AFEFF37B
:107050000583FB60FB680F2B15D9184AFB681344A6
:107060001B78FB72164B1B78FA7A9A420BD24FF0C0
:10707000500383F31188BFF36F8FBFF34F8F7B6093
:1070800000BF00BFFDE70F4B1B6803F4E0620E4B2F
:107090001B689A420BD94FF0500383F31188BFF35A
:1070A0006F8FBFF34F8F3B6000BF00BFFDE700BF96
:1070B0001437BD465DF8047B704700BFF0E300E085
:1070C000144A00200CED00E0184A002080B500AF03
:1070D000FBF7BCFA00F012F800F080F800F024FA98
:1070E00000F05AFA00F090F900F05AFBFFF780FA2E
:1070F00000F038F9FFF7A0FA00BFFDE780B594B0C3
:1071000000AF07F1200330220021184606F058FF97
:1071100007F10C0300221A605A609A60DA601A6163
:107120000023BB60284B1B6C274A43F08053136439
:10713000254B1B6C03F08053BB60BB6800237B6056
:10714000224B1B68214A43F4804313601F4B1B688A
:1071500003F480437B607B6802233B620123FB6274
:1071600010233B630223BB630023FB6308233B64C0
:10717000A8237B640223BB640423FB6407F1200380
:107180001846F9F711FF0346002B01D000F020F854
:107190000F23FB6002233B6100237B614FF4A0536C
:1071A000BB614FF48053FB6107F10C0305211846C6
:1071B000FAF772F90346002B01D000F009F800BF7E
:1071C0005037BD4680BD00BF00380240007000400F
:1071D00080B400AF72B600BF00BFFDE780B58CB0D1
:1071E00000AF07F11C0300221A605A609A60DA604F
:1071F0001A610023BB61574B1B6B564A43F0400397
:107200001363544B1B6B03F04003BB61BB6900234A
:107210007B61504B1B6B4F4A43F0020313634D4B92
:107220001B6B03F002037B617B6900233B61494BCD
:107230001B6B484A43F001031363464B1B6B03F07F
:1072400001033B613B690023FB60424B1B6B414ADE
:1072500043F0080313633F4B1B6B03F00803FB6011
:10726000FB680023BB603B4B1B6B3A4A43F00403B3
:107270001363384B1B6B03F00403BB60BB68002334
:107280007B60344B1B6B334A43F080031363314BF9
:107290001B6B03F080037B607B6800224FF48071DE
:1072A0002D48FAF78DFC002210212C48FAF788FCB3
:1072B000002201212A48FAF783FC4FF48073FB6116
:1072C00001233B6200237B620023BB6207F11C03A6
:1072D00019462148FAF7C0FA1023FB6101233B62EB
:1072E00000237B620023BB6207F11C0319461B4885
:1072F000FAF7B2FA3023FB614FF488133B620023A4
:107300007B6207F11C0319461348FAF7A5FA01231B
:10731000FB6101233B6200237B620023BB6207F118
:107320001C0319460E48FAF797FA002205210A2095
:10733000FBF755F90A20FBF76EF90022052117200B
:10734000FBF74DF91720FBF766F900BF3037BD4654
:1073500080BD00BF0038024000080240000002402B
:107360000004024080B500AF144A00211448FFF722
:1073700089F90346134A1360134A00211348FFF7A3
:1073800081F90346124A1360124A00211248FFF79E
:1073900079F90346114A1360114A00211148FFF799
:1073A00071F90346104A1360104A00211048FFF794
:1073B00069F903460F4A136000BF80BD84E30008EB
:1073C000F97300081C4A0020A8E3000879C90008E6
:1073D000204A0020CCE30008DD830008244A002076
:1073E000F0E300088D870008284A002014E4000814
:1073F000618800082C4A002080B582B000AF786018
:107400000120FFF7D1F9FBE780B500AF184B194A0F
:107410001A60174B03225A60154B00229A60144BD6
:107420004FF08072DA60124B4FF4C0221A61104B99
:107430004FF4A0025A610E4B00221A760C4B002228
:107440005A760B4B00229A76094B0122DA76084BCA
:1074500000221A77064B00225A770548F8F70AFFF0
:107460000346002B01D0FFF7B3FE00BF80BD00BF75
:10747000304A00200064004080B58AB000AF7860D8
:1074800007F1140300221A605A609A60DA601A61E8
:107490007B681B68214A93423BD100233B61204B10
:1074A0001B6C1F4A43F0007313641D4B1B6C03F0ED
:1074B00000733B613B690023FB60194B1B6B184A4F
:1074C00043F008031363164B1B6B03F00803FB60C8
:1074D000FB6803237B610223BB610023FB61032361
:1074E0003B6209237B6207F1140319460D48FAF742
:1074F000B3F9002205211420FBF771F81420FBF7E3
:107500008AF8002205211520FBF769F81520FBF702
:1075100082F800BF2837BD4680BD00BF0064004030
:1075200000380240000C024080B582B000AF00235A
:107530007B60184B1B6B174A43F480031363154B96
:107540001B6B03F480037B607B68002205213820DD
:10755000FBF745F83820FBF75EF8002205213920BB
:10756000FBF73DF83920FBF756F8002205213B20B8
:10757000FBF735F83B20FBF74EF8002205214520AC
:10758000FBF72DF84520FBF746F800BF0837BD464E
:1075900080BD00BF0038024080B500AF174B184ACD
:1075A0001A60164B4FF482725A60144B00229A6094
:1075B000124B0022DA60114B02221A610F4B01229A
:1075C0005A610E4B4FF400729A610C4B1022DA6133
:1075D0000A4B00221A62094B00225A62074B002212
:1075E0009A62064B0A22DA620448FBF7A1F80346C6
:1075F000002B01D0FFF7ECFD00BF80BD584A0020F2
:107600000030014080B58AB000AF786007F1140304
:1076100000221A605A609A60DA601A617B681B68FF
:10762000574A934240F0A88000233B61554B5B6C66
:10763000544A43F480535364524B5B6C03F48053BD
:107640003B613B690023FB604E4B1B6B4D4A43F093
:10765000020313634B4B1B6B03F00203FB60FB68DD
:107660000023BB60474B1B6B464A43F00103136387
:10767000444B1B6B03F00103BB60BB6818237B61A9
:107680000223BB610023FB6103233B6205237B6272
:1076900007F1140319463C48FAF7DEF880237B61B2
:1076A0000223BB610023FB6103233B6205237B6252
:1076B00007F1140319463548FAF7CEF8344B354A2A
:1076C0001A60334B4FF0C0625A60314B40229A60CF
:1076D0002F4B0022DA602E4B4FF480621A612C4B44
:1076E00000225A612A4B00229A61294B0022DA615A
:1076F000274B4FF400321A62254B00225A6224486D
:10770000FAF790FA0346002B01D0FFF761FD7B6882
:107710001F4A9A641E4A7B6893631F4B1F4A1A6074
:107720001D4B4FF0C0625A601B4B00229A601A4BEF
:107730000022DA60184B4FF480621A61164B002267
:107740005A61154B00229A61134B0022DA61124BE9
:107750004FF400321A62104B00225A620E48FAF7B8
:1077600061FA0346002B01D0FFF732FD7B680A4A1D
:10777000DA64094A7B68936300BF2837BD4680BD41
:107780000030014000380240000402400000024086
:10779000B04A002058640240104B002010640240A0
:1077A00080B500AF104B114A1A600F4B104A5A6057
:1077B0000D4B00229A600C4B0022DA600A4B00222B
:1077C0001A61094B0C225A61074B00229A61064B41
:1077D0000022DA610448FBF7B9FA0346002B01D016
:1077E000FFF7F6FC00BF80BD704B00200014014085
:1077F0000094110080B58AB000AF786007F11403DF
:1078000000221A605A609A60DA601A617B681B680D
:107810004C4A934240F0928000233B614A4B5B6CA0
:10782000494A43F020035364474B5B6C03F0200349
:107830003B613B690023FB60434B1B6B424A43F0B7
:1078400040031363404B1B6B03F04003FB60FB687A
:107850004FF484437B610223BB610023FB6103235C
:107860003B6208237B6207F1140319463748F9F796
:10787000F3FF374B374A1A60354B4FF020625A609E
:10788000334B40229A60324B0022DA60304B4FF487
:1078900080621A612E4B00225A612D4B00229A61A0
:1078A0002B4B0022DA612A4B00221A62284B00225D
:1078B0005A622748FAF7B6F90346002B01D0FFF7C2
:1078C00087FC7B68224A9A63214A7B689363224B38
:1078D000224A1A60204B4FF020625A601E4B002251
:1078E0009A601D4B0022DA601B4B4FF480621A61D4
:1078F000194B00225A61184B00229A61164B002244
:10790000DA61154B4FF480321A62134B00225A622F
:107910001148FAF787F90346002B01D0FFF758FC0E
:107920007B680D4ADA630C4A7B6893630022052169
:107930004720FAF754FE4720FAF76DFE00BF2837BC
:10794000BD4680BD001401400038024000180240CE
:10795000B84B0020A0640240184C0020286402406C
:1079600080B400AF00BFFDE780B400AF00BFFDE70B
:1079700080B400AF00BFFDE780B400AF00BFFDE7FB
:1079800080B400AF00BFFDE780B400AF00BFBD46CC
:107990005DF8047B704780B500AFFAF7A9FEFEF7EB
:1079A00021F80346012B01D0FFF7FEFA00BF80BD8E
:1079B00080B500AF1020FAF71DF900BF80BD0000B0
:1079C00080B500AF0248F9F7C0F800BF80BD00BF26
:1079D000304A002080B500AF0248F9F7B6F800BF82
:1079E00080BD00BF304A002080B500AF2020FAF7EC
:1079F00001F900BF80BD000080B500AF0248FAF772
:107A0000A9FA00BF80BD00BF184C002080B500AFB0
:107A10000248FAF79FFA00BF80BD00BFB04A0020BD
:107A200080B500AF0248FAF795FA00BF80BD00BFED
:107A3000B84B002080B500AF0248FBF7ADFA00BF9D
:107A400080BD00BF704B002080B582B000AF002326
:107A50007B60124B5B6C114A43F4804353640F4BC1
:107A60005B6C03F480437B607B6800233B600B4BC3
:107A70001B6C0A4A43F080531364084B1B6C03F0E1
:107A800080533B603B6800220F216FF00100FAF742
:107A9000A6FD00BF0837BD4680BD00BF00380240CC
:107AA000DFF834D0F8F7D4FB0C480D490D4A002319
:107AB00002E0D458C4500433C4188C42F9D30A4AA3
:107AC0000A4C002301E013600432A242FBD306F00B
:107AD00085FAFFF7FBFA7047000002200000002043
:107AE000AC000020A4E40008AC0000205C4F0020A3
:107AF000FEE780B485B000AFF860B9601346FB7153
:107B0000FB6800221A70FB68FA795A70FB684FF024
:107B100000025A60FB684FF000029A60FB684FF069
:107B20000002DA60FB68BA681A61FB68184614370D
:107B3000BD465DF8047B704780B582B000AF7860C9
:107B400000220121786801F023F800BF0837BD4604
:107B500080BD80B582B000AF87ED010AC7ED000A95
:107B6000D7ED000A97ED010A05F0DAFEF0EE407A53
:107B7000B0EE670A0837BD4680BD80B483B000AF61
:107B800087ED010A97ED017AD7ED017AB4EE677AB5
:107B9000F1EE10FA6CBF01230023DBB2002B14BFFF
:107BA00001230023DBB218460C37BD465DF8047B89
:107BB000704780B48BB000AF78620B4687ED070A40
:107BC000C7ED060A87ED051AC7ED041A87ED032AEB
:107BD000C7ED022A87ED013A87F823307B6A4FF020
:107BE00000021A607B6A97F823201A717B6AFA698F
:107BF0009A607B6ABA69DA607B6A7A691A617B6A21
:107C00003A695A617B6AFA689A617B6ABA68DA6192
:107C10007B6A7A681A627B6A4FF000025A627B6A5A
:107C20004FF000029A627B6A4FF00002DA627B6AD0
:107C30004FF000021A637B6A18462C37BD465DF888
:107C4000047B704780B584B000AF786087ED000A90
:107C50007B6893ED007AD7ED007A77EE677AC7ED0F
:107C6000037A7B681B79002B67D17B6893ED0B7AD5
:107C7000D7ED037A77EE277A7B68C3ED0B7A7B68C2
:107C8000D3ED057AB0EE670AFFF777FF034683F07E
:107C90000103DBB2002B0ED07B6893ED0B7A7B687F
:107CA000D3ED057AB4EEE77AF1EE10FA03DB7B68E8
:107CB0005A697B68DA627B68D3ED067AB0EE670AB0
:107CC000FFF75BFF034683F00103DBB2002B0ED00E
:107CD0007B6893ED0B7A7B68D3ED067AB4EEE77A96
:107CE000F1EE10FA03D87B689A697B68DA627B68E8
:107CF00093ED027AD7ED037A27EE277A7B68D3EDEE
:107D0000036A7B68D3ED0B7A66EEA77A37EE277AA3
:107D10007B68D3ED046A7B68D3ED097A97ED036A3B
:107D200076EE677A66EEA77A77EE277A7B68C3ED00
:107D30000C7A7B68FA685A623CE07B681B79012BFD
:107D400038D17B6893ED0C7A7B68D3ED026A7B684F
:107D5000D3ED097A97ED036A76EE677A66EEA76A45
:107D60007B6893ED036AD7ED037A66EE277A76EEA9
:107D7000A76A7B6893ED046A7B68D3ED097A77EE96
:107D8000A77AD7ED035A75EEE75A7B68D3ED0A7AE6
:107D900075EEA77A66EE277A76EEA77A77EE277ADF
:107DA0007B68C3ED0C7A7B685A6A7B689A627B6851
:107DB000FA685A627B68D3ED077AB0EE670AFFF77C
:107DC000DCFE034683F00103DBB2002B0ED07B68A0
:107DD00093ED0C7A7B68D3ED077AB4EEE77AF1EE97
:107DE00010FA03DB7B68DA697B681A637B68D3ED82
:107DF000087AB0EE670AFFF7C0FE034683F001037E
:107E0000DBB2002B0ED07B6893ED0C7A7B68D3ED50
:107E1000087AB4EEE77AF1EE10FA03D87B681A6AB2
:107E20007B681A637B681B6B07EE903AB0EE670ABB
:107E30001037BD4680BDB0B489B000AFF861B961FC
:107E40007A6187ED040AC7ED030ABB6087ED011A6A
:107E5000FB6900221A70FB6900225A70FB694FF01F
:107E600000025A60FB694FF000029A60FB69BA6930
:107E7000DA60FB697A691A61FB69BA6803F1140474
:107E800015460FCD0FC40FCD0FC40FCD0FC42B68F7
:107E90002360FB693A6B03F1480415460FCD0FC40C
:107EA0000FCD0FC40FCD0FC42B682360FB697A6818
:107EB000DA67FB694FF00002C3F88020FB694FF0DE
:107EC0000002C3F88420FB693A69C3F88820FB6983
:107ED000FA68C3F88C20FB6918462437BD46B0BC4D
:107EE000704780B582B000AF78607B68DB68184669
:107EF000FFF722FE7B681B691846FFF71DFE7B68B3
:107F000001221A7000BF0837BD4680BD80B483B01F
:107F100000AF78607B681B7883F00103DBB2002B35
:107F200013D17B685A687B685A617B6893ED027A4B
:107F30007B681B69D3ED027A77EE277A7B68C3ED05
:107F4000127A7B6801225A7000E000BF0C37BD46F0
:107F50005DF8047B7047000080B584B000AFF86026
:107F600087ED020AC7ED010AFB681B7883F0010365
:107F7000DBB2002B40F0F581FB68BA685A60FB6801
:107F80001B6993ED027AD7ED017A77EE277AFB68C9
:107F9000C3ED027AFB685B7883F00103DBB2002B50
:107FA00065D0FB68DA68FB68D3ED207AB0EE670A2B
:107FB000104600F0BFFEFB68D3ED217AF5EEC07AE3
:107FC000F1EE10FA19DDFB681B6993ED027AFB688C
:107FD000D3ED237A77EE677A9FEDCE1ADFEDCE0AE6
:107FE000B0EE670A00F0C4F9F0EE407AB6EE007A1F
:107FF000F4EEC77AF1EE10FA21DCFB68D3ED217ABA
:10800000F5EEC07AF1EE10FA1BD5FB681B6993ED13
:10801000027AFB68D3ED237A77EE677A9FEDBD1A7B
:10802000DFEDBD0AB0EE670A00F0A2F9F0EE407A8B
:10803000BEEE007AF4EEC77AF1EE10FA01D5012314
:1080400000E00023002B07D0FB681B699FEDB30AFB
:10805000184600F06FFE85E1FB681A69FB68D3EDF6
:10806000217AB0EE670A104600F064FE7AE1FB6800
:1080700093ED057AFB68D3ED206AFB68D3ED1F7A98
:1080800066EEA77A77EEA77ADFEDA26A67EEA66AB8
:108090009FEDA36AC6EE867A77EE277AFB68C3ED7A
:1080A000057AFB68D3ED057A9FED9E1ADFED9B0AFA
:1080B000B0EE670A00F05CF9F0EE407AFB68C3EDC1
:1080C000057AFB6893ED057AFB68D3ED017A77EECC
:1080D000677A9FED907AF4EEC77AF1EE10FA14DD2C
:1080E000FB6803F11402FB68D3ED017A9FED8D7AF2
:1080F00077EE877AB0EE670A1046FFF7A3FDF0EE41
:10810000407A894BC3ED007A33E0FB6893ED057A42
:10811000FB68D3ED017A77EE677A9FED7F7AF4EE14
:10812000C77AF1EE10FA14D5FB6803F11402FB686C
:10813000D3ED017A9FED7B7A77EEC77AB0EE670ACE
:108140001046FFF77FFDF0EE407A774BC3ED007AE3
:108150000FE0FB6803F11402FB68D3ED017AB0EE87
:10816000670A1046FFF76EFDF0EE407A6E4BC3EDE6
:10817000007AFB68DB686C4AD2ED007AB0EE670AE1
:10818000184600F009FEFB68D3ED217AF5EEC07ABF
:10819000F1EE10FA19DDFB681B6993ED027AFB68BA
:1081A000D3ED237A77EE677A9FED5A1ADFED5A0AFC
:1081B000B0EE670A00F0DCF8F0EE407AB6EE007A36
:1081C000F4EEC77AF1EE10FA21DCFB68D3ED217AE8
:1081D000F5EEC07AF1EE10FA1BD5FB681B6993ED42
:1081E000027AFB68D3ED237A77EE677A9FED491A1E
:1081F000DFED490AB0EE670A00F0BAF8F0EE407A17
:10820000BEEE007AF4EEC77AF1EE10FA01D5012342
:1082100000E00023002B0AD0FB68D3ED127A9FED1B
:108220003F7A77EE877AFB68C3ED127A19E0FB6834
:1082300093ED127AFB68D3ED216AFB68D3ED1F7AC8
:1082400066EEA77A77EEA77ADFED326A67EEA66A66
:108250009FED336AC6EE867A77EE277AFB68C3ED28
:10826000127AFB68D3ED127A9FED2E1ADFED2B0AFE
:10827000B0EE670A00F07CF8F0EE407AFB68C3EDE0
:10828000127AFB6893ED127AFB68D3ED027A77EEEF
:10829000677A9FED207AF4EEC77AF1EE10FA14DDDA
:1082A000FB6803F14802FB68D3ED027A9FED1D7A6B
:1082B00077EE877AB0EE670A1046FFF7C3FCF0EE60
:1082C000407A194BC3ED007A40E0FB6893ED127AD7
:1082D000FB68D3ED027A77EE677A9FED0F7AF4EEC2
:1082E000C77AF1EE10FA21D5FB6803F14802FB686A
:1082F000D3ED027A9FED0B7A77EEC77AB0EE670A7C
:108300001046FFF79FFCF0EE407A074BC3ED007A72
:108310001CE000BFDB0F4940DB0F49C0000000003C
:1083200000007042DB0FC940784C0020FB6803F16D
:108330004802FB68D3ED027AB0EE670A1046FFF7F9
:1083400081FCF0EE407A094BC3ED007AFB681B69B3
:10835000064AD2ED007AB0EE670A184600F01CFD1E
:1083600000E000BF1037BD4680BD00BF784C002044
:1083700080B584B000AF87ED030AC7ED020A87ED30
:10838000011A97ED037AD7ED027A77EE676A97EDD7
:10839000017AD7ED027A77EE677AF0EE670AB0EEEF
:1083A000660AFFF7D6FB87ED030AD7ED037AF5EEF1
:1083B000C07AF1EE10FA06D597ED037AD7ED017A7F
:1083C00077EE277A05E097ED037AD7ED027A77EE1C
:1083D000277AB0EE670A1037BD4680BD80B582B0FF
:1083E00000AF786000F054F82248FFF7A5FB224860
:1083F000FFF7A2FB9FED210A1E4800F065FC9FEDF0
:108400001F0A1D4800F060FC4FF4FA60FEF7CCF93B
:1084100001224FF480711A48F9F7D2FB1948FFF78F
:1084200060FD3220FEF7C0F91648FFF76FFD00BF70
:108430004FF0FF310120FDF763FB0346012B14BF12
:1084400001230023DBB2002BF2D10F4BD3ED007AD6
:108450000D4B93ED017AF0EE470AB0EE670A09483A
:10846000FFF77AFD094B1868002302220021FDF76F
:108470008FFBDCE77C4C0020904C002000000000CB
:1084800000080240A44C0020144E0020284A00207E
:1084900080B58AB000AF00237B610023BB6101235C
:1084A000FB6100237B6000233B600023FB60002313
:1084B000BB6000233B6101233B620E237B623B4692
:1084C00019461648F7F7D2FF0346002B14BF0123C5
:1084D0000023DBB2002B01D0FEF77AFE0F48F8F73D
:1084E000A3F80346002B14BF01230023DBB2002BAB
:1084F00001D0FEF76DFE02210848F8F700FB0346A5
:10850000002B14BF01230023DBB2002B01D0FEF7A8
:108510005FFE00BF2837BD4680BD00BF304A002047
:1085200080B58CB000AF78607B68164A934225D145
:1085300007F10C0307F1140200217868F8F7BDF980
:108540007B69B3F5A06F19D37B69B3F5A16F15D81B
:108550007B69B3F5A06F06D107F10C0319460A48F1
:1085600000F05AFB0AE07B6940F20152934205D1C8
:1085700007F10C031946054800F04EFB00BF3037E9
:10858000BD4680BD304A00207C4C0020904C00202D
:1085900080B59CB002AF002233493448FFF7A9FAF6
:1085A000012231493248FFF7A4FA3B46BFEE003AB8
:1085B000F7EE002A9FED2F2ADFED2F1A9FED2F1ADD
:1085C000DFED2F0AB1EE040A00211846FFF7F1FA99
:1085D00007F13403BFEE003AF7EE002A9FED252A9B
:1085E000DFED251AB3EE0E1ADFED260A9FED260AFF
:1085F00000211846FFF7DDFA3A4607F134030093ED
:108600009FED221A1346DFED220A9FED210A184A38
:1086100016492048FFF70FFCBAEE043AF2EE042A9E
:10862000BAEE042AF2EE041AB3EE0E1ADFED180ABF
:108630009FED190A00211948FFF7BBFAB9EE043A79
:10864000F1EE042ABAEE042AF2EE041A9FED141A8F
:10865000DFED0F0ABBEE090A00211248FFF7A9FA65
:1086600000BF6837BD4680BD304A00207C4C0020EA
:10867000904C00206666E6BF6666E63F0000DC427E
:10868000CDCCCC3D7B142E3E333393406F12833AD6
:1086900000000000A44C002000007042344D002077
:1086A00000000CC2684D002080B500AFFFF770FFDE
:1086B00080BD80B400AF00231846BD465DF8047B42
:1086C000704780B483B000AF78607B6818460C3781
:1086D000BD465DF8047B704780B582B000AF78601E
:1086E00000220221786800F053FA00BF0837BD4627
:1086F00080BD000080B582B000AF78607B68DB6829
:108700009FED0F0A184600F047FB7B681B699FED41
:108710000C0A184600F040FB7B68DB681846FFF740
:10872000DBFF7B681B691846FFF7D6FF786800F00F
:1087300009F87B6800221A7000BF0837BD4680BD6B
:108740000000000080B483B000AF78607B68002236
:108750005A7000BF0C37BD465DF8047B704780B48B
:1087600085B000AFF86087ED020AC7ED010AFB682B
:10877000BA68C3F88020FB687A68C3F8842000BF19
:108780001437BD465DF8047B7047000080B584B0A7
:1087900000AF786000BF4FF0FF310120FDF7B0F966
:1087A0000346012B14BF01230023DBB2002BF2D1BF
:1087B0004FF480712348F9F7EBF903461A46224B30
:1087C0001A77224B1B781A461F4B5A771F4B5B7840
:1087D0001A461D4B9A771E4B1B681B4A13601C4B95
:1087E0005B68194A53601A4B9B68174A9360174B92
:1087F0005B68154AD360154B9B68134A1361154B90
:108800009B68114A5361144B9B680F4A9361002384
:10881000FB730023BB6009E0BB680B4A13441A7862
:10882000FB7B1344FB73BB680133BB60BB681E2B2F
:10883000F2D9054AFB7BD377202203490748FAF790
:10884000D5FAA7E7000802409C4D0020A44C002068
:10885000144E00207C4C0020904C0020704B0020D7
:1088600080B52DED028B8CB000AF786000220C211A
:108870000520FBF73EFE0346454A136007F10C0353
:1088800000221A605A609A600C2242494248FAF764
:1088900029FB3F4B1B6807F10C014FF0FF321846D4
:1088A000FCF726F8002387F82F300023BB620BE08B
:1088B000384ABB6A13441A7897F82F30134487F864
:1088C0002F30BB6A0133BB62BB6A0A2BF0D9314B34
:1088D000DB7A97F82F209A42DBD13B7D002B02D028
:1088E0003B7D012B0BD13B7D002B01D0012300E010
:1088F00000231A464FF480712848F9F761F97B7D0F
:10890000002B02D07B7D012B09D17B7D002B03D076
:108910002348FFF7E6FA02E02148FFF7EBFEBB7DB4
:10892000002B02D0BB7D012B09D1BB7D002B03D0D6
:108930001B48FFF7EBFA02E01948FFF703FF194B5A
:10894000BB61194BFB6107F11C0207F1180107F12C
:108950000C03184600F066F8034693ED008A114BAD
:108960003B62114B7B6207F1240207F1200107F102
:108970000C030433184600F055F80346D3ED007A93
:10898000F0EE670AB0EE480A0548FFF7E8FE80E718
:10899000BC4D0020C04D0020704B0020000802405C
:1089A000A44C0020000048C20000484280B584B0BA
:1089B00000AF78600B467B807B681A68154B1B689C
:1089C0009A4223D17B880C2B1BD1134B186807F1DB
:1089D000080200231149FBF7EDFEBB68002B07D00E
:1089E0000F4B4FF080521A60BFF34F8FBFF36F8F62
:1089F0000023FB6007F10C031A460C21074800F026
:108A000039F80C2205490348FAF76CFA00BF103711
:108A1000BD4680BD704B0020BC4D0020C04D0020E5
:108A200004ED00E080B584B000AFF860B9607A6012
:108A3000FFF73FFE0346002B0CD07B6893ED007AD6
:108A4000BB68D3ED007AB4EEE77AF1EE10FA01D507
:108A5000012300E00023002BB968F86800F020F83B
:108A600003467968184600F034F803461846103774
:108A7000BD4680BDB0B584B000AFF860B9607A6023
:108A8000FC68B868FFF71DFE014600BF2B467A68F8
:108A9000204600F037F8034618461037BD46B0BDF3
:108AA00080B483B000AF786039607B6893ED007A62
:108AB0003B68D3ED007AB4EEE77AF1EE10FA01D517
:108AC0003B6800E07B6818460C37BD465DF8047BC8
:108AD000704780B483B000AF786039603B6893ED35
:108AE000007A7B68D3ED007AB4EEE77AF1EE10FA03
:108AF00001D53B6800E07B6818460C37BD465DF841
:108B0000047B704780B584B000AFF860B9607A60CC
:108B10003B70BB68002B01D1FB680AE0FA68BB68B8
:108B200013447A681946F86800F007F8FA68BB68D9
:108B3000134418461037BD4680BD80B584B000AFE1
:108B4000F860B9607A607A68B968F86800F004F88B
:108B500000BF1037BD4680BD80B487B000AFF8605D
:108B6000B9607A607B681B687B6106E07B69DAB27A
:108B7000FB681A70FB680133FB60FA68BB689A42B5
:108B8000F4D100BF00BF1C37BD465DF8047B7047C1
:108B900080B58AB000AF78600B46FB7013463B800F
:108BA0001B4AFB7813701B4A3B88138001237B62AE
:108BB00000237B610023BB617B685B7803F58063E6
:108BC000FB607B685B7803F580633B61002387F87B
:108BD00020300323FB617B68186907F1240307F148
:108BE0000C010B4AF7F764FD00BF7B681B69184650
:108BF000F7F72EFE0346002B0CBF01230023DBB248
:108C0000002BF2D100BF00BF2837BD4680BD00BF9A
:108C1000CC4D0020CD4D002080B483B000AF7860F3
:108C200039603B681B7803F00103002B14BF01235C
:108C30000023DAB27B681A703B680233B3F9003064
:108C400007EE903AF8EEE77AB2EE047A27EE877AEA
:108C5000DFED196AC7EE267A7B68C3ED037A3B68BD
:108C60000433B3F9003007EE903AF8EEE77A9FED5F
:108C7000137A27EE877ADFED106AC7EE267A7B68D3
:108C8000C3ED017A3B6806331B885B0007EE903A20
:108C9000F8EEE77A9FED0A7A27EE877ADFED096A28
:108CA000C7EE267A7B68C3ED027A00BF0C37BD465B
:108CB0005DF8047B704700BF00FEFF4600007A4469
:108CC000DB0F494000FF7F4780B584B000AF78607C
:108CD00087ED000A4FF00003BB60134BFB6007F108
:108CE0000C0207F108013B461846FFF79BFED7ED43
:108CF000007AF0EE006A87EEA67ADFED0C6AC7EE26
:108D0000267A9FED0B7A67EE877AFDEEE77A17EE0B
:108D1000903A1BB21A4605217868FFF739FF00BF69
:108D20001037BD4680BD00BFDB0FC940DB0F494097
:108D300000FF7F4780B584B000AF786087ED000A00
:108D4000114BBB60114BFB6007F10C0207F10801EE
:108D50003B461846FFF766FE97ED007ADFED0C6A9A
:108D6000C7EE267A9FED0B7A67EE877AFDEEE77AFB
:108D700017EE903A1BB21A4604217868FFF708FFF5
:108D800000BF1037BD4680BD00007AC400007A44A1
:108D900000007A4400FEFF4680B584B000AF7860E2
:108DA00087ED000A114BBB60114BFB6007F10C0211
:108DB00007F108013B461846FFF734FE97ED007AAD
:108DC000F2EE046AC7EE267A9FED0A7A67EE877A9A
:108DD000FDEEE77A17EE903A1BB21A460321786847
:108DE000FFF7D6FE00BF1037BD4680BD000020C192
:108DF0000000204100FEFF4680B582B000AF002396
:108E0000FB7100F032FD00F037FD00F081F9034600
:108E1000002B04D0FB7963F07F03FB7106E000F0C8
:108E20001BF803461A46FB791343FB7100F04EFB17
:108E30000346002B04D0FB7943F04003FB7106E0AE
:108E400000F0CAF803461A46FB791343FB71FB791D
:108E500018460837BD4680BD80B582B000AF0023FC
:108E6000BB710023FB7100F027FD802000F054FD52
:108E7000552000F051FD552000F04EFD0346BB711A
:108E800000F026FD962000F00BFD00F015FD80207F
:108E900000F042FD552000F03FFD552000F03CFD64
:108EA0000346BB7100F014FD962000F0F9FC00F0C1
:108EB00003FDB6217E2000F087FC00F009FD502064
:108EC00000F0E1FC00F0F8FC802000F025FD5520CA
:108ED00000F022FD552000F01FFD0346BB7100F09D
:108EE000F7FC962000F0DCFC00F0E6FC802000F0AF
:108EF00013FD552000F010FD552000F00DFD034638
:108F0000BB7100F0E5FC962000F0CAFCBB79DBB237
:108F10001E2B01D0012358E00023FB7151E000F02B
:108F2000CBFCFA792B4913465B0013440B441878A9
:108F3000FA79284913465B0013440B4401331B782C
:108F4000194600F041FC00F0C3FC962000F0A8FC9C
:108F500000F0B2FCFA791F4913465B0013440B443E
:108F60001B7863F07F03DBB2184600F0D5FC552078
:108F700000F0D2FC552000F0CFFC0346BB7100F09E
:108F8000A7FC962000F08CFCFA79124913465B008E
:108F900013440B4401331A78BB79DBB29A420DD0EB
:108FA000FA790C4913465B0013440B4402331B78D7
:108FB000002B14BF01230023DBB206E0FB79013351
:108FC000FB71FB79052BAAD9002318460837BD464B
:108FD00080BD00BF1800002080B582B000AF002324
:108FE000FB710023BB7100F07FFCBB1D1946002004
:108FF00000F0FEFB00F084FC962000F051FC00F035
:1090000073FCBB1D1946002000F0F2FB00F078FC59
:10901000962000F045FC00F067FCB621142000F01B
:10902000D3FB00F06DFC502000F02DFC00F05CFC48
:10903000BB1D1946002000F0DBFB00F061FC962010
:1090400000F02EFC00F050FCBB1D1946002000F083
:10905000CFFB00F055FC962000F022FCBB790F2BD3
:1090600001D001234EE00023FB7147E000F03CFCFF
:10907000FA79264913465B0013440B441878FA79B1
:10908000224913465B0013440B4401331B781946F5
:1090900000F09AFB00F034FC962000F001FC00F098
:1090A00023FCFA79194913465B0013440B441B78DF
:1090B000BA1D1146184600F09BFB00F021FC9620DB
:1090C00000F0EEFBFA79114913465B0013440B44A0
:1090D00001331A78BB799A420DD0FA790B491346BD
:1090E0005B0013440B4402331B78002B14BF012395
:1090F0000023DBB206E0FB790133FB71FB79052B22
:10910000B4D9002318460837BD4680BD2C00002086
:1091100080B588B000AF07F1080300221A609A807A
:109120000023FB710023FB7700F0C6FB802000F0DA
:10913000F3FB552000F0F0FB552000F0EDFB03465B
:10914000FB7100F0C5FB962000F0AAFB00F0B4FB19
:10915000802000F0E1FB552000F0DEFB552000F000
:10916000DBFB0346FB7100F0B3FB962000F098FB9D
:1091700000F0A2FBB6217E2000F026FB00F0A8FB49
:10918000502000F080FB00F097FB802000F0C4FB33
:10919000552000F0C1FB552000F0BEFB0346FB71DB
:1091A00000F096FB962000F07BFB00F085FB802012
:1091B00000F0B2FB552000F0AFFB552000F0ACFBF7
:1091C0000346FB7100F084FB962000F069FBFB79FD
:1091D000DBB21E2B01D0012371E10023FB7754E0A9
:1091E00000F06AFBFA7FB84913465B0013440B4456
:1091F0001878FA7FB44913465B0013440B440133DB
:109200001B78194600F0E0FA00F062FB962000F0AF
:1092100047FB00F051FBFA7FAB4913465B00134458
:109220000B441B7863F07F03DBB2184600F074FB3D
:10923000552000F071FB552000F06EFB0346FB71DA
:1092400000F046FB962000F02BFBFA7F9E49134668
:109250005B0013440B4401331A78FB79DBB29A426A
:109260000DD0FA7F984913465B0013440B44023338
:109270001B78002B14BF01230023DBB21FE1502019
:1092800000F001FBFB7F0133FB77FB7F032BA7D9AA
:109290000023FB779DE000F00FFBFB7F1A1D8A493E
:1092A00013465B0013440B441878FB7F1A1D864954
:1092B00013465B0013440B4401331B78194600F03E
:1092C00083FA00F005FB962000F0EAFA00F0F4FAC9
:1092D000FB7F1A1D7C4913465B0013440B441B782B
:1092E00063F07F03DBB2184600F016FB552000F058
:1092F00013FB552000F010FB0346FB7100F0E8FA69
:10930000962000F0CDFAFB7F1A1D6F4913465B00D3
:1093100013440B4401331A78FB79DBB29A420ED026
:10932000FB7F1A1D684913465B0013440B4402334C
:109330001B78002B14BF01230023DBB2BFE05020B9
:1093400000F0A1FA00F0B8FA922000F0E5FA07F177
:10935000080306221946122000F062FA00F0B8FA5B
:109360007B7A1BB21B0219B23B7A1BB2FA7F0B430A
:1093700019B213465B0013445B0020333B44103B9F
:109380000A461A80FB7A1BB21B0219B2BB7A1BB2C7
:10939000FA7F0B4319B213465B0013445B00203382
:1093A0003B440E3B0A461A807B7B1BB21B0219B260
:1093B0003B7B1BB2FA7F0B4319B213465B0013448D
:1093C0005B0020333B440C3B0A461A80FB7F013391
:1093D000FB77FB7F012B7FF65EAF00F06DFA00217B
:1093E0006D2000F0F1F900F073FA962000F058FAC1
:1093F00000F062FAED2000F08FFA552000F08CFAB0
:10940000552000F089FA0346FB7100F061FA9620BE
:1094100000F046FAFB79DBB2002B01D001234EE0CD
:1094200000F04AFAB6217E2000F0CEF900F050FAA2
:10943000502000F028FAB7F910301A46B7F9163064
:10944000D31A40F25452934212DDB7F912301A4641
:10945000B7F91830D31A40F25452934208DDB7F9E5
:1094600014301A46B7F91A30D31AB3F52A7F01DA45
:10947000012324E000F020FA802000F04DFA55206E
:1094800000F04AFA552000F047FA0346FB7100F05D
:109490001FFA962000F004FA00F00EFA802000F087
:1094A0003BFA552000F038FA552000F035FA034613
:1094B000FB7100F00DFA962000F0F2F90023184637
:1094C0002037BD4680BD00BF38E4000880B582B0BB
:1094D00000AF0023BB710023FB7100F005FABB1D38
:1094E0001946002000F084F900F00AFA962000F0F6
:1094F000D7F900F0F9F9BB1D1946002000F078F902
:1095000000F0FEF9962000F0CBF900F0EDF9B6215D
:10951000142000F059F900F0F3F9502000F0B3F9ED
:1095200000F0E2F9BB1D1946002000F061F900F0DF
:10953000E7F9962000F0B4F900F0D6F9BB1D194602
:10954000002000F055F900F0DBF9962000F0A8F9B2
:1095500000F0CAF901213C2000F036F900F0D0F902
:10956000502000F090F900F0BFF9BB1D19463C20D7
:1095700000F03EF900F0C4F9962000F091F9FB7973
:109580000133FB71BB7903F00203002B02D1FB799D
:10959000092BE8D9FB790A2B01D1012307E0BB791C
:1095A00003F00403002B01D0012300E00023184640
:1095B0000837BD4680BD80B485B000AF78603960A3
:1095C0007B681B781BB2DB001AB27B6801331B7807
:1095D0005B09DBB21BB21343FB81B7F90E30B3F565
:1095E000806F04DBFB89A3F500639BB2FB81B7F9B5
:1095F0000E3007EE903AF8EEE77AB4EE007A67EEB6
:10960000877AB3EE077A77EE877A3B68C3ED007A04
:1096100000BF1437BD465DF8047B704780B487B047
:1096200000AFF860B9607A60FB6801331B781BB249
:109630001B021AB2FB681B781BB21343FB82B7F9FB
:10964000163007EE903AB8EEE77A2F4BD3ED007A5A
:1096500067EE277ABB68C3ED007AFB6803331B789B
:109660001BB21B021AB2FB6802331B781BB21343F6
:10967000FB82B7F9163007EE903AB8EEE77A224B44
:10968000D3ED007ABB68043367EE277AC3ED007A26
:10969000FB6805331B781BB21B021AB2FB6804334C
:1096A0001B781BB21343FB82B7F9163007EE903AD2
:1096B000B8EEE77A144BD3ED007ABB68083367EE57
:1096C000277AC3ED007AFB6808331B781A04FB681D
:1096D00007331B781B021343FA68063212781343D0
:1096E0003B613B6907EE903AF8EE677A9FED077AA7
:1096F00067EE877A7B68C3ED007A00BF1C37BD46F2
:109700005DF8047B704700BF1000002000401C4241
:1097100080B485B000AF786039607B6801331B7816
:109720001BB21B021AB27B681B781BB21343FB816E
:10973000B7F90E3007EE903AB8EEE77A214BD3ED49
:10974000007A67EE277A3B68C3ED007A7B680333C3
:109750001B781BB21B021AB27B6802331B781BB248
:109760001343FB81B7F90E3007EE903AB8EEE77A73
:10977000144BD3ED007A3B68043367EE277AC3EDD0
:10978000007A7B6805331B781BB21B021AB27B6818
:1097900004331B781BB21343FB81B7F90E3007EE7D
:1097A000903AB8EEE77A074BD3ED007A3B6808337E
:1097B00067EE277AC3ED007A00BF1437BD465DF827
:1097C000047B70471400002080B582B000AF0346D0
:1097D0000A46FB711346BB71FB79184600F09CF8F2
:1097E000BB79184600F098F800BF0837BD4680BD29
:1097F00080B582B000AF03463960FB71FB7963F03E
:109800007F03DBB2184600F087F8552000F084F89B
:1098100003461A463B681A7000BF0837BD4680BD34
:1098200080B582B000AF03463960FB711346BB714F
:10983000FB7963F07F03DBB2184600F06DF80CE0B3
:10984000552000F069F803461A463B681A703B68D9
:1098500001333B60BB79013BBB71BB79002BEFD17E
:1098600000BF00BF0837BD4680BD80B400AF00BF59
:10987000BD465DF8047B704780B400AF00BFBD46B5
:109880005DF8047B704780B582B000AF0346FB8073
:10989000FB881846FCF788FF00BF0837BD4680BD2F
:1098A00080B582B000AF0346FB800120FCF77CFF4F
:1098B00000BF0837BD4680BD80B500AF0022102133
:1098C0000248F8F77DF900BF80BD00BF00000240EC
:1098D00080B500AF012210210248F8F771F900BFEE
:1098E00080BD00BF0000024080B500AF0022012112
:1098F0000248F8F765F900BF80BD00BF00040240D0
:1099000080B500AF012201210248F8F759F900BFE4
:1099100080BD00BF0004024080B586B002AF0346A0
:10992000FB7107F10F02F91D4FF47A7300930123C5
:109930000348F8F786FFFB7B18461037BD4680BD0D
:10994000584A002080B400AF124B1B685A68114B74
:109950001B6842F002025A600E4B1B685A680D4B9E
:109960001B6842F001025A600A4B1B681A68094BD7
:109970001B6842F040021A60074B1B681A68064BCE
:109980001B6842F010021A6000BFBD465DF8047B00
:10999000704700BF584A0020104B002080B485B0AB
:1099A00000AFF860B9601346FB808C4B1B681A68E7
:1099B0008A4B1B6822F001021A60894B1B681A68E7
:1099C000874B1B6822F001021A6007E0834B1B687B
:1099D0001A68824B1B6822F001021A607F4B1B68D9
:1099E0001B6803F00103002BF0D107E07C4B1B68E0
:1099F0001A687B4B1B6822F001021A60784B1B68C7
:109A00001B6803F00103002BF0D1764BDB6C1B6865
:109A10001A46754B9A426CD9724BDB6C1B68734AC1
:109A2000934262D06F4BDB6C1B68714A93425AD0F1
:109A30006C4BDB6C1B686F4A934252D0694BDB6CFA
:109A40001B686D4A93424AD0664BDB6C1B686B4ABD
:109A5000934241D0634BDB6C1B68694A934238D018
:109A6000604BDB6C1B68674A93422FD05D4BDB6C0D
:109A70001B68654A934226D05A4BDB6C1B68634ACD
:109A800093421DD0574BDB6C1B68614A934214D044
:109A9000544BDB6C1B685F4A93420BD0514BDB6C21
:109AA0001B685D4A934202D14FF400131EE04FF051
:109AB00000631BE04FF4001318E04FF4001315E0AF
:109AC0004FF4001312E04FF400630FE04FF4006313
:109AD0000CE04FF4006309E04FF4006306E020233C
:109AE00004E0202302E0202300E020234B4AD3603F
:109AF00097E13C4BDB6C1B681A46494B9A4240F29B
:109B00009180384BDB6C1B68384A934262D0354BEE
:109B1000DB6C1B68364A93425AD0324BDB6C1B68B5
:109B2000344A934252D02F4BDB6C1B68324A93422B
:109B30004AD02C4BDB6C1B68304A934241D0294BF6
:109B4000DB6C1B682E4A934238D0264BDB6C1B68BB
:109B50002C4A93422FD0234BDB6C1B682A4A93423A
:109B600026D0204BDB6C1B68284A93421DD01D4B2E
:109B7000DB6C1B68264A934214D01A4BDB6C1B68C3
:109B8000244A93420BD0174BDB6C1B68224A93424A
:109B900002D14FF400131EE04FF000631BE04FF4BE
:109BA000001318E04FF4001315E04FF4001312E017
:109BB0004FF400630FE04FF400630CE04FF40063D8
:109BC00009E04FF4006306E0202304E0202302E0D4
:109BD000202300E02023114A936022E1104B002053
:109BE000B04A0020584A00205864024010600240E9
:109BF00010640240706002407064024028600240BD
:109C0000286402408860024088640240406002404C
:109C100040640240A0600240A06402400064024030
:109C2000B86002406E4BDB6C1B681A466D4B9A4263
:109C30006CD96B4BDB6C1B686B4A934262D0684BF0
:109C4000DB6C1B68694A93425AD0654BDB6C1B681E
:109C5000674A934252D0624BDB6C1B68654A934261
:109C60004AD05F4BDB6C1B68634A934241D05C4B2C
:109C7000DB6C1B68614A934238D0594BDB6C1B6824
:109C80005F4A93422FD0564BDB6C1B685D4A934270
:109C900026D0534BDB6C1B685B4A93421DD0504B64
:109CA000DB6C1B68594A934214D04D4BDB6C1B682C
:109CB000574A93420BD04A4BDB6C1B68554A934280
:109CC00002D14FF400131EE04FF000631BE04FF48D
:109CD000001318E04FF4001315E04FF4001312E0E6
:109CE0004FF400630FE04FF400630CE04FF40063A7
:109CF00009E04FF4006306E0202304E0202302E0A3
:109D0000202300E02023444AD3608AE0344BDB6CFC
:109D10001B68354A934200F08180314BDB6C1B6835
:109D2000324A93425AD02E4BDB6C1B68304A934226
:109D300052D02B4BDB6C1B682E4A93424AD0284BE7
:109D4000DB6C1B682C4A934241D0254BDB6C1B68B3
:109D50002A4A934238D0224BDB6C1B68284A934234
:109D60002FD01F4BDB6C1B68264A934226D01C4B1E
:109D7000DB6C1B68244A93421DD0194BDB6C1B68BB
:109D8000224A934214D0164BDB6C1B68204A934244
:109D90000BD0134BDB6C1B681E4A934202D14FF46D
:109DA00000133CE04FF0006339E04FF4001336E05D
:109DB0004FF4001333E04FF4001330E04FF400632E
:109DC0002DE04FF400632AE04FF4006327E04FF4E6
:109DD000006324E0202322E0202320E020231EE053
:109DE000584A00205860024010600240106402404F
:109DF00070600240706402402860024028640240A3
:109E00008860024088640240406002404064024032
:109E1000A0600240A0640240006002402023754A16
:109E20009360754BDB6C1B681A46744B9A426CD975
:109E3000714BDB6C1B68724A934262D06E4BDB6CD9
:109E40001B68704A93425AD06B4BDB6C1B686E4A9E
:109E5000934252D0684BDB6C1B686C4A93424AD0E9
:109E6000654BDB6C1B686A4A934241D0624BDB6CEA
:109E70001B68684A934238D05F4BDB6C1B68664AAC
:109E800093422FD05C4BDB6C1B68644A934226D014
:109E9000594BDB6C1B68624A93421DD0564BDB6CFE
:109EA0001B68604A934214D0534BDB6C1B685E4ABC
:109EB00093420BD0504BDB6C1B685C4A934202D13F
:109EC0004FF480131EE04FF080631BE04FF48013CB
:109ED00018E04FF4801315E04FF4801312E04FF4B4
:109EE00080630FE04FF480630CE04FF4806309E07F
:109EF0004FF4806306E0102304E0102302E01023F7
:109F000000E010234A4AD36095E13B4BDB6C1B68B1
:109F10001A46484B9A4240F28F80374BDB6C1B68E5
:109F2000374A934262D0344BDB6C1B68354A93420C
:109F30005AD0314BDB6C1B68334A934252D02E4BC4
:109F4000DB6C1B68314A93424AD02B4BDB6C1B689D
:109F50002F4A934241D0284BDB6C1B682D4A934219
:109F600038D0254BDB6C1B682B4A93422FD0224BF9
:109F7000DB6C1B68294A934226D01F4BDB6C1B68A5
:109F8000274A93421DD01C4BDB6C1B68254A934229
:109F900014D0194BDB6C1B68234A93420BD0164B31
:109FA000DB6C1B68214A934202D14FF480131EE000
:109FB0004FF080631BE04FF4801318E04FF48013E0
:109FC00015E04FF4801312E04FF480630FE04FF47C
:109FD00080630CE04FF4806309E04FF4806306E097
:109FE000102304E0102302E0102300E01023104AA5
:109FF000936020E100600240584A0020586402400B
:10A0000010600240106402407060024070640240C0
:10A010002860024028640240886002408864024050
:10A020004060024040640240A0600240A0640240E0
:10A0300000640240B86002406E4BDB6C1B681A463D
:10A040006D4B9A426CD96B4BDB6C1B686B4A93422D
:10A0500062D0684BDB6C1B68694A93425AD0654BEF
:10A06000DB6C1B68674A934252D0624BDB6C1B6807
:10A07000654A93424AD05F4BDB6C1B68634A93424C
:10A0800041D05C4BDB6C1B68614A934238D0594B22
:10A09000DB6C1B685F4A93422FD0564BDB6C1B680E
:10A0A0005D4A934226D0534BDB6C1B685B4A93425C
:10A0B0001DD0504BDB6C1B68594A934214D04D4B5A
:10A0C000DB6C1B68574A93420BD04A4BDB6C1B6816
:10A0D000554A934202D14FF480131EE04FF0806343
:10A0E0001BE04FF4801318E04FF4801315E04FF499
:10A0F000801312E04FF480630FE04FF480630CE0B4
:10A100004FF4806309E04FF4806306E0102304E01D
:10A11000102302E0102300E01023444AD3608AE0B9
:10A12000344BDB6C1B68354A934200F08180314B25
:10A13000DB6C1B68324A93425AD02E4BDB6C1B6897
:10A14000304A934252D02B4BDB6C1B682E4A934211
:10A150004AD0284BDB6C1B682C4A934241D0254BDC
:10A16000DB6C1B682A4A934238D0224BDB6C1B689D
:10A17000284A93422FD01F4BDB6C1B68264A934220
:10A1800026D01C4BDB6C1B68244A93421DD0194B14
:10A19000DB6C1B68224A934214D0164BDB6C1B68A5
:10A1A000204A93420BD0134BDB6C1B681E4A934230
:10A1B00002D14FF480133CE04FF0806339E04FF45C
:10A1C000801336E04FF4801333E04FF4801330E017
:10A1D0004FF480632DE04FF480632AE04FF48063F6
:10A1E00027E04FF4806324E0102322E0102320E0D6
:10A1F00010231EE0584A00205860024010600240C0
:10A2000010640240706002407064024028600240A6
:10A210002864024088600240886402404060024036
:10A2200040640240A0600240A0640240006002401E
:10A230001023754A9360754BDB6C1B681A46744B90
:10A240009A426CD9714BDB6C1B68724A934262D0A4
:10A250006E4BDB6C1B68704A93425AD06B4BDB6CC5
:10A260001B686E4A934252D0684BDB6C1B686C4A89
:10A2700093424AD0654BDB6C1B686A4A934241D0DB
:10A28000624BDB6C1B68684A934238D05F4BDB6CD7
:10A290001B68664A93422FD05C4BDB6C1B68644A98
:10A2A000934226D0594BDB6C1B68624A93421DD007
:10A2B000564BDB6C1B68604A934214D0534BDB6CEB
:10A2C0001B685E4A93420BD0504BDB6C1B685C4AA8
:10A2D000934202D14FF400231EE04FF000731BE0C5
:10A2E0004FF4002318E04FF4002315E04FF400234F
:10A2F00012E04FF400730FE04FF400730CE04FF4E2
:10A30000007309E04FF4007306E0082304E008231B
:10A3100002E0082300E008234A4AD36095E13B4B62
:10A32000DB6C1B681A46484B9A4240F28F80374BD1
:10A33000DB6C1B68374A934262D0344BDB6C1B6882
:10A34000354A93425AD0314BDB6C1B68334A9342F7
:10A3500052D02E4BDB6C1B68314A93424AD02B4BB8
:10A36000DB6C1B682F4A934241D0284BDB6C1B6887
:10A370002D4A934238D0254BDB6C1B682B4A934205
:10A380002FD0224BDB6C1B68294A934226D01F4BEF
:10A39000DB6C1B68274A93421DD01C4BDB6C1B688F
:10A3A000254A934214D0194BDB6C1B68234A934215
:10A3B0000BD0164BDB6C1B68214A934202D14FF441
:10A3C00000231EE04FF000731BE04FF4002318E061
:10A3D0004FF4002315E04FF4002312E04FF4007314
:10A3E0000FE04FF400730CE04FF4007309E04FF4FA
:10A3F000007306E0082304E0082302E0082300E0DD
:10A400000823104A936020E100600240584A00206F
:10A4100058640240106002401064024070600240C4
:10A420007064024028600240286402408860024054
:10A43000886402404060024040640240A0600240E4
:10A44000A064024000640240B86002406E4BDB6CC6
:10A450001B681A466D4B9A426CD96B4BDB6C1B68C0
:10A460006B4A934262D0684BDB6C1B68694A93422B
:10A470005AD0654BDB6C1B68674A934252D0624BE3
:10A48000DB6C1B68654A93424AD05F4BDB6C1B68F0
:10A49000634A934241D05C4BDB6C1B68614A934238
:10A4A00038D0594BDB6C1B685F4A93422FD0564B18
:10A4B000DB6C1B685D4A934226D0534BDB6C1B68F8
:10A4C0005B4A93421DD0504BDB6C1B68594A934248
:10A4D00014D04D4BDB6C1B68574A93420BD04A4B50
:10A4E000DB6C1B68554A934202D14FF400231EE0F7
:10A4F0004FF000731BE04FF4002318E04FF40023EB
:10A5000015E04FF4002312E04FF400730FE04FF416
:10A5100000730CE04FF4007309E04FF4007306E0A1
:10A52000082304E0082302E0082300E00823444A4B
:10A53000D3608AE0344BDB6C1B68354A934200F0F1
:10A540008180314BDB6C1B68324A93425AD02E4BD0
:10A55000DB6C1B68304A934252D02B4BDB6C1B6880
:10A560002E4A93424AD0284BDB6C1B682C4A9342FC
:10A5700041D0254BDB6C1B682A4A934238D0224BD2
:10A58000DB6C1B68284A93422FD01F4BDB6C1B6887
:10A59000264A934226D01C4BDB6C1B68244A93420C
:10A5A0001DD0194BDB6C1B68224A934214D0164B0A
:10A5B000DB6C1B68204A93420BD0134BDB6C1B688F
:10A5C0001E4A934202D14FF400233CE04FF0007347
:10A5D00039E04FF4002336E04FF4002333E04FF42A
:10A5E000002330E04FF400732DE04FF400732AE0B5
:10A5F0004FF4007327E04FF4007324E0082322E0B7
:10A60000082320E008231EE0584A0020586002403A
:10A6100010600240106402407060024070640240AA
:10A62000286002402864024088600240886402403A
:10A630004060024040640240A0600240A0640240CA
:10A64000006002400823754A9360754BDB6C1B6801
:10A650001A46744B9A426CD9714BDB6C1B68724A78
:10A66000934262D06E4BDB6C1B68704A93425AD0A7
:10A670006B4BDB6C1B686E4A934252D0684BDB6CB1
:10A680001B686C4A93424AD0654BDB6C1B686A4A74
:10A69000934241D0624BDB6C1B68684A934238D0CE
:10A6A0005F4BDB6C1B68664A93422FD05C4BDB6CC4
:10A6B0001B68644A934226D0594BDB6C1B68624A84
:10A6C00093421DD0564BDB6C1B68604A934214D0FA
:10A6D000534BDB6C1B685E4A93420BD0504BDB6CD8
:10A6E0001B685C4A934202D14FF480231EE04FF076
:10A6F00080731BE04FF4802318E04FF4802315E0B3
:10A700004FF4802312E04FF480730FE04FF4807316
:10A710000CE04FF4807309E04FF4807306E00423EB
:10A7200004E0042302E0042300E004234A4AD36047
:10A7300095E13B4BDB6C1B681A46484B9A4240F252
:10A740008F80374BDB6C1B68374A934262D0344BA7
:10A75000DB6C1B68354A93425AD0314BDB6C1B686B
:10A76000334A934252D02E4BDB6C1B68314A9342E2
:10A770004AD02B4BDB6C1B682F4A934241D0284BAD
:10A78000DB6C1B682D4A934238D0254BDB6C1B6871
:10A790002B4A93422FD0224BDB6C1B68294A9342F1
:10A7A00026D01F4BDB6C1B68274A93421DD01C4BE5
:10A7B000DB6C1B68254A934214D0194BDB6C1B6879
:10A7C000234A93420BD0164BDB6C1B68214A934201
:10A7D00002D14FF480231EE04FF080731BE04FF452
:10A7E000802318E04FF4802315E04FF4802312E01B
:10A7F0004FF480730FE04FF480730CE04FF48073DC
:10A8000009E04FF4807306E0042304E0042302E02F
:10A81000042300E00423104A936020E1006002401A
:10A82000584A002058640240106002401064024000
:10A830007060024070640240286002402864024058
:10A8400088600240886402404060024040640240E8
:10A85000A0600240A064024000640240B860024070
:10A860006E4BDB6C1B681A466D4B9A426CD96B4B76
:10A87000DB6C1B686B4A934262D0684BDB6C1B68D5
:10A88000694A93425AD0654BDB6C1B68674A934216
:10A8900052D0624BDB6C1B68654A93424AD05F4BD7
:10A8A000DB6C1B68634A934241D05C4BDB6C1B68DA
:10A8B000614A934238D0594BDB6C1B685F4A934224
:10A8C0002FD0564BDB6C1B685D4A934226D0534B0E
:10A8D000DB6C1B685B4A93421DD0504BDB6C1B68E2
:10A8E000594A934214D04D4BDB6C1B68574A934234
:10A8F0000BD04A4BDB6C1B68554A934202D14FF494
:10A9000080231EE04FF080731BE04FF4802318E09B
:10A910004FF4802315E04FF4802312E04FF480734E
:10A920000FE04FF480730CE04FF4807309E04FF4B4
:10A93000807306E0042304E0042302E0042300E023
:10A940000423444AD3608AE0344BDB6C1B68354AED
:10A95000934200F08180314BDB6C1B68324A93429A
:10A960005AD02E4BDB6C1B68304A934252D02B4B93
:10A97000DB6C1B682E4A93424AD0284BDB6C1B6869
:10A980002C4A934241D0254BDB6C1B682A4A9342E8
:10A9900038D0224BDB6C1B68284A93422FD01F4BC8
:10A9A000DB6C1B68264A934226D01C4BDB6C1B6871
:10A9B000244A93421DD0194BDB6C1B68224A9342F8
:10A9C00014D0164BDB6C1B68204A93420BD0134B00
:10A9D000DB6C1B681E4A934202D14FF480233CE09B
:10A9E0004FF0807339E04FF4802336E04FF480233A
:10A9F00033E04FF4802330E04FF480732DE04FF4C8
:10AA000080732AE04FF4807327E04FF4807324E0D2
:10AA1000042322E0042320E004231EE0584A0020FF
:10AA200058600240106002401064024070600240B2
:10AA3000706402402860024028640240886002403E
:10AA4000886402404060024040640240A0600240CE
:10AA5000A0640240006002400423714A9360714B7D
:10AA6000DB6C1B681A46704B9A4268D96D4BDB6CE5
:10AA70001B686E4A93425ED06A4BDB6C1B686C4A63
:10AA8000934256D0674BDB6C1B686A4A93424ED0A8
:10AA9000644BDB6C1B68684A934246D0614BDB6CAD
:10AAA0001B68664A93423ED05E4BDB6C1B68644A6F
:10AAB000934236D05B4BDB6C1B68624A93422ED0CC
:10AAC000584BDB6C1B68604A934226D0554BDB6CBD
:10AAD0001B685E4A93421DD0524BDB6C1B685C4A7C
:10AAE000934214D04F4BDB6C1B685A4A93420BD0F5
:10AAF0004C4BDB6C1B68584A934202D14FF48033B5
:10AB00001AE04FF4800317E04FF4803314E04FF461
:10AB1000803311E04FF480330EE040230CE04023FB
:10AB20000AE0402308E0402306E0012304E001237B
:10AB300002E0012300E00123484AD36089E1394B58
:10AB4000DB6C1B681A46464B9A4240F28B80354BB1
:10AB5000DB6C1B68354A93425ED0324BDB6C1B6862
:10AB6000334A934256D02F4BDB6C1B68314A9342D9
:10AB70004ED02C4BDB6C1B682F4A934246D0294B9E
:10AB8000DB6C1B682D4A93423ED0264BDB6C1B6866
:10AB90002B4A934236D0234BDB6C1B68294A9342E5
:10ABA0002ED0204BDB6C1B68274A934226D01D4BCE
:10ABB000DB6C1B68254A93421DD01A4BDB6C1B686B
:10ABC000234A934214D0174BDB6C1B68214A9342F3
:10ABD0000BD0144BDB6C1B681F4A934202D14FF41D
:10ABE00080331AE04FF4800317E04FF4803314E011
:10ABF0004FF4803311E04FF480330EE040230CE03B
:10AC000040230AE0402308E0402306E0012304E05B
:10AC1000012302E0012300E00123104A936018E1C0
:10AC200000600240584A0020586402401060024010
:10AC3000106402407060024070640240286002406C
:10AC400028640240886002408864024040600240FC
:10AC500040640240A0600240A064024000640240E0
:10AC6000B86002406A4BDB6C1B681A46694B9A421B
:10AC700068D9674BDB6C1B68674A93425ED0644BB4
:10AC8000DB6C1B68654A934256D0614BDB6C1B68DA
:10AC9000634A93424ED05E4BDB6C1B68614A934221
:10ACA00046D05B4BDB6C1B685F4A93423ED0584BEF
:10ACB000DB6C1B685D4A934236D0554BDB6C1B68DE
:10ACC0005B4A93422ED0524BDB6C1B68594A93422D
:10ACD00026D04F4BDB6C1B68574A93421DD04C4B20
:10ACE000DB6C1B68554A934214D0494BDB6C1B68E4
:10ACF000534A93420BD0464BDB6C1B68514A93423C
:10AD000002D14FF480331AE04FF4800317E04FF480
:10AD1000803314E04FF4803311E04FF480330EE0C1
:10AD200040230CE040230AE0402308E0402306E0F3
:10AD3000012304E0012302E0012300E00123424A51
:10AD4000D36086E0324BDB6C1B68334A93427DD084
:10AD50002F4BDB6C1B68314A934256D02C4BDB6C7B
:10AD60001B682F4A93424ED0294BDB6C1B682D4A3F
:10AD7000934246D0264BDB6C1B682B4A93423ED055
:10AD8000234BDB6C1B68294A934236D0204BDB6C8B
:10AD90001B68274A93422ED01D4BDB6C1B68254A4B
:10ADA000934226D01A4BDB6C1B68234A93421DD07A
:10ADB000174BDB6C1B68214A934214D0144BDB6C9D
:10ADC0001B681F4A93420BD0114BDB6C1B681D4A5A
:10ADD000934202D14FF4803339E04FF4800336E0E0
:10ADE0004FF4803333E04FF4803330E04FF480335E
:10ADF0002DE040232BE0402329E0402327E040239F
:10AE000025E0012323E0012321E001231FE000BF0F
:10AE1000584A00205860024010600240106402400E
:10AE20007060024070640240286002402864024062
:10AE300088600240886402404060024040640240F2
:10AE4000A0600240A0640240006002400123754AF5
:10AE50009360754B9B6C1B681A46744B9A426CD975
:10AE6000714B9B6C1B68724A934262D06E4B9B6C19
:10AE70001B68704A93425AD06B4B9B6C1B686E4A9E
:10AE8000934252D0684B9B6C1B686C4A93424AD0E9
:10AE9000654B9B6C1B686A4A934241D0624B9B6C2A
:10AEA0001B68684A934238D05F4B9B6C1B68664AAC
:10AEB00093422FD05C4B9B6C1B68644A934226D014
:10AEC000594B9B6C1B68624A93421DD0564B9B6C3E
:10AED0001B68604A934214D0534B9B6C1B685E4ABC
:10AEE00093420BD0504B9B6C1B685C4A934202D13F
:10AEF0004FF400131EE04FF000631BE04FF400130B
:10AF000018E04FF4001315E04FF4001312E04FF473
:10AF100000630FE04FF400630CE04FF4006309E0BE
:10AF20004FF4006306E0202304E0202302E0202306
:10AF300000E020234A4AD36095E13B4B9B6C1B68A1
:10AF40001A46484B9A4240F28F80374B9B6C1B68E5
:10AF5000374A934262D0344B9B6C1B68354A93420C
:10AF60005AD0314B9B6C1B68334A934252D02E4BC4
:10AF70009B6C1B68314A93424AD02B4B9B6C1B68DD
:10AF80002F4A934241D0284B9B6C1B682D4A934219
:10AF900038D0254B9B6C1B682B4A93422FD0224BF9
:10AFA0009B6C1B68294A934226D01F4B9B6C1B68E5
:10AFB000274A93421DD01C4B9B6C1B68254A934229
:10AFC00014D0194B9B6C1B68234A93420BD0164B31
:10AFD0009B6C1B68214A934202D14FF400131EE080
:10AFE0004FF000631BE04FF4001318E04FF4001320
:10AFF00015E04FF4001312E04FF400630FE04FF43C
:10B0000000630CE04FF4006309E04FF4006306E0D6
:10B01000202304E0202302E0202300E02023104A24
:10B02000936020E100600240584A002058640240CA
:10B030001060024010640240706002407064024080
:10B040002860024028640240886002408864024010
:10B050004060024040640240A0600240A0640240A0
:10B0600000640240B86002406E4B9B6C1B681A463D
:10B070006D4B9A426CD96B4B9B6C1B686B4A93422D
:10B0800062D0684B9B6C1B68694A93425AD0654BEF
:10B090009B6C1B68674A934252D0624B9B6C1B6847
:10B0A000654A93424AD05F4B9B6C1B68634A93424C
:10B0B00041D05C4B9B6C1B68614A934238D0594B22
:10B0C0009B6C1B685F4A93422FD0564B9B6C1B684E
:10B0D0005D4A934226D0534B9B6C1B685B4A93425C
:10B0E0001DD0504B9B6C1B68594A934214D04D4B5A
:10B0F0009B6C1B68574A93420BD04A4B9B6C1B6856
:10B10000554A934202D14FF400131EE04FF0006302
:10B110001BE04FF4001318E04FF4001315E04FF458
:10B12000001312E04FF400630FE04FF400630CE0F3
:10B130004FF4006309E04FF4006306E0202304E0CD
:10B14000202302E0202300E02023444AD3608AE049
:10B15000344B9B6C1B68354A934200F08180314B25
:10B160009B6C1B68324A93425AD02E4B9B6C1B68D7
:10B17000304A934252D02B4B9B6C1B682E4A934211
:10B180004AD0284B9B6C1B682C4A934241D0254BDC
:10B190009B6C1B682A4A934238D0224B9B6C1B68DD
:10B1A000284A93422FD01F4B9B6C1B68264A934220
:10B1B00026D01C4B9B6C1B68244A93421DD0194B14
:10B1C0009B6C1B68224A934214D0164B9B6C1B68E5
:10B1D000204A93420BD0134B9B6C1B681E4A934230
:10B1E00002D14FF400133CE04FF0006339E04FF41C
:10B1F000001336E04FF4001333E04FF4001330E057
:10B200004FF400632DE04FF400632AE04FF4006335
:10B2100027E04FF4006324E0202322E0202320E0F5
:10B2200020231EE0584A002058600240106002406F
:10B230001064024070600240706402402860024066
:10B2400028640240886002408864024040600240F6
:10B2500040640240A0600240A064024000600240DE
:10B260002023754A9360754B9B6C1B681A46744B80
:10B270009A426CD9714B9B6C1B68724A934262D0A4
:10B280006E4B9B6C1B68704A93425AD06B4B9B6C05
:10B290001B686E4A934252D0684B9B6C1B686C4A89
:10B2A00093424AD0654B9B6C1B686A4A934241D0DB
:10B2B000624B9B6C1B68684A934238D05F4B9B6C17
:10B2C0001B68664A93422FD05C4B9B6C1B68644A98
:10B2D000934226D0594B9B6C1B68624A93421DD007
:10B2E000564B9B6C1B68604A934214D0534B9B6C2B
:10B2F0001B685E4A93420BD0504B9B6C1B685C4AA8
:10B30000934202D14FF480131EE04FF080631BE0A4
:10B310004FF4801318E04FF4801315E04FF48013BE
:10B3200012E04FF480630FE04FF480630CE04FF4C1
:10B33000806309E04FF4806306E0102304E01023EB
:10B3400002E0102300E010234A4AD36095E13B4B12
:10B350009B6C1B681A46484B9A4240F28F80374BD1
:10B360009B6C1B68374A934262D0344B9B6C1B68C2
:10B37000354A93425AD0314B9B6C1B68334A9342F7
:10B3800052D02E4B9B6C1B68314A93424AD02B4BB8
:10B390009B6C1B682F4A934241D0284B9B6C1B68C7
:10B3A0002D4A934238D0254B9B6C1B682B4A934205
:10B3B0002FD0224B9B6C1B68294A934226D01F4BEF
:10B3C0009B6C1B68274A93421DD01C4B9B6C1B68CF
:10B3D000254A934214D0194B9B6C1B68234A934215
:10B3E0000BD0164B9B6C1B68214A934202D14FF441
:10B3F00080131EE04FF080631BE04FF4801318E0D1
:10B400004FF4801315E04FF4801312E04FF4806383
:10B410000FE04FF480630CE04FF4806309E04FF4D9
:10B42000806306E0102304E0102302E0102300E014
:10B430001023104A936020E100600240584A002027
:10B440005864024010600240106402407060024084
:10B450007064024028600240286402408860024014
:10B46000886402404060024040640240A0600240A4
:10B47000A064024000640240B86002406E4B9B6CC6
:10B480001B681A466D4B9A426CD96B4B9B6C1B68C0
:10B490006B4A934262D0684B9B6C1B68694A93422B
:10B4A0005AD0654B9B6C1B68674A934252D0624BE3
:10B4B0009B6C1B68654A93424AD05F4B9B6C1B6830
:10B4C000634A934241D05C4B9B6C1B68614A934238
:10B4D00038D0594B9B6C1B685F4A93422FD0564B18
:10B4E0009B6C1B685D4A934226D0534B9B6C1B6838
:10B4F0005B4A93421DD0504B9B6C1B68594A934248
:10B5000014D04D4B9B6C1B68574A93420BD04A4B4F
:10B510009B6C1B68554A934202D14FF480131EE086
:10B520004FF080631BE04FF4801318E04FF480135A
:10B5300015E04FF4801312E04FF480630FE04FF4F6
:10B5400080630CE04FF4806309E04FF4806306E011
:10B55000102304E0102302E0102300E01023444AEB
:10B56000D3608AE0344B9B6C1B68354A934200F0F1
:10B570008180314B9B6C1B68324A93425AD02E4BD0
:10B580009B6C1B68304A934252D02B4B9B6C1B68C0
:10B590002E4A93424AD0284B9B6C1B682C4A9342FC
:10B5A00041D0254B9B6C1B682A4A934238D0224BD2
:10B5B0009B6C1B68284A93422FD01F4B9B6C1B68C7
:10B5C000264A934226D01C4B9B6C1B68244A93420C
:10B5D0001DD0194B9B6C1B68224A934214D0164B0A
:10B5E0009B6C1B68204A93420BD0134B9B6C1B68CF
:10B5F0001E4A934202D14FF480133CE04FF0806327
:10B6000039E04FF4801336E04FF4801333E04FF409
:10B61000801330E04FF480632DE04FF480632AE024
:10B620004FF4806327E04FF4806324E0102322E08E
:10B63000102320E010231EE0584A002058600240EA
:10B64000106002401064024070600240706402406A
:10B6500028600240286402408860024088640240FA
:10B660004060024040640240A0600240A06402408A
:10B67000006002401023754A9360754B9B6C1B68F9
:10B680001A46744B9A426CD9714B9B6C1B68724A78
:10B69000934262D06E4B9B6C1B68704A93425AD0A7
:10B6A0006B4B9B6C1B686E4A934252D0684B9B6CF1
:10B6B0001B686C4A93424AD0654B9B6C1B686A4A74
:10B6C000934241D0624B9B6C1B68684A934238D0CE
:10B6D0005F4B9B6C1B68664A93422FD05C4B9B6C04
:10B6E0001B68644A934226D0594B9B6C1B68624A84
:10B6F00093421DD0564B9B6C1B68604A934214D0FA
:10B70000534B9B6C1B685E4A93420BD0504B9B6C17
:10B710001B685C4A934202D14FF400231EE04FF0B5
:10B7200000731BE04FF4002318E04FF4002315E0F2
:10B730004FF4002312E04FF400730FE04FF4007356
:10B740000CE04FF4007309E04FF4007306E00823A7
:10B7500004E0082302E0082300E008234A4AD360FB
:10B7600095E13B4B9B6C1B681A46484B9A4240F252
:10B770008F80374B9B6C1B68374A934262D0344BA7
:10B780009B6C1B68354A93425AD0314B9B6C1B68AB
:10B79000334A934252D02E4B9B6C1B68314A9342E2
:10B7A0004AD02B4B9B6C1B682F4A934241D0284BAD
:10B7B0009B6C1B682D4A934238D0254B9B6C1B68B1
:10B7C0002B4A93422FD0224B9B6C1B68294A9342F1
:10B7D00026D01F4B9B6C1B68274A93421DD01C4BE5
:10B7E0009B6C1B68254A934214D0194B9B6C1B68B9
:10B7F000234A93420BD0164B9B6C1B68214A934201
:10B8000002D14FF400231EE04FF000731BE04FF411
:10B81000002318E04FF4002315E04FF4002312E05A
:10B820004FF400730FE04FF400730CE04FF400731B
:10B8300009E04FF4007306E0082304E0082302E067
:10B84000082300E00823104A936020E100600240D2
:10B85000584A0020586402401060024010640240C0
:10B860007060024070640240286002402864024018
:10B8700088600240886402404060024040640240A8
:10B88000A0600240A064024000640240B860024030
:10B890006E4B9B6C1B681A466D4B9A426CD96B4B76
:10B8A0009B6C1B686B4A934262D0684B9B6C1B6815
:10B8B000694A93425AD0654B9B6C1B68674A934216
:10B8C00052D0624B9B6C1B68654A93424AD05F4BD7
:10B8D0009B6C1B68634A934241D05C4B9B6C1B681A
:10B8E000614A934238D0594B9B6C1B685F4A934224
:10B8F0002FD0564B9B6C1B685D4A934226D0534B0E
:10B900009B6C1B685B4A93421DD0504B9B6C1B6821
:10B91000594A934214D04D4B9B6C1B68574A934233
:10B920000BD04A4B9B6C1B68554A934202D14FF493
:10B9300000231EE04FF000731BE04FF4002318E0DB
:10B940004FF4002315E04FF4002312E04FF400738E
:10B950000FE04FF400730CE04FF4007309E04FF474
:10B96000007306E0082304E0082302E0082300E057
:10B970000823444AD3608AE0344B9B6C1B68354AE9
:10B98000934200F08180314B9B6C1B68324A93429A
:10B990005AD02E4B9B6C1B68304A934252D02B4B93
:10B9A0009B6C1B682E4A93424AD0284B9B6C1B68A9
:10B9B0002C4A934241D0254B9B6C1B682A4A9342E8
:10B9C00038D0224B9B6C1B68284A93422FD01F4BC8
:10B9D0009B6C1B68264A934226D01C4B9B6C1B68B1
:10B9E000244A93421DD0194B9B6C1B68224A9342F8
:10B9F00014D0164B9B6C1B68204A93420BD0134B00
:10BA00009B6C1B681E4A934202D14FF400233CE01A
:10BA10004FF0007339E04FF4002336E04FF4002379
:10BA200033E04FF4002330E04FF400732DE04FF487
:10BA300000732AE04FF4007327E04FF4007324E012
:10BA4000082322E0082320E008231EE0584A0020B3
:10BA50005860024010600240106402407060024072
:10BA600070640240286002402864024088600240FE
:10BA7000886402404060024040640240A06002408E
:10BA8000A0640240006002400823754A9360754B31
:10BA90009B6C1B681A46744B9A426CD9714B9B6C19
:10BAA0001B68724A934262D06E4B9B6C1B68704A53
:10BAB00093425AD06B4B9B6C1B686E4A934252D098
:10BAC000684B9B6C1B686C4A93424AD0654B9B6CDD
:10BAD0001B686A4A934241D0624B9B6C1B68684A60
:10BAE000934238D05F4B9B6C1B68664A93422FD0C1
:10BAF0005C4B9B6C1B68644A934226D0594B9B6CF1
:10BB00001B68624A93421DD0564B9B6C1B68604A6F
:10BB1000934214D0534B9B6C1B685E4A93420BD0EC
:10BB2000504B9B6C1B685C4A934202D14FF48023BC
:10BB30001EE04FF080731BE04FF4802318E04FF4B9
:10BB4000802315E04FF4802312E04FF480730FE060
:10BB50004FF480730CE04FF4807309E04FF480736E
:10BB600006E0042304E0042302E0042300E00423AD
:10BB70004A4AD36095E13B4B9B6C1B681A46484B85
:10BB80009A4240F28F80374B9B6C1B68374A934236
:10BB900062D0344B9B6C1B68354A93425AD0314B70
:10BBA0009B6C1B68334A934252D02E4B9B6C1B6894
:10BBB000314A93424AD02B4B9B6C1B682F4A9342CD
:10BBC00041D0284B9B6C1B682D4A934238D0254BA3
:10BBD0009B6C1B682B4A93422FD0224B9B6C1B689B
:10BBE000294A934226D01F4B9B6C1B68274A9342DD
:10BBF0001DD01C4B9B6C1B68254A934214D0194BDB
:10BC00009B6C1B68234A93420BD0164B9B6C1B68A2
:10BC1000214A934202D14FF480231EE04FF08073FB
:10BC20001BE04FF4802318E04FF4802315E04FF41D
:10BC3000802312E04FF480730FE04FF480730CE028
:10BC40004FF4807309E04FF4807306E0042304E0AE
:10BC5000042302E0042300E00423104A936020E15F
:10BC600000600240584A00205864024010600240C0
:10BC7000106402407060024070640240286002401C
:10BC800028640240886002408864024040600240AC
:10BC900040640240A0600240A06402400064024090
:10BCA000B86002406E4B9B6C1B681A466D4B9A4203
:10BCB0006CD96B4B9B6C1B686B4A934262D0684B90
:10BCC0009B6C1B68694A93425AD0654B9B6C1B68FE
:10BCD000674A934252D0624B9B6C1B68654A934201
:10BCE0004AD05F4B9B6C1B68634A934241D05C4BCC
:10BCF0009B6C1B68614A934238D0594B9B6C1B6804
:10BD00005F4A93422FD0564B9B6C1B685D4A93420F
:10BD100026D0534B9B6C1B685B4A93421DD0504B03
:10BD20009B6C1B68594A934214D04D4B9B6C1B680B
:10BD3000574A93420BD04A4B9B6C1B68554A93421F
:10BD400002D14FF480231EE04FF080731BE04FF4CC
:10BD5000802318E04FF4802315E04FF4802312E095
:10BD60004FF480730FE04FF480730CE04FF4807356
:10BD700009E04FF4807306E0042304E0042302E0AA
:10BD8000042300E00423444AD3608AE0344B9B6CD4
:10BD90001B68354A934200F08180314B9B6C1B68D5
:10BDA000324A93425AD02E4B9B6C1B68304A9342C6
:10BDB00052D02B4B9B6C1B682E4A93424AD0284B87
:10BDC0009B6C1B682C4A934241D0254B9B6C1B6893
:10BDD0002A4A934238D0224B9B6C1B68284A9342D4
:10BDE0002FD01F4B9B6C1B68264A934226D01C4BBE
:10BDF0009B6C1B68244A93421DD0194B9B6C1B689B
:10BE0000224A934214D0164B9B6C1B68204A9342E3
:10BE10000BD0134B9B6C1B681E4A934202D14FF40C
:10BE200080233CE04FF0807339E04FF4802336E00C
:10BE30004FF4802333E04FF4802330E04FF48073DD
:10BE40002DE04FF480732AE04FF4807327E04FF425
:10BE5000807324E0042322E0042320E004231EE076
:10BE6000584A0020586002401060024010640240AE
:10BE70007060024070640240286002402864024002
:10BE80008860024088640240406002404064024092
:10BE9000A0600240A0640240006002400423714A96
:10BEA0009360714B9B6C1B681A46704B9A4268D921
:10BEB0006D4B9B6C1B686E4A93425ED06A4B9B6CC9
:10BEC0001B686C4A934256D0674B9B6C1B686A4A4E
:10BED00093424ED0644B9B6C1B68684A934246D099
:10BEE000614B9B6C1B68664A93423ED05E4B9B6CD9
:10BEF0001B68644A934236D05B4B9B6C1B68624A5A
:10BF000093422ED0584B9B6C1B68604A934226D0BC
:10BF1000554B9B6C1B685E4A93421DD0524B9B6CE9
:10BF20001B685C4A934214D04F4B9B6C1B685A4A67
:10BF300093420BD04C4B9B6C1B68584A934202D1E6
:10BF40004FF480331AE04FF4800317E04FF480334E
:10BF500014E04FF4803311E04FF480330EE04023BF
:10BF60000CE040230AE0402308E0402306E00123E0
:10BF700004E0012302E0012300E00123484AD360EA
:10BF80006AE1394B9B6C1B681A46464B9A4240F259
:10BF90008B80354B9B6C1B68354A93425ED0324B8D
:10BFA0009B6C1B68334A934256D02F4B9B6C1B688B
:10BFB000314A93424ED02C4B9B6C1B682F4A9342C4
:10BFC00046D0294B9B6C1B682D4A93423ED0264B92
:10BFD0009B6C1B682B4A934236D0234B9B6C1B688F
:10BFE000294A93422ED0204B9B6C1B68274A9342D0
:10BFF00026D01D4B9B6C1B68254A93421DD01A4BC3
:10C000009B6C1B68234A934214D0174B9B6C1B6894
:10C01000214A93420BD0144B9B6C1B681F4A9342DE
:10C0200002D14FF480331AE04FF4800317E04FF44D
:10C03000803314E04FF4803311E04FF480330EE08E
:10C0400040230CE040230AE0402308E0402306E0C0
:10C05000012304E0012302E0012300E00123104A50
:10C060009360F9E000600240584A002058640240A2
:10C070001060024010640240706002407064024030
:10C0800028600240286402408860024088640240C0
:10C090004060024040640240A0600240A064024050
:10C0A00000640240B8600240824B9B6C1B681A46D9
:10C0B000814B9A4268D97F4B9B6C1B687F4A9342A5
:10C0C0005ED07C4B9B6C1B687D4A934256D0794B6B
:10C0D0009B6C1B687B4A93424ED0764B9B6C1B68D3
:10C0E000794A934246D0734B9B6C1B68774A9342C4
:10C0F0003ED0704B9B6C1B68754A934236D06D4B9B
:10C100009B6C1B68734A93422ED06A4B9B6C1B68D6
:10C11000714A934226D0674B9B6C1B686F4A9342CF
:10C120001DD0644B9B6C1B686D4A934214D0614BCD
:10C130009B6C1B686B4A93420BD05E4B9B6C1B68DD
:10C14000694A934202D14FF480331AE04FF48003DE
:10C1500017E04FF4803314E04FF4803311E04FF4D4
:10C1600080330EE040230CE040230AE0402308E047
:10C17000402306E0012304E0012302E0012300E064
:10C1800001235A4AD36067E04A4B9B6C1B684B4AB9
:10C1900093425ED0474B9B6C1B68494A934256D0F2
:10C1A000444B9B6C1B68474A93424ED0414B9B6C5F
:10C1B0001B68454A934246D03E4B9B6C1B68434AE2
:10C1C00093423ED03B4B9B6C1B68414A934236D016
:10C1D000384B9B6C1B683F4A93422ED0354B9B6C6F
:10C1E0001B683D4A934226D0324B9B6C1B683B4AEE
:10C1F00093421DD02F4B9B6C1B68394A934214D03D
:10C200002C4B9B6C1B68374A93420BD0294B9B6C81
:10C210001B68354A934202D14FF480331AE04FF441
:10C22000800317E04FF4803314E04FF4803311E0C3
:10C230004FF480330EE040230CE040230AE040231B
:10C2400008E0402306E0012304E0012302E001238B
:10C2500000E00123254A9360254B1B68BA68DA6029
:10C26000234B1B68234A9A60234B1B68FA68DA60E9
:10C27000214B1B681F4A9A601D4B1B68FA885A6045
:10C280001D4B1B68FA885A60194B1B681A68184BBB
:10C290001B6842F001021A60174B1B681A68164BA4
:10C2A0001B6842F001021A6000BF1437BD465DF8FA
:10C2B000047B7047584A00205860024010600240DA
:10C2C00010640240706002407064024028600240C6
:10C2D0002864024088600240886402404060024056
:10C2E00040640240A0600240A0640240006002403E
:10C2F000104B00200C300140B04A002080B483B0C5
:10C3000000AF786087ED000A7B684FF07E521A60BC
:10C310007B684FF000025A607B684FF000029A6021
:10C320007B684FF00002DA607B683A681A617B68CC
:10C330004FF000025A617B684FF000029A617B68FF
:10C340004FF00002DA617B6818460C37BD465DF895
:10C35000047B704780B52DED028B92B000AFF86181
:10C3600087ED060AC7ED050A87ED041AC7ED031A23
:10C3700087ED022AC7ED012AD7ED037AF5EE407A60
:10C38000F1EE10FA0ED1D7ED027AF5EE407AF1EE29
:10C3900010FA07D1D7ED017AF5EE407AF1EE10FAF6
:10C3A00000F0FE80D7ED037A27EEA77AD7ED027A68
:10C3B00067EEA77A37EE277AD7ED017A67EEA77A8C
:10C3C00077EE277AB0EE670A00F064FA87ED110A7B
:10C3D00097ED037AD7ED117A67EE277AC7ED037AE6
:10C3E00097ED027AD7ED117A67EE277AC7ED027AD8
:10C3F00097ED017AD7ED117A67EE277AC7ED017ACA
:10C40000FB690121184601F04DFA034693ED008ABD
:10C41000FB690321184601F045FA0346D3ED007A83
:10C4200028EE278AFB690021184601F03BFA0346F3
:10C43000D3ED008AFB690221184601F033FA034666
:10C44000D3ED007A68EEA77A78EE677AC7ED107AB6
:10C45000FB690021184601F025FA034693ED008A96
:10C46000FB690121184601F01DFA0346D3ED007A5D
:10C4700028EE278AFB690221184601F013FA0346C9
:10C48000D3ED008AFB690321184601F00BFA03463D
:10C49000D3ED007A68EEA77A78EE277AC7ED0F7AA7
:10C4A000FB690021184601F0FDF9034693ED008A6F
:10C4B000FB690021184601F0F5F90346D3ED007A37
:10C4C00068EE277AB6EE007A37EEC78AFB69032159
:10C4D000184601F0E7F90346D3ED008AFB69032112
:10C4E000184601F0DFF90346D3ED007A68EEA77A2B
:10C4F00078EE277AC7ED0E7A97ED027AD7ED0E7AAD
:10C5000027EE277AD7ED016AD7ED0F7A66EEA77A84
:10C5100077EE677AC7ED0D7A97ED017AD7ED107A4D
:10C5200027EE277AD7ED036AD7ED0E7A66EEA77A63
:10C5300077EE677AC7ED0C7A97ED037AD7ED0F7A2D
:10C5400027EE277AD7ED026AD7ED107A66EEA77A42
:10C5500077EE677AC7ED0B7AFB694FF000025A61FC
:10C56000FB694FF000029A61FB694FF00002DA614B
:10C5700097ED067AD7ED0D7A77EE277AC7ED067A32
:10C5800097ED057AD7ED0C7A77EE277AC7ED057A25
:10C5900097ED047AD7ED0B7A77EE277AC7ED047A18
:10C5A000FB6993ED047AF7EE006AC6EE877AB6EE81
:10C5B000007A67EE877A97ED067A67EE277AC7EDFD
:10C5C000067AFB6993ED047AF7EE006AC6EE877A85
:10C5D000B6EE007A67EE877A97ED057A67EE277AEE
:10C5E000C7ED057AFB6993ED047AF7EE006AC6EEB3
:10C5F000877AB6EE007A67EE877A97ED047A67EE6F
:10C60000277AC7ED047AFB690021184601F04AF940
:10C6100003461B68BB62FB690121184601F042F921
:10C6200003461B687B62FB690221184601F03AF958
:10C6300003461B683B62D7ED097AB1EE677AD7ED06
:10C64000067A27EE277AD7ED086AD7ED057A66EEE7
:10C65000A77A37EE678AFB690321184601F022F9B1
:10C66000034693ED007AD7ED047A67EE277A38EE29
:10C67000678AFB690021184601F014F90346D3EDDF
:10C68000007A78EE277AC3ED007A97ED0A7AD7ED33
:10C69000067A27EE277AD7ED086AD7ED047A66EE98
:10C6A000A77A37EE278AFB690321184601F0FAF8CA
:10C6B000034693ED007AD7ED057A67EE277A38EED8
:10C6C000678AFB690121184601F0ECF80346D3EDB7
:10C6D000007A78EE277AC3ED007A97ED0A7AD7EDE3
:10C6E000057A27EE277AD7ED096AD7ED047A66EE48
:10C6F000A77A37EE678AFB690321184601F0D2F862
:10C70000034693ED007AD7ED067A67EE277A38EE86
:10C71000278AFB690221184601F0C4F80346D3EDCD
:10C72000007A78EE277AC3ED007AFB690321184678
:10C7300001F0B8F8034693ED007AD7ED0A6AD7ED19
:10C74000047A66EEA76A97ED096AD7ED057A66EE78
:10C75000277A76EEA76A97ED086AD7ED067A66EE35
:10C76000277A76EEE77A77EE277AC3ED007AFB69CF
:10C770000021184601F096F8034693ED008AFB6904
:10C780000021184601F08EF80346D3ED007A28EE1A
:10C79000278AFB690121184601F084F80346D3ED8E
:10C7A000008AFB690121184601F07CF80346D3EDAD
:10C7B000007A68EEA77A38EE278AFB6902211846CC
:10C7C00001F070F80346D3ED008AFB690221184698
:10C7D00001F068F80346D3ED007A68EEA77A38EEE8
:10C7E000278AFB690321184601F05CF80346D3ED64
:10C7F000008AFB690321184601F054F80346D3ED83
:10C80000007A68EEA77A78EE277AB0EE670A00F031
:10C8100041F887ED110AFB690021184601F042F842
:10C82000034693ED007AD7ED117A67EE277AC3EDD0
:10C83000007AFB690121184601F034F8034693EDB4
:10C84000007AD7ED117A67EE277AC3ED007AFB699B
:10C850000221184601F026F8034693ED007AD7ED41
:10C86000117A67EE277AC3ED007AFB690321184637
:10C8700001F018F8034693ED007AD7ED117A67EED0
:10C88000277AC3ED007A00BF4837BD46BDEC028B66
:10C8900080BD000080B487B000AF87ED010AD7EDFE
:10C8A000017AB6EE007A67EE877AC7ED057A7B6883
:10C8B0003B6107F110031B68FB60FB685A10124BC9
:10C8C0009B1AFB6007F10C031B683B6197ED047A30
:10C8D000D7ED057A27EE277AD7ED047A67EE277A27
:10C8E000B7EE087A37EE677AD7ED047A67EE277AE3
:10C8F000C7ED047A3B6907EE903AB0EE670A1C3741
:10C90000BD465DF8047B7047DF59375F80B584B062
:10C9100000AF87ED030AC7ED020A87ED011A97ED14
:10C92000037AD7ED027A77EE676A97ED017AD7ED51
:10C93000027A77EE677AF0EE670AB0EE660AFBF7E6
:10C9400008F987ED030AD7ED037AF5EEC07AF1EE28
:10C9500010FA06D597ED037AD7ED017A77EE277AAC
:10C9600005E097ED037AD7ED027A77EE277AB0EEFD
:10C97000670A1037BD4680BD80B58AB000AF7860C9
:10C980000720F9F711FF02E06420F9F70DFFFCF72B
:10C9900033FA0346002B14BF01230023DBB2002B24
:10C9A000F2D107F108039FED5B0A1846FFF7A6FCDA
:10C9B000FCF7C8FF584B01221A7000BF4FF0FF313F
:10C9C0000120F9F79DF80346012B14BF0123002332
:10C9D000DBB2002BF2D1514B1B78DBB203F0040326
:10C9E000002B14BF01230023DBB2002B0CD04B4BD8
:10C9F0001B78DBB223F00403DAB2484B1A70484BC1
:10CA000048491846FCF784FE474B1B78DBB203F01D
:10CA10000403002B14BF01230023DBB2002B0DD035
:10CA2000414B1B78DBB223F00403DAB23E4B1A70A1
:10CA30003E4B3F4A3F491846FCF7F0FD3E4B1B7802
:10CA4000DBB203F00403002B14BF01230023DBB28D
:10CA5000002B0CD0384B1B78DBB223F00403DAB286
:10CA6000354B1A70354B36491846FCF7A4FD354B4B
:10CA7000D3ED057A334B93ED067A324BD3ED076A4B
:10CA8000304B93ED016A2F4BD3ED025A2D4B93EDB2
:10CA9000035A07F10803F0EE452AB0EE652AF0EEDE
:10CAA000461AB0EE661AF0EE470AB0EE670A18466C
:10CAB000FFF750FC07F10800234A244B244900F0FB
:10CAC00053F8244B93ED007A234BD3ED007A77EEA5
:10CAD000277A204BC3ED007A1D4B93ED007A1D4B56
:10CAE000D3ED007A77EE677A9FED1C1ADFED1C0A12
:10CAF000B0EE670AFFF70AFFF0EE407A144BC3ED81
:10CB0000007A184B1868002302220021F9F740F838
:10CB100053E700BF00007A44EF4D0020EC4D0020A9
:10CB2000D54D0020044E0020ED4D0020DE4D0020AC
:10CB3000104E0020F44D0020EE4D0020EA4D002064
:10CB4000004E0020F04D0020184E00201C4E00200A
:10CB5000144E0020D04D002040000020DB0F494043
:10CB6000DB0F49C0244A002080B584B000AFF860D4
:10CB7000B9607A603B60FB6893ED007AFB680C3328
:10CB8000D3ED007A27EE277AFB680433D3ED006AF1
:10CB9000FB680833D3ED007A66EEA77A77EE277A42
:10CBA00037EEA76AFB6893ED007AFB68D3ED007A55
:10CBB00027EE277AFB680433D3ED006AFB68043361
:10CBC000D3ED007A66EEA77A77EE277A77EEA77A2A
:10CBD000B7EE007A77EEC77AF0EE670AB0EE460A53
:10CBE00000F09CFEF0EE407ABB68C3ED007AFB6873
:10CBF000043393ED007AFB680C33D3ED007A27EE13
:10CC0000277AFB68D3ED006AFB680833D3ED007A1E
:10CC100066EEA77A77EE677AB8EE007A67EE877AE3
:10CC2000B0EE670A00F04EFEF0EE407A7B68C3ED8E
:10CC3000007AFB6893ED007AFB680433D3ED007A49
:10CC400027EE277AFB680833D3ED006AFB680C33C4
:10CC5000D3ED007A66EEA77A77EE277A37EEA76AE9
:10CC6000FB6893ED007AFB68D3ED007A27EE277A14
:10CC7000FB680C33D3ED006AFB680C33D3ED007A0C
:10CC800066EEA77A77EE277A77EEA77AB7EE007A84
:10CC900077EEC77AF0EE670AB0EE460A00F03EFE85
:10CCA000F0EE407A3B68C3ED007A00BF1037BD4616
:10CCB00080BD000080B582B000AF0346FB80FB88DA
:10CCC000102B1CD11B4B1B78DBB243F00103DAB2F3
:10CCD000184B1A70184B1B78DBB243F00103DAB221
:10CCE000154B1A70154B1B78DBB2002B14BF0123B8
:10CCF0000023DBB2002B19D000F024F816E0FB88EB
:10CD0000202B13D10E4B1B78DBB243F00103DAB2B8
:10CD10000B4B1A70094B1B78DBB2002B14BF01239D
:10CD20000023DBB2002B01D000F00CF800BF083765
:10CD3000BD4680BDED4D0020EE4D0020EF4D0020A2
:10CD4000EC4D002080B500AF694B1B78DBB203F0DF
:10CD50000103002B1FD0674B9B6C1B681B6803F003
:10CD60000103002B17D1634BDB6C1B681B6803F0BE
:10CD70000103002B0FD1604B1B78DBB203F00203E1
:10CD8000002B08D15D4B1B78DBB203F00203002BB4
:10CD900001D1012300E00023002B1BD0544B1B7852
:10CDA000DBB223F00103DAB2514B1A70504B1B78FF
:10CDB000DBB243F00203DAB24D4B1A7000220121BC
:10CDC0004F48F4F7FDFE4F4B4F4908221846FCF739
:10CDD000E5FD8BE0484B1B78DBB203F00103002B31
:10CDE0001FD0444B9B6C1B681B6803F00103002B96
:10CDF00017D1404BDB6C1B681B6803F00103002B51
:10CE00000FD13B4B1B78DBB203F00203002B08D1A0
:10CE10003A4B1B78DBB203F00203002B01D1012354
:10CE200000E00023002B1BD0334B1B78DBB223F038
:10CE30000103DAB2304B1A702F4B1B78DBB243F090
:10CE40000203DAB22C4B1A70002210212F48F4F79B
:10CE5000B7FE2F4B2F4909221846FCF79FFD45E0EE
:10CE6000264B1B78DBB203F00103002B1FD0214BB4
:10CE70009B6C1B681B6803F00103002B17D11D4B33
:10CE8000DB6C1B681B6803F00103002B0FD1184BF0
:10CE90001B78DBB203F00203002B08D1164B1B7882
:10CEA000DBB203F00203002B01D1012300E00023D9
:10CEB000002B1BD0114B1B78DBB223F00103DAB23D
:10CEC0000E4B1A700D4B1B78DBB243F00203DAB243
:10CED0000A4B1A70002210210C48F4F771FE0E4B19
:10CEE0000E4904221846FCF759FD00BF80BD00BF63
:10CEF000EC4D0020584A0020ED4D0020EE4D002062
:10CF00000004024044000020D44D002000000240F4
:10CF10004C000020DC4D002058000020E84D00208F
:10CF200080B500AF754BDB6C1B681A46744B9A4298
:10CF30006DD9744B5A68714BDB6C1B6872498B421C
:10CF400062D06E4BDB6C1B6870498B425AD06B4BC6
:10CF5000DB6C1B686E498B4252D0684BDB6C1B68E4
:10CF60006C498B424AD0654BDB6C1B686A498B422B
:10CF700041D0624BDB6C1B6868498B4238D05F4BF9
:10CF8000DB6C1B6866498B422FD05C4BDB6C1B68EB
:10CF900064498B4226D0594BDB6C1B6862498B423B
:10CFA0001DD0564BDB6C1B6860498B4214D0534B31
:10CFB000DB6C1B685E498B420BD0504BDB6C1B68F3
:10CFC0005C498B4202D14FF400131EE04FF0006326
:10CFD0001BE04FF4001318E04FF4001315E04FF47A
:10CFE000001312E04FF400630FE04FF400630CE015
:10CFF0004FF4006309E04FF4006306E0202304E0EF
:10D00000202302E0202300E02023134098E13B4B43
:10D01000DB6C1B681A46484B9A4240F28F80394BB2
:10D020001A68364BDB6C1B6837498B4262D0334B36
:10D03000DB6C1B6835498B425AD0304BDB6C1B686C
:10D0400033498B4252D02D4BDB6C1B6831498B42EC
:10D050004AD02A4BDB6C1B682F498B4241D0274BAF
:10D06000DB6C1B682D498B4238D0244BDB6C1B6872
:10D070002B498B422FD0214BDB6C1B6829498B42FB
:10D0800026D01E4BDB6C1B6827498B421DD01B4BE7
:10D09000DB6C1B6825498B4214D0184BDB6C1B687A
:10D0A00023498B420BD0154BDB6C1B6821498B420B
:10D0B00002D14FF400131EE04FF000631BE04FF469
:10D0C000001318E04FF4001315E04FF4001312E0C2
:10D0D0004FF400630FE04FF400630CE04FF4006383
:10D0E00009E04FF4006306E0202304E0202302E07F
:10D0F000202300E02023134022E100BF584A0020F3
:10D100005864024000640240106002401064024013
:10D11000706002407064024028600240286402404F
:10D1200088600240886402404060024040640240DF
:10D13000A0600240A0640240B8600240704BDB6C0B
:10D140001B681A466F4B9A426DD96F4B5A686C4BED
:10D15000DB6C1B686D498B4262D0694BDB6C1B68D2
:10D160006B498B425AD0664BDB6C1B6869498B421A
:10D1700052D0634BDB6C1B6867498B424AD0604BD3
:10D18000DB6C1B6865498B4241D05D4BDB6C1B68D7
:10D1900063498B4238D05A4BDB6C1B6861498B4228
:10D1A0002FD0574BDB6C1B685F498B4226D0544B0A
:10D1B000DB6C1B685D498B421DD0514BDB6C1B68DF
:10D1C0005B498B4214D04E4BDB6C1B6859498B4238
:10D1D0000BD04B4BDB6C1B6857498B4202D14FF491
:10D1E00000131EE04FF000631BE04FF4001318E043
:10D1F0004FF4001315E04FF4001312E04FF40063F6
:10D200000FE04FF400630CE04FF4006309E04FF4CB
:10D21000006306E0202304E0202302E0202300E056
:10D22000202313408CE0384B1A68354BDB6C1B68AD
:10D2300036498B4200F08280314BDB6C1B683449ED
:10D240008B425AD02E4BDB6C1B6832498B4252D03A
:10D250002B4BDB6C1B6830498B424AD0284BDB6C74
:10D260001B682E498B4241D0254BDB6C1B682C4937
:10D270008B4238D0224BDB6C1B682A498B422FD063
:10D280001F4BDB6C1B6828498B4226D01C4BDB6C88
:10D290001B6826498B421DD0194BDB6C1B68244947
:10D2A0008B4214D0164BDB6C1B6822498B420BD08F
:10D2B000134BDB6C1B6820498B4202D14FF40013E7
:10D2C0003DE04FF000633AE04FF4001337E04FF4D5
:10D2D000001334E04FF4001331E04FF400632EE00C
:10D2E0004FF400632BE04FF4006328E04FF4006339
:10D2F00025E0202323E0202321E020231FE000BF9E
:10D30000584A00205860024000600240106002400D
:10D310001064024070600240706402402860024065
:10D3200028640240886002408864024040600240F5
:10D3300040640240A0600240A064024020231340E9
:10D34000002B14BF01230023DBB2002B00F09682D8
:10D35000744BDB6C1B681A46734B9A426CD9714B49
:10D36000DB6C1B68714A934262D06E4BDB6C1B68AE
:10D370006F4A93425AD06B4BDB6C1B686D4A9342E9
:10D3800052D0684BDB6C1B686B4A93424AD0654BAA
:10D39000DB6C1B68694A934241D0624BDB6C1B68B3
:10D3A000674A934238D05F4BDB6C1B68654A9342F7
:10D3B0002FD05C4BDB6C1B68634A934226D0594BE1
:10D3C000DB6C1B68614A93421DD0564BDB6C1B68BB
:10D3D0005F4A934214D0534BDB6C1B685D4A934207
:10D3E0000BD0504BDB6C1B685B4A934202D14FF46D
:10D3F00000131EE04FF000631BE04FF4001318E031
:10D400004FF4001315E04FF4001312E04FF40063E3
:10D410000FE04FF400630CE04FF4006309E04FF4B9
:10D42000006306E0202304E0202302E0202300E044
:10D4300020234A4AD36094E13A4BDB6C1B681A46BE
:10D44000474B9A4240F28E80364BDB6C1B68374A62
:10D45000934262D0334BDB6C1B68354A93425AD0FF
:10D46000304BDB6C1B68334A934252D02D4BDB6C44
:10D470001B68314A93424AD02A4BDB6C1B682F4A07
:10D48000934241D0274BDB6C1B682D4A934238D026
:10D49000244BDB6C1B682B4A93422FD0214BDB6C57
:10D4A0001B68294A934226D01E4BDB6C1B68274A17
:10D4B00093421DD01B4BDB6C1B68254A934214D052
:10D4C000184BDB6C1B68234A93420BD0154BDB6C6B
:10D4D0001B68214A934202D14FF400131EE04FF023
:10D4E00000631BE04FF4001318E04FF4001315E045
:10D4F0004FF4001312E04FF400630FE04FF40063A9
:10D500000CE04FF4006309E04FF4006306E02023D1
:10D5100004E0202302E0202300E020230F4A936050
:10D520001FE100BF584A00205864024010600240CA
:10D530001064024070600240706402402860024043
:10D5400028640240886002408864024040600240D3
:10D5500040640240A0600240A064024000640240B7
:10D56000B86002406E4BDB6C1B681A466D4B9A42EA
:10D570006CD96B4BDB6C1B686B4A934262D0684B77
:10D58000DB6C1B68694A93425AD0654BDB6C1B68A5
:10D59000674A934252D0624BDB6C1B68654A9342E8
:10D5A0004AD05F4BDB6C1B68634A934241D05C4BB3
:10D5B000DB6C1B68614A934238D0594BDB6C1B68AB
:10D5C0005F4A93422FD0564BDB6C1B685D4A9342F7
:10D5D00026D0534BDB6C1B685B4A93421DD0504BEB
:10D5E000DB6C1B68594A934214D04D4BDB6C1B68B3
:10D5F000574A93420BD04A4BDB6C1B68554A934207
:10D6000002D14FF400131EE04FF000631BE04FF413
:10D61000001318E04FF4001315E04FF4001312E06C
:10D620004FF400630FE04FF400630CE04FF400632D
:10D6300009E04FF4006306E0202304E0202302E029
:10D64000202300E02023444AD3608AE0344BDB6C83
:10D650001B68354A934200F08180314BDB6C1B68BC
:10D66000324A93425AD02E4BDB6C1B68304A9342AD
:10D6700052D02B4BDB6C1B682E4A93424AD0284B6E
:10D68000DB6C1B682C4A934241D0254BDB6C1B683A
:10D690002A4A934238D0224BDB6C1B68284A9342BB
:10D6A0002FD01F4BDB6C1B68264A934226D01C4BA5
:10D6B000DB6C1B68244A93421DD0194BDB6C1B6842
:10D6C000224A934214D0164BDB6C1B68204A9342CB
:10D6D0000BD0134BDB6C1B681E4A934202D14FF4F4
:10D6E00000133CE04FF0006339E04FF4001336E0E4
:10D6F0004FF4001333E04FF4001330E04FF40063B5
:10D700002DE04FF400632AE04FF4006327E04FF46C
:10D71000006324E0202322E0202320E020231EE0D9
:10D72000584A0020586002401060024010640240D5
:10D730007060024070640240286002402864024029
:10D7400088600240886402404060024040640240B9
:10D75000A0600240A0640240006002402023484ACA
:10D760009360484B1B78DBB203F00203002B14BF1D
:10D7700001230023DBB2002B14D0424B1B78DBB219
:10D7800023F00203DAB23F4B1A703E4B1B78DBB238
:10D7900043F00403DAB23B4B1A70012201213A48EC
:10D7A000F4F70EFA394B1B78DBB203F00203002BBF
:10D7B00014BF01230023DBB2002B14D0334B1B78A2
:10D7C000DBB223F00203DAB2304B1A702F4B1B7816
:10D7D000DBB243F00403DAB22C4B1A7001221021A1
:10D7E0002B48F4F7EDF92B4B1B78DBB203F0020367
:10D7F000002B14BF01230023DBB2002B14D0254BD8
:10D800001B78DBB223F00203DAB2224B1A70214BF1
:10D810001B78DBB243F00403DAB21E4B1A7001220C
:10D8200010211B48F4F7CCF9FFF78CFA154B1B7845
:10D83000DBB203F00403002B14BF01230023DBB28F
:10D84000002B1BD0F8F7CEF80346012B14BF0123A1
:10D850000023DBB2002B11D00F4B1B680F49184679
:10D86000F8F750FA0D4B1B68002B07D00C4B4FF00C
:10D8700080521A60BFF34F8FBFF36F8F00BF80BD20
:10D8800000600240EC4D002000040240ED4D0020FD
:10D8900000000240EE4D0020204A0020204E0020D3
:10D8A00004ED00E080B483B000AF786039603B687D
:10D8B0009B007A68134418460C37BD465DF8047B1C
:10D8C0007047000008B52DED028BB0EE408A00F0E5
:10D8D00059F8B4EE488AF1EE10FAF0EE408A0AD612
:10D8E000B0EE480A00F040F8F7EE007AB4EEE70A2E
:10D8F000F1EE10FA04DCB0EE680ABDEC028B08BD54
:10D9000000F066FBBDEC028B034621221A60024840
:10D91000BDE8084000F030B84CE4000800F02EB933
:10D9200008B52DED028BF0EE408AB0EE608A00F073
:10D93000CDF9F4EE488AF1EE10FA06D6DFED098A49
:10D94000B4EE688AF1EE10FA02D0BDEC028B08BD8D
:10D9500000F03EFB88EEA80ABDEC028B2123036099
:10D9600008BD00BF0000000010EE103A23F0004395
:10D9700000EE103A704700BF9FED010A704700BFEC
:10D980000000C07F38B510EE105A25F00044B4F105
:10D990007E5F2DED048BF0EE407A7FD077D8B4F126
:10D9A0007C5F0ED2B4F1485F80F092809FED637A85
:10D9B00030EE077AF7EE006AB4EEE67AF1EE10FA8E
:10D9C00062DCB0EE670AFFF7CFFFF7EE007A37EEC2
:10D9D000C08AB6EE007A28EE078ADFED596A9FED1D
:10D9E000597A9FED596A9FED595ADFED595ADFED8B
:10D9F000598AE8EE076A9FED587AA8EE067A9FEDFD
:10DA0000576AA6EE885AA7EE086A9FED557ADFEDB1
:10DA1000556AE5EE085AA6EE087AE5EE886AE7EE62
:10DA2000087AE6EE888AB0EE480AB0EE679A00F00F
:10DA3000C3FA4D4B9C4268EE888A3AD810EE103AF1
:10DA40006FF30B0306EE903AA6EEE68A70EE267AA6
:10DA500088EE895AC8EE274A9FED447ADFED447A72
:10DA6000B0EE006AA4EEC67A30EE000AF0EE675A15
:10DA700090EE057AE6EEC65A37EE657A37EEC70ABB
:10DA8000002D01DCB1EE400ABDEC048B38BDBDECCD
:10DA9000048B70EE407A87EEA70A38BDBDEC048B8C
:10DAA0009FED320A9FED337A27EE800AA7EE870AB0
:10DAB00038BD88EE896A9FED307ADFED2E7AA0EED0
:10DAC000060AF0EE006AA0EE267A37EEC70AD7E71C
:10DAD00020EE007ADFED1B6A9FED196ADFED1B5A1D
:10DAE0009FED195ADFED1A4AA7EE266ABDEC048BAA
:10DAF000E6EE075ADFED186A9FED186AE7EE056A51
:10DB0000E5EE874AA6EE876A9FED165ADFED145AB6
:10DB1000DFED106AA4EE875AE6EE075AE5EE076AD3
:10DB2000B7EE006AA5EE876A26EE877AC7EE066A28
:10DB3000E0EE267AB0EE670A38BD00BFCAF249713E
:10DB4000047F4F3A08EF11382EC69D3D461124BD83
:10DB5000A80A4E3EABAA2A3E613330BF2D57014082
:10DB600039D119C090B0A6BE9999793F2EBD3BB36B
:10DB7000DB0F493FDB0FC93F2EBD3B3310B582B0F1
:10DB8000CDED010A019B23F00042B2F1FF4FF0EE10
:10DB9000407A30D810EE100A20F00041B1F1FF4F6A
:10DBA00029D8B3F17E5F42D09C1704F0020444EA06
:10DBB000D07431B37AB3B2F1FF4F40D0B1F1FF4F1F
:10DBC00029D0891AB1F1F45F4FEAE15234DA002B1F
:10DBD00042DA3C3240DA9FED340A012C4ED0022C5E
:10DBE00043D064B19FED317ADFED317A30EE070A30
:10DBF00030EE670A03E09DED017A37EE270A02B0A6
:10DC000010BD022C10D09FED2B7A032C08BFB0EE74
:10DC1000470A02B010BD9FED280ADFED287A0028E0
:10DC2000A8BFB0EE670AEAE79FED210AE7E702B076
:10DC3000BDE8104000F0EAB89FED200ACDE7B1F151
:10DC4000FF4F04F1FF3420D0022C26D81C4B03EBED
:10DC5000840393ED000AD2E79DED017A87EE870AEF
:10DC6000FFF782FE00F0D2F8B7E79FED107ADFED04
:10DC7000107A30EE070A37EEC00AC0E710EE103A0D
:10DC800003F1004300EE103AB9E7022C08D80D4B1F
:10DC900003EB840393ED000AB1E79FED030AAEE7BF
:10DCA0009FED090AABE700BF000000002EBDBB33AB
:10DCB000DB0F4940DB0F49C0DB0FC9BFDB0FC93F9A
:10DCC00050E400085CE40008DB0F493F30B583B046
:10DCD000CDED010A019A22F0004E0EF1FF33B3F1AF
:10DCE000FF4F42D210EE104A24F00040B0F1FF4F37
:10DCF0003BD270453FDB04F000413ED014F0FF4FB3
:10DD000002F0FF4558D14FEA002C6FF07D034FEA37
:10DD10004C0CBCF1000F03F1FF33F8DC002D5CD19B
:10DD20004FEA0E226FF07D0C52000CF1FF3CFBD548
:10DD300013F17E0F63DA6FF07D02D21A90406FF01C
:10DD40007D02A2EB0C020EFA02F2B3EB0C0305D13A
:10DD50001AE012D04FEA4E00013B15D0A0EB020EA4
:10DD6000BEF1000FF5DA4000F6E7DDED017A60EE76
:10DD7000277A87EEA70A03B030BD234B03EB51731C
:10DD800093ED000A03B030BD831A48BF03461BB9A8
:10DD9000F3E75B000CF1FF3CB3F5000FF9DB1CF17E
:10DDA0007E0F23DBA3F500030CF17F0C0B4343EA4A
:10DDB000CC5300EE103ADEE7C3157F3B002DAFD009
:10DDC0004FEAEE5EC4F31604AEF17F0C44F400009B
:10DDD000C2F3160242F40002B7E76FF07D044FEA87
:10DDE000EE5EE41AAEF17F0CA040F1E76FF07D0229
:10DDF000A2EB0C0213410B4300EE103ABBE7C4F355
:10DE0000160444F400009AE768E4000838B510EE00
:10DE1000105A25F00044B4F1A14FF0EE407A0DD332
:10DE2000B4F1FF4F5BD8DFED517A9FED517A002DB1
:10DE3000CCBFB0EE470AB0EE670A38BD4D4B9C42EE
:10DE40005CD8B4F1445F4DD34FF0FF3327EEA76A9F
:10DE50009FED495A9FED497ADFED495ADFED494A76
:10DE600066EE066A5A1CA6EE857AE6EEA54A9FED96
:10DE7000465ADFED465AA7EE265AE4EEA65A9FED23
:10DE8000447ADFED444AA5EE267AE5EEA64A9FEDF8
:10DE9000425ADFED425AA7EE265A9FED417AA4EE90
:10DEA000A67AE5EE265A27EE267AA5EE867A27EEA2
:10DEB000877A38D03B493C4A01EB8301D1ED006AB7
:10DEC00037EE667A02EB8303D3ED006A37EE677AAA
:10DED000002D36EEC70AB0DAB1EE400A38BD30EE9A
:10DEE000000A38BD9FED317A30EE077AF7EE006A0E
:10DEF000B4EEE67AF1EE10FAA6DD38BDFFF734FD98
:10DF00002B4B9C4212D8A3F5D0039C4223D8F0EEB1
:10DF1000007ABFEE007AA0EE277A002330EE270ABF
:10DF2000C7EE007A92E737EEC70A38BD214B9C4214
:10DF30000BD8F7EE087AB7EE007AA0EE277A022324
:10DF400030EE670AC0EE077A80E7BFEE007AC7EED0
:10DF5000007A03237AE7F7EE007A30EE677A30EE44
:10DF6000270A0123C7EE007A70E700BFDB0FC9BFA5
:10DF7000DB0FC93FFFFFDF3ED769853C59DA4B3DD8
:10DF800021A215BD6BF16EBD356B883D95879DBD9A
:10DF90006E2EBA3D388EE3BD2549123EABAAAA3E8D
:10DFA000CDCC4CBE70E4000880E40008CAF2497190
:10DFB000FFFF973FFFFF1B40B1EEC00A704700BF55
:10DFC00002440346934200D1704703F8011BF9E76E
:10DFD000014B1868704700BF5C00002070B50D4D04
:10DFE0000D4C641BA4100026A64209D10B4D0C4C0D
:10DFF00000F084F9641BA4100026A64205D170BD70
:10E0000055F8043B98470136EEE755F8043B98472E
:10E010000136F2E798E4000898E4000898E4000864
:10E02000A0E400080A44914200F1FF3300D1704798
:10E0300010B511F8014B03F8014F9142F9D110BD11
:10E040002DE9F047089D0E4604460F46002B4AD1A5
:10E0500094468C45B2FA82F260D942B1C2F12003F3
:10E06000974020FA03F30CFA02FC1F4394404FEA56
:10E070001C4E1FFA8CF6B7FBFEF1230C0EFB11773A
:10E0800043EA074301FB06F098420AD91CEB03035D
:10E0900001F1FF3780F01581984240F21281023978
:10E0A00063441B1AA4B2B3FBFEF00EFB103344EA28
:10E0B000034400FB06F6A6420AD91CEB040400F157
:10E0C000FF3380F00081A64240F2FD8064440238B4
:10E0D00040EA0140A41B00211DB1D4400023C5E942
:10E0E0000043BDE8F0878B4205D90DB1C5E90001B9
:10E0F00000210846F5E7B3FA83F1002946D1B3427F
:10E1000002D3824200F2F580841A66EB03020120FA
:10E110001746002DE5D0C5E90047E2E7002A40F0A8
:10E120009380A1EB0C034FEA1C471FFA8CFE0121E0
:10E13000B3FBF7F607FB1630230C43EA00430EFB54
:10E1400006F0984208D91CEB030306F1FF3802D20F
:10E15000984200F2D08046461B1AA4B2B3FBF7F0F7
:10E1600007FB103344EA03440EFB00FEA64508D922
:10E170001CEB040400F1FF3302D2A64500F2B68086
:10E180001846A4EB0E0440EA0640A5E7C1F12007BB
:10E190008B4022FA07FC4CEA030C06FA01FE20FA37
:10E1A00007F426FA07F344EA0E0400FA01F84FEAEE
:10E1B0001C404FEA1449B3FBF0FE1FFA8CF600FB3B
:10E1C0001E3349EA03430EFB06F9994502FA01F2B0
:10E1D0000BD91CEB03030EF1FF3A80F085809945C3
:10E1E00040F28280AEF1020E6344A3EB0909A4B2AF
:10E1F000B9FBF0F300FB139944EA094403FB06F66C
:10E20000A64208D91CEB040403F1FF3068D2A642F1
:10E2100066D9023B644443EA0E40A41BA0FB02E61D
:10E22000B4427346B14652D34FD05DB1B8EB03024E
:10E2300064EB090404FA07F722FA01F31F43CC4008
:10E24000C5E9007400214CE7C2F1200120FA01F376
:10E250000CFA02FC26FA01F1964033434FEA1C47C0
:10E260001FFA8CFEB1FBF7F007FB1016190C41EA00
:10E27000064100FB0EF68E4204FA02F408D91CEBAC
:10E28000010100F1FF382DD28E422BD902386144B2
:10E29000891B9BB2B1FBF7F607FB161143EA01435A
:10E2A00006FB0EF1994208D91CEB030306F1FF3877
:10E2B00014D2994212D9023E63445B1A46EA0041E5
:10E2C00036E73946EDE6184602E7F045ADD2BEEB3B
:10E2D000020366EB0C060138B146A6E74646ECE7BA
:10E2E000034698E74046D3E7D6467EE764440238C3
:10E2F00047E708460DE7023E63442DE7F8B500BF47
:10E30000F8BC08BC9E467047F8B500BFF8BC08BC16
:04E310009E4670476E
:10E3140049444C4500000000546D7220537663005C
:10E32400546D725100000000446562756754617356
:10E334006B000000496E730047696D62616C546143
:10E34400736B00005472616E736D69745461736B06
:10E3540000000000526563656976655461736B0063
:10E364000000000000000000010203040607080981
:10E374000000000001020304000610160006101637
:10E384002CE3000800000000000000000000000072
:10E39400000000000002000018000000000000005F
:10E3A4000000000038E30008000000000000000046
:10E3B4000000000000000000000200003000000027
:10E3C40000000000000000003CE300080000000022
:10E3D4000000000000000000000000000004000035
:10E3E40018000000000000000000000048E30008DE
:10E3F4000000000000000000000000000000000019
:10E4040000040000180000000000000000000000EC
:10E4140058E30008000000000000000000000000B5
:10E4240000000000000400001800000000000000CC
:10E434000000000040AC037D04014103057C0002A0
:10E444006D0D026D09020000000000000000008054
:10E45400DB0F4940DB0F49C0DB0F49BFE4CB16405B
:10E46400E4CB16C000000000000000806937AC3126
:10E4740068212233B40F14336821A2333863ED3E8C
:0CE48400DA0F493F5E987B3FDA0FC93F7A
:08E49000B0FBFF7F010000005A
:08E498002D020008A98600080E
:04E4A0000502000869
:10E4A4000024F4001000000001000000AAAAAAAA97
:10E4B400E7416B3A58A08B3A7D04017C000240ABE3
:10E4C4000341000553080658040700000F00081014
:10E4D400820911000A15800B16000C18010D0000AA
:10E4E4008B8803B582FFFFFFFFFFFFFF92FFFFFF53
:10E4F400FFFFFFFFFF000000A2FFFFFF60000020FE
:10E5040000000000244E00208C4E0020F44E002019
:10E5140000000000000000000000000000000000F7
:10E5240000000000000000000000000000000000E7
:10E5340000000000000000000000000000000000D7
:0CE54400000000000000000000000000CB
:0400000508007AA1D4
:00000001FF
